:100000000C94A60E0C94CD860C94D70E0C94D70E9F
:100010000C94D70E0C9487520C94A79E0C94D70E78
:100020000C94D70E0C94D70E0C94D70E0C94D70EBC
:100030000C94D70E0C94D70E0C94D70E0C94D70EAC
:100040000C94D70E0C9440410C940B520C94D70E88
:100050000C94D70E0C94D70E0C94D70E0C94BF842E
:100060000C94D70E0C94024A0C94D9490C94D70ED8
:100070000C94D70E0C94D70E0C94D70E0C94D70E6C
:100080000C94BB920C94D70E0C94D70E0C94D70EF4
:100090000C94B0490C9487490C94D70E0C94D70E4D
:1000A0000C94D70E0C94D70E0C94D70E0C94D70E3C
:1000B0000C94D70E0C947B880C94D70E0C94D70E0E
:1000C0000C94D70E0C94D70E0C94D70E0C945E495A
:1000D0000C9435490C94D70E0C940C490C94E348BD
:1000E0000C94D70EC01BC31BCA1BCD1BD01BD31B2C
:1000F000DA1BE11BE41BEB1BF21BF91B9D21CB213F
:100100000222392214234B237923A7236E246E2441
:100110006E246E246E246E246E246E246E246E244F
:100120006E246E246E246E246E246E246E246E243F
:100130006E246E246E246E246E246E246E246E242F
:100140006E246E246E247022A722DF22D52303247E
:100150003B246C26722678267E2684268A269026C4
:1001600096269C26A226A826AE26C026C626CC26E3
:10017000E426EA26F026F626FC26022708270E2784
:1001800014271A27202726272C2732273E274A27DD
:10019000502756275C2774277A27802786278C27A5
:1001A0009227822888288E28A028A628AC28BE2836
:1001B000C428CA28D028D628DC2806290C293629A4
:1001C0003C2942294829602966296C297229072A75
:1001D000072A072A072A072A072A072A072A882917
:1001E0008C29902996299A299E29A229A629AA29EB
:1001F000AE29B429D229D829DE29622798279E273B
:10020000A427AA27B027B6274E2954295A29782986
:100210007E298429E429EA29F029E228E828BC2754
:10022000C227C827CE27D427DA279428B228442704
:10023000B426BA2668276E27F629FC29022A382711
:10024000122918291E2924292A293029E027E627DE
:10025000EC27F227F827FE2704280A28102816285A
:100260001C28222828282E2834283A2840284628C6
:10027000522858285E2864286A28702876287C2806
:10028000C629C029BA29CC299A28B828D226D82626
:10029000DE26EE284C28F428FA280029E230BF3068
:1002A0009830FF3056311E314D313C310732EA3142
:1002B000C33157322432243246322F32ED38ED38F2
:1002C000FC38ED38093922393D395839AF45B24546
:1002D000A145A545AB45E945B645BA45C045C44528
:1002E000C845CE45D245D645E945DC45E045E4451F
:1002F0006C4B714B764B804B8A4B034C944B9C4B15
:10030000A44BAE4BB84BC24BD14BDB4B034CE54B34
:10031000EF4BF94BD962DD62E162E562E962ED62C1
:10032000F162F562F962FD6201632D633163386346
:1003300045635263656378639163AA63C863DE6350
:1003400051688568BA68DA680F6977698769B16A40
:10035000FB69056A396A6E6A7C6AB16A4369AA8870
:10036000B388BB88CF88E188F388FE88909AA79AE3
:10037000BE9AD59AEC9A1A9B319B489B5F9B7E9BB9
:10038000969BAD9BCC9BE29B039B05A84CCDB2D426
:100390004EB93836A9020C50B9918688083CA6AAF5
:1003A000AA2ABE000000803F3400330032004E6FA6
:1003B0006E650053746F70706564004E657574727D
:1003C000616C205475726E004D6F76696E672052B5
:1003D000657665727365004D6F76696E6720466F4E
:1003E0007277617264004272616B696E670054419A
:1003F0004E4B20524553544F52454400250048650A
:10040000616C7468204C6576656C3A2000564548EE
:1004100049434C452052455041495220434F4D508D
:100420004C4554450054414E4B2044455354524F83
:100430005945440025004865616C7468204C657618
:10044000656C3A2000290056454849434C452052E6
:1004500045504149522053544152544544202800AC
:10046000524550414952204F5045524154494F4EF8
:100470002043414E43454C4C45440029004D4143E7
:1004800048494E452047554E2048495421202800D0
:10049000524550414952204F5045524154494F4EC8
:1004A0002043414E43454C4C454400290043414EB6
:1004B0004E4F4E20484954212028005475727265D1
:1004C0007420726F746174696F6E206973206E6F2F
:1004D00074206F66207479706520536572766F2E74
:1004E000204E6F20736574757020617661696C6150
:1004F000626C652E004E6F207374656572696E675D
:1005000020736572766F2061737369676E65642C02
:100510002072652D636865636B2076656869636C1E
:100520006520747970652E0054757272657420654B
:100530006C65766174696F6E206973206E6F7420CC
:100540006F66207479706520536572766F2E204E29
:100550006F20736574757020617661696C61626C7F
:10056000652E00546F70204C65667400546F7020C7
:1005700043656E74657200546F70205269676874C9
:10058000004D6964646C65204C656674004D696457
:10059000646C652043656E746572004D6964646CBB
:1005A0006520526967687400426F74746F6D204CE7
:1005B00065667400426F74746F6D2043656E746578
:1005C0007200426F74746F6D2052696768740046E0
:1005D00049524D574152452056455253494F4E3A84
:1005E00020006942757300534275730050504D00EE
:1005F0004E6F6E6520446574656374656400417A6E
:10060000696D7574682020202000456C65766174E2
:10061000696F6E2020005475726E202020202020EB
:1006200020005468726F74746C652020200053742D
:1006300069636B202020202020204D696E2020201F
:100640002043656E7465722020204D617820202043
:10065000204465616462616E642020526576657233
:1006600073656400524144494F20494E464F202D46
:1006700020004E4F542044455445435445440049BE
:10068000474E4F52454400416E616C6F67004469AC
:10069000676974616C00417578204368616E2E2033
:1006A00020204D696E20202020204D6178202020C0
:1006B000202054797065004368616E6E656C73200C
:1006C0007574696C697A65643A20004368616E6E7E
:1006D000656C732064657465637465643A200020FA
:1006E0002844697361626C656429002028456E6145
:1006F000626C656429004D656368616E6963616C55
:10070000207265636F696C00416972736F66740073
:100710004D656368616E6963616C204261727265E8
:100720006C3A200020284D31290020284D32290024
:10073000202842290042617272656C20456C657602
:100740006174696F6E3A20200020284D3029002006
:10075000284D312900202841290054757272657492
:1007600020526F746174696F6E3A2020200020411E
:100770006D70732900202843757272656E74204C69
:10078000696D69743A20004472697665204D6F7412
:100790006F72733A202020202020004D4F544F527A
:1007A00020545950455300496E646570656E646508
:1007B0006E7420547265616420436F6E74726F6C46
:1007C0000054616E6B202854616D69796120444D3D
:1007D00044290054616E6B2028444B4C4D204765E2
:1007E0006172626F7829004361720048616C6674BF
:1007F0007261636B0054616E6B00554E4B4E4F57E8
:100800004E00596573004E6F002900252C20446569
:1008100063656C65726174696F6E20666163746F85
:1008200072200020284B69636B6261636B207370D8
:100830006565642000547261636B205265636F6963
:100840006C20456E61626C65643A202020004E2F5A
:100850004120666F722076656869636C65207479E3
:100860007065005475726E204D6F64653A202020CB
:10087000202020202020202020202000250053742C
:10088000656572696E672050637420746F2074729E
:10089000656164733A20004E2F4120666F722076A6
:1008A000656869636C6520747970650059657320AB
:1008B0002854616D69796129002500202D20004EA2
:1008C00065757472616C205475726E20416C6C6F2A
:1008D0007765643A202020002073656300547261BC
:1008E0006E736D697373696F6E2044656C61793ADC
:1008F0002020202020002073656300456E67696E0C
:10090000652050617573652054696D653A2020201B
:1009100020202000207365630053686966742054AA
:10092000696D653A202020202020202020202020D2
:1009300020004175746F6D61746963004D616E755F
:10094000616C005472616E736D697373696F6E20B0
:10095000547970653A202020202020002500596518
:1009600073202D2000526576657273652053706583
:100970006564204C696D697465643A202000250027
:10098000596573202D2000466F7277617264205381
:1009900070656564204C696D697465643A20200057
:1009A000206D73290025207468726F74746C652043
:1009B000666F7220002028004D6F746F72204E7594
:1009C00064676520456E61626C65643A2020202072
:1009D0000029004E6F6E65004E6F6E65002C205032
:1009E00072657365743A20002900202841646A7595
:1009F0007374656420746F200020284C6576656CE4
:100A00003A2000446563656C2052616D7020456E2C
:100A100061626C65643A20202020200029004E6F1E
:100A20006E65004E6F6E65002C20507265736574A4
:100A30003A20002900202841646A75737465642097
:100A4000746F200020284C6576656C3A2000416365
:100A500063656C2052616D7020456E61626C6564E7
:100A60003A2020202020004163746976652044727A
:100A70006976696E672050726F66696C653A20000E
:100A800056656869636C6520547970653A2020204A
:100A90002020202020202020004452495645205369
:100AA000455454494E4753002073656300526563B3
:100AB0006F696C2064656C61793A202020202020C9
:100AC0002020202020202020202020202000250061
:100AD000596573202D200042617272656C20456C4F
:100AE00065766174696F6E205370656564204C692A
:100AF0006D697465643A20002500596573202D20C6
:100B00000054757272657420526F746174696F6EEF
:100B1000205370656564204C696D697465643A2082
:100B200020005455525245542053455454494E4781
:100B30005300556E6B6E6F776E0045787065726905
:100B40006D656E74616C00536570617261746520CF
:100B50004865617420262046616E00436F6D6269AE
:100B60006E6564204865617420262046616E00250C
:100B70000044697361626C656400536D6F6B65203E
:100B80007768656E2064657374726F7965643A2066
:100B90000046616E206D61782073706565643A204F
:100BA000202020202020200046616E206661737482
:100BB0002069646C652073706565643A2020004686
:100BC000616E2069646C652073706565643A2020ED
:100BD000202020202000202863757272656E746CBE
:100BE000792064697361626C6564290020736563B0
:100BF0006F6E6473004E2F41005072652D68656101
:100C0000742064656C61793A202020202020200027
:100C1000536D6F6B657220547970653A20202020E7
:100C200020202020202000536D6F6B6572206F758F
:100C30007470757420636F6E74726F6C6C65642071
:100C40006D616E75616C6C7900534D4F4B45520070
:100C5000556E6B6E6F776E004865617679004D65F5
:100C60006469756D004C6967687400437573746FCF
:100C70006D00556E6B6E6F776E004E6F6E65004F38
:100C800070656E2050616E7A65720054616D69798D
:100C90006120537065630020736563207265636F24
:100CA000766572792900207365632072656C6F61C7
:100CB000642C2000204D4720686974732C2000208C
:100CC00063616E6E6F6E20686974732C200028005B
:100CD00057656967687420436C6173733A202020FC
:100CE00020200044616D6167652050726F66696CF9
:100CF000653A202020005965732028004163636510
:100D00007074204D472044616D6167653A20005939
:100D1000657320280053656E64204D47204952209A
:100D2000436F64653A2020004E2F41005265706188
:100D3000697265642062793A202020202020004ECC
:100D40002F41004869742050726F746F636F6C207C
:100D5000323A20202000290020285465616D2000AF
:100D6000466972652050726F746F636F6C3A202011
:100D7000202000466972652050726F746F636F6C3B
:100D80003A2020202000497320526570616972204A
:100D900054616E6B3F202020004952202620546170
:100DA0006E6B20426174746C696E67204469736174
:100DB000626C656400424154544C4520494E464F94
:100DC00000554E4B4E4F574E0042656E6564696E3E
:100DD0006920544253204D6963726F004265696512
:100DE000722055534D2D52432D3200546169676571
:100DF0006E20536F756E642043617264004F70659E
:100E00006E2050616E7A657220536F756E64204358
:100E10006172640042656E6564696E692054425374
:100E2000204D696E6900536F756E64206361726452
:100E30003A2000534F554E44204341524400556ED2
:100E40006B6E6F776E0042617272656C20456C65E7
:100E5000766174696F6E20436F6D6D616E640054CE
:100E6000757272657420526F746174696F6E20437D
:100E70006F6D6D616E64005374656572696E672095
:100E8000436F6D6D616E640056656869636C6520C3
:100E9000537065656400456E67696E6520537065C3
:100EA0006564005468726F74746C6520436F6D6D77
:100EB000616E64005370656564206465637265618A
:100EC0007365732062656C6F77200053706565648D
:100ED00020696E637265617365732061626F766508
:100EE00020005475726E2053746F70706564004CEE
:100EF000656674205475726E2053746172746564F3
:100F0000005269676874205475726E205374617260
:100F10007465640056656869636C652053746F700E
:100F2000706564004D6F76696E67205265766572F4
:100F30007365004D6F76696E6720466F72776172D8
:100F40006400456E67696E652053746F7000456E6E
:100F500067696E652053746172740043616E6E6FD1
:100F60006E2052656C6F61646564005665686963E4
:100F70006C652044657374726F7965640043616EBB
:100F80006E6F6E20486974004272616B6573204118
:100F900070706C696564005661726961626C6500AD
:100FA000290020286F662000506F7320004175785B
:100FB000204368616E6E656C2000566172696162E3
:100FC0006C65004F6E004F66660042004100457838
:100FD0007465726E616C20496E707574200007082C
:100FE00009090B0C0C0B0C0C5475727265742053B0
:100FF0007469636B202D200046756E6374696F6E93
:10100000202300202D3E200020736563005475725C
:10101000726574206D6F76656D656E742064656CA5
:1010200061793A2020004E6F6E6500596573005457
:10103000757272657420737469636B2066756E6374
:1010400074696F6E733A200046554E4354494F4EB3
:101050002054524947474552530076206375746FB8
:10106000666629002028004C564320456E61626C5C
:1010700065643A202020202020007600566F6C7492
:101080006167653A20202020202020202020005960
:101090006573004E6F004261747465727920446517
:1010A0007465637465643A20004241545445525952
:1010B0000053657269616C20332054782042617559
:1010C000643A2020004175782053657269616C2074
:1010D000426175643A202020004D6F746F72205376
:1010E000657269616C20426175643A200055534213
:1010F0002053657269616C20426175643A2020203A
:10110000004241554420524154455300212000469D
:101110004143544F52592052455345542120000019
:10112000002100240027002A002D00300033000198
:10113000010000040107010A010000220025002827
:10114000002B002E003100340002010000050108D0
:10115000010B01000020002300260029002C002F95
:101160000032000001000003010601090105050528
:1011700005070508080808020202020A0A0808040E
:10118000040404010101010101010103030303033C
:10119000030303040707070C0C0C0C0C0C0C0C02CB
:1011A00002020206060606060606060B0B0B0B0BD2
:1011B0000B0B0B01021020200808102040102040CB
:1011C000800201020108040201010204081020400B
:1011D0008080402010080402018004020180402029
:1011E0001008040201080402010102040810204052
:1011F00080010204081020408000000A0B02090C44
:101200000D0E0807030401000000000000000000AC
:1012100000000000000000000000000000000000CE
:10122000000000000012111000000000000000008B
:101230000000000000000000000000000000005559
:101240006E6B6E6F776E004F6E626F617264204DD1
:101250006F746F7220447269766572732043202622
:1012600020440044657461636865642F4E410052F8
:1012700065636F696C20536572766F0050616E20F4
:10128000536572766F00536572766F2F4553430036
:101290004F6E626F617264204D6F746F7220447282
:1012A00069766572004F70656E2050616E7A657266
:1012B0002053636F75742053657269616C204553C8
:1012C00043005361626572746F6F74682053657276
:1012D00069616C00506F6C6F6C7520536572696149
:1012E0006C00536572766F203100536572766F2003
:1012F0003200536572766F203300536572766F202B
:101300003400536572766F203500536572766F2016
:101310003600536572766F203700536572766F2002
:101320003800494F20506F72742042202D20507594
:101330006C73656400494F20506F72742042202DF9
:1013400020537461727420426C696E6B696E670021
:10135000557365722046756E6374696F6E20310037
:10136000557365722046756E6374696F6E20320026
:10137000466F72776172642047656172004E6575D1
:101380007472616C20476561720052657665727394
:101390006520476561720053657420416363656C25
:1013A0002052616D70204C6576656C3A2000536563
:1013B0007420446563656C2052616D70204C6576C5
:1013C000656C3A2000416E616C6F672055736572E1
:1013D0002046756E6374696F6E2031202D200041A8
:1013E0006E616C6F6720557365722046756E63740D
:1013F000696F6E2032202D20002D00202D2000202E
:1014000000545255450046414C5345002500576154
:101410006974696E6720666F7220726164696F2EED
:101420002E2E200020287769746820495229004612
:101430006972652043616E6E6F6E00466972652049
:10144000526570616972205369676E616C00416911
:1014500072736F6674202D204D616E75616C20541F
:10146000726967676572004D656368616E69636183
:101470006C205265636F696C202D204D616E756123
:101480006C205472696767657200536572766F20CD
:101490005265636F696C202D204D616E75616C2003
:1014A00054726967676572004869676820496E749D
:1014B000656E7369747920466C61736820556E6936
:1014C00074202D204D616E75616C205472696767C0
:1014D0006572004D47205374617274004D4720536C
:1014E000746F70004952204E4F5420656E61626CDB
:1014F0006564202D206E6F2049522070726F746FCA
:10150000636F6C732073656C65637465642E00553E
:101510006E61626C6520746F20656E61626C65201F
:10152000495200495220656E61626C6564004952FF
:101530002064697361626C656400417578204F7541
:101540007470757420466C617368656400417578C9
:10155000204F757470757420496E766572736520BE
:10156000466C61736865640053746F7020417578D0
:10157000204F757470757420426C696E6B696E676C
:101580000053746F70205265766F6C76696E6720B9
:10159000417578204C696768740053746F702041FE
:1015A0006C6C205573657220536F756E64730049BF
:1015B0004F20506F72742041202D2050756C736540
:1015C0006400494F20506F72742041202D205374C5
:1015D00061727420426C696E6B696E67004169725A
:1015E000736F6674202D2044697361626C656400BA
:1015F0004D656368616E6963616C205265636F69F4
:101600006C202D2044697361626C656400436F6DCA
:101610006D73206368616E67656420746F20555335
:101620004200436F6D6D73206368616E676564206F
:10163000746F2053657269616C2031004472697661
:10164000696E672050726F66696C652073657420DF
:10165000746F2023002500537065656420726564F3
:101660007563656420746F20005370656564207233
:101670006573746F726564005475726E20456E6791
:10168000696E65204F6E00207365636F6E64732012
:1016900061676F202D20736D6F6B657220707265AE
:1016A0006865617420736B697070656400456E676E
:1016B000696E65206C6173742073746F70706564FB
:1016C0002000207365636F6E647300536D6F6B65EC
:1016D00072207072652D6865617420737461727414
:1016E0006564202D20656E67696E652077696C6C76
:1016F000207475726E206F6E20696E20004D616ED1
:1017000075616C207472616E736D697373696F6E4D
:10171000202D2070757420696E206E65757472615D
:101720006C2067656172206265666F7265207374F4
:10173000617274696E6720656E67696E6521004528
:101740006E67696E65204175746F205368757464A7
:101750006F776E00456E67616765205472616E73C6
:101760006D697373696F6E00446973656E67616755
:1017700065205472616E736D697373696F6E005387
:101780006574205475726E204D6F64653A20310087
:10179000536574205475726E204D6F64653A203223
:1017A00000536574205475726E204D6F64653A2045
:1017B0003300456E61626C65204E65757472616CB4
:1017C000205475726E730044697361626C65204EBB
:1017D00065757472616C205475726E7300401F7071
:1017E00017D007A00FA00FDC05D007C40910278869
:1017F00013983A102758026C0258026C0258026C77
:101800000258026C0258026C0258026C0258026CB8
:101810000258026C025802B0366C023A026C023A6C
:10182000026C023A026C02B036384A5C121C255C2B
:10183000125C121C255C12BC7FC7F2C07887A5B76A
:10184000C5A00F8813B80B401FB80BB80B7017401A
:101850001F494F20506F72742041204F757470756E
:1018600074202D204F6E00494F20506F727420411C
:10187000204F7574707574202D204F666600494F97
:1018800020506F72742042204F7574707574202D33
:10189000204F6E00494F20506F72742042204F75C8
:1018A00074707574202D204F6666004C5643204599
:1018B000786974202D20566F6C74616765205265BD
:1018C00073746F726564007629004C564320746807
:1018D000726573686F6C642072656163686564210A
:1018E0002028004C696768742031204F6E004C69D5
:1018F0006768742031204F6666004C696768742001
:1019000032204F6E004C696768742032204F666643
:1019100000326E64204D472053746F7000326E6445
:10192000204D472053746172740052756E6E696E5B
:1019300067204C6967687473204F6E0052756E6E35
:10194000696E67204C6967687473204F6666004152
:101950007578204F7574707574204F6E00417578DE
:10196000204F7574707574204F66660053746F70E5
:10197000205265766F6C76696E6720417578204CD1
:10198000696768740053746F7020417578204F75D3
:101990007470757420426C696E6B696E6700417576
:1019A00078204F757470757420507265736574205B
:1019B00044696D00537461727420417578204F75CD
:1019C0007470757420426C696E6B696E6700526149
:1019D00064696F205265616479202D20005265761C
:1019E00065727365643A2020004D61782050756CF3
:1019F00073653A20004D696E2050756C73653A200E
:101A000000456E642056616C75657300456E6420F8
:101A10005265636F696C20536572766F20536574ED
:101A2000757000456E6420526F746174696F6E202A
:101A3000536572766F20536574757000456E64202F
:101A40005374656572696E6720536572766F2053B3
:101A50006574757000456E64205374656572696EB7
:101A60006720536572766F20536574757000456EFC
:101A70006420456C65766174696F6E20536572767B
:101A80006F20536574757000536572766F20756EA4
:101A90002D726576657273656400536572766F208A
:101AA00072657665727365640052657665727365FA
:101AB000643A2020004D61782050756C73653A209F
:101AC000004D696E2050756C73653A200053746147
:101AD00072742056616C75657300494E56414C49CD
:101AE0004420534552564F2E204E4F2053455455B7
:101AF000502E005365747570205265636F696C20B9
:101B0000536572766F0053657475702054757272E8
:101B1000657420526F746174696F6E2050616E201D
:101B2000536572766F0053657475702053746565E4
:101B300072696E6720536572766F20284F757470D6
:101B4000757420322900536574757020537465656F
:101B500072696E6720536572766F20284F757470B6
:101B60007574203429005365747570205475727231
:101B7000657420456C65766174696F6E205365727B
:101B8000766F004865617420416D743A20004865A5
:101B900061743A200053616D652061732066616E47
:101BA000005374617274205265766F6C76696E674B
:101BB00020417578204C6967687400536D6F6B65C0
:101BC0007220656E61626C656400536D6F6B657247
:101BD0002064697361626C65640053657420766F7C
:101BE0006C756D653A2000202D205374617274204D
:101BF000526570656174696E6700202D2053746FA3
:101C000070005573657220536F756E64200041201B
:101C10002D200042202D2000536F756E64204261FC
:101C20006E6B2000506C61792F53746F7000506C94
:101C300061792052616E646F6D00506C6179205043
:101C4000726576696F757300506C6179204E6578A6
:101C5000740054616967656E2056322F5633005305
:101C60006F6E790052435441204D616368696E651F
:101C70002047756E00436C61726B204D616368692B
:101C80006E652047756E0052435441205265706165
:101C90006972004942552052657061697200436C57
:101CA00061726B20526570616972004F70656E5091
:101CB000616E7A657200567354616E6B00464F56C2
:101CC0000054616967656E2056310048656E672073
:101CD0004C6F6E670054616D69796120312F333527
:101CE0000054616D69796120322D53686F7400541E
:101CF000616D69796100556E6B6E6F776E003A2089
:101D00000042697420004761703A20004169727393
:101D10006F6674202D20456E61626C6564004D65B0
:101D20006368616E6963616C205265636F696C20E2
:101D30002D20456E61626C656400524144494F201C
:101D40004641494C53414645000047B511241FBE4A
:101D5000CFEFD1E2DEBFCDBF00E00CBF17E0A0E0C7
:101D6000B2E0E0E3F1EB01E00BBF02C007900D929F
:101D7000A231B107D9F724E1A2E1B7E001C01D9279
:101D8000A03DB207E1F71EE0C6EADEE000E006C0D3
:101D900021970109802FFE010E94D0C4C53AD107C6
:101DA00080E00807A9F70E94ADA20C9423C70C9409
:101DB00000002F923F924F925F926F927F928F928C
:101DC0009F92AF92BF92CF92DF92EF92FF920F93CA
:101DD0001F93CF93DF93CDB7DEB7E6970FB6F89496
:101DE000DEBF0FBECDBF80918D1390918E130E94E8
:101DF000B7470E943F576FEC75E080918D1390912B
:101E00008E130E94AF486BE676E0CE0101960E94E9
:101E1000374780918D1390918E13DC01ED91FC91E9
:101E20004D815E8169817A810280F381E02D19956F
:101E300063E776E080918D1390918E130E94AE48F7
:101E40002AE041EE51E060E070E080918D139091C6
:101E50008E130E946F4765EC76E080918D13909110
:101E60008E130E94BA47CE0101960E94DB460E9463
:101E7000E99780918D1390918E13DC01ED91FC9187
:101E80000680F781E02D199580918D1390918E1326
:101E90000E94B7470E943F5764E676E080918D1319
:101EA00090918E130E94AF48E091F60BE4300CF055
:101EB000E0E080EF95E09A8389838CEE95E09C8347
:101EC0008B8387EE95E09E838D8382EE95E09887E5
:101ED0008F83EE0FFF0B21E030E02C0F3D1FE20F50
:101EE000F31F6081718180918D1390918E130E94F8
:101EF000D3480E943F576EE276E080918D13909117
:101F00008E130E94D3480E943F5762E276E0809190
:101F10008D1390918E130E94AF48E091C410F09100
:101F2000C51081819281883E934014F40E942F57FE
:101F3000E091C410F091C5106181728180918D1380
:101F400090918E130E94876C84E00E940B95E09123
:101F5000C410F091C5106581768180918D139091A8
:101F60008E130E94876C85E00E940B95E091C4104F
:101F7000F091C5106381748180918D1390918E13BF
:101F80000E94876C84E00E940B95E091C410F09150
:101F9000C510678180918D1390918E130E94D76A2E
:101FA00088E00E940B95E091C410F091C5108085E7
:101FB0000E94155766E176E080918D1390918E1303
:101FC0000E94AF48E091CE10F091CF1081819281B4
:101FD000883E934014F40E942F57E091CE10F09168
:101FE000CF106181728180918D1390918E130E9428
:101FF000876C84E00E940B95E091CE10F091CF1099
:102000006581768180918D1390918E130E94876CEB
:1020100085E00E940B95E091CE10F091CF10638186
:10202000748180918D1390918E130E94876C84E04F
:102030000E940B95E091CE10F091CF1067818091B6
:102040008D1390918E130E94D76A88E00E940B95A1
:10205000E091CE10F091CF1080850E9415576AE074
:1020600076E080918D1390918E130E94AF48E0919D
:10207000D810F091D91081819281883E934014F458
:102080000E942F57E091D810F091D9106181728190
:1020900080918D1390918E130E94876C84E00E9432
:1020A0000B95E091D810F091D910658176818091DF
:1020B0008D1390918E130E94876C85E00E940B9582
:1020C000E091D810F091D9106381748180918D13C3
:1020D00090918E130E94876C84E00E940B95E09192
:1020E000D810F091D910678180918D1390918E1343
:1020F0000E94D76A88E00E940B95E091D810F09179
:10210000D91080850E9415576EEF75E080918D1370
:1021100090918E130E94AF48E091E210F091E3108D
:1021200081819281883E934014F40E942F57E09160
:10213000E210F091E3106181728180918D13909192
:102140008E130E94876C84E00E940B95E091E21050
:10215000F091E3106581768180918D1390918E13BB
:102160000E94876C85E00E940B95E091E210F0914F
:10217000E3106381748180918D1390918E130E947E
:10218000876C84E00E940B95E091E210F091E310DF
:10219000678180918D1390918E130E94D76A88E099
:1021A0000E940B95E091E210F091E31080850E946F
:1021B000155780918D1390918E130E94B7470E94FE
:1021C00027A1C82E66E976E080918D1390918E1339
:1021D0000E94D3480E943F5708E610E1E12CF12C01
:1021E000D12C5701BFEFAB1ABB0AB50180918D13FB
:1021F00090918E130E94876CE9E0EE16F10410F4C2
:102200008BE001C08AE00E940B95D8012C9180914F
:102210008D1390918E132223C9F11596ED91FC91A7
:102220001697618172810E94876CD8011596ED9195
:10223000FC91169781819281883E934014F40E940C
:102240002F5784E00E940B95D8011596ED91FC91D3
:1022500016976381748180918D1390918E130E94E3
:10226000876C84E00E940B95D8011596ED91FC9146
:102270001697278180918D1390918E13222319F048
:102280006EE876E00BC067E876E008C0EC14FD0469
:102290001CF46FE776E002C062E776E00E94D34864
:1022A000095F1F4F7501BCE0AB16B10409F099CF6F
:1022B0000E943F576BEC76E080918D1390918E13C6
:1022C0000E94AF480E9427A1682F80918D139091A2
:1022D0008E130E94C06A67EB76E080918D13909117
:1022E0008E130E94AF486091F30B7091F40B8091B4
:1022F0008D1390918E130E94BD6C0E94E99780917E
:102300008D1390918E13DC01ED91FC910680F78185
:10231000E02D199580918D1390918E130E94B747EF
:102320000E943F576BE977E080918D1390918E1357
:102330000E94D3480E943F5767E877E080918D1351
:1023400090918E130E94AF488091C3120E94FA4D63
:10235000BC0180918D1390918E130E94AF488091A3
:10236000C3128A30C1F465E777E080918D139091B4
:102370008E130E94AF486091811380918D139091CC
:102380008E130E94D76A6EE677E080918D1390914C
:102390008E130E94AF4880918D1390918E130E94EE
:1023A000B7476AE577E080918D1390918E130E9474
:1023B000AF488091C4120E94FA4DBC0180918D13E8
:1023C00090918E130E94AF482091C41280918D137A
:1023D00090918E132B303CF4293054F4283069F45A
:1023E00069E477E007C02B3041F465E577E002C08F
:1023F0006FE477E00E94D34802C00E94B74765E3CC
:1024000077E080918D1390918E130E94AF48809158
:10241000C5120E94FA4DBC0180918D1390918E13CC
:102420000E94AF482091C51280918D1390918E1318
:102430002B303CF4293054F4283069F464E277E01E
:1024400007C02B3041F460E377E002C06AE277E036
:102450000E94D34802C00E94B74760E177E08091B4
:102460008D1390918E130E94AF482091D7128091C6
:102470008D1390918E13222319F068E077E002C04B
:1024800066EF76E00E94AF482091E31380918D13B0
:1024900090918E13222319F06BEE76E002C06FED5F
:1024A00076E00E94AF4880918D1390918E130E9428
:1024B000B7470E94E99780918D1390918E13DC01AC
:1024C000ED91FC910680F781E02D19958091000235
:1024D000823011F00C94F41CF090FE120091011364
:1024E00010E080918D1390918E130E94B7470E9447
:1024F0003F5769E97AE080918D1390918E130E9485
:10250000D3480E943F5760E87AE080918D13909104
:102510008E130E94AF48E0910E13E7300CF0E0E01C
:102520008AEF97E09A83898385EF97E09C838B837A
:102530008BEE97E09E838D8387EE97E098878F835D
:1025400083ED97E09A87898781EC97E09C878B875A
:1025500087EA97E09E878D87EE0FFF0B21E030E042
:102560002C0F3D1FE20FF31F6081718180918D134D
:1025700090918E130E94D34867E67AE080918D1384
:1025800090918E130E94AF486091000280918D134C
:1025900090918E130E94C06A6EE47AE080918D1350
:1025A00090918E130E94AF488F2D0E940057FF20FC
:1025B00009F44BC064E47AE080918D1390918E13FE
:1025C0000E94AF4880918D1390918E13112339F0A2
:1025D0006091F9120E94D76A9091F91206C0609139
:1025E000FF120E94D76A9091FF1280919B1498135A
:1025F0000C94FB1C68E27AE080918D1390918E130D
:102600000E94AF4880918D1390918E13112339F061
:102610006091FA1261110CC063E27AE006C0609129
:102620000013611105C06EE17AE00E94AF4805C059
:10263000062E000C770B0E94876C6CE17AE080918B
:102640008D1390918E130E94AF4880918D139091BD
:102650008E130E94B74763E07AE080918D139091CA
:102660008E130E94AF48802F0E940057002309F468
:102670004BC069EF79E080918D1390918E130E9489
:10268000AF4880918D1390918E13112339F0609192
:10269000FC120E94D76A9091FC1206C0609102134E
:1026A0000E94D76A9091021380919D1498130C9404
:1026B000151D6DED79E080918D1390918E130E9420
:1026C000AF4880918D1390918E13112339F0609152
:1026D000FD1261110CC068ED79E006C06091031332
:1026E000611105C063ED79E00E94AF4805C0062E78
:1026F000000C770B0E94876C61ED79E080918D135F
:1027000090918E130E94AF4880918D1390918E13FB
:102710000E94B74768EB79E080918D1390918E13FA
:102720000E94AF4880911713811103C00E940E5779
:1027300035C062E078E080918D1390918E130E94F5
:10274000AF4865EB79E080918D1390918E130E94D4
:10275000AF486091171380918D1390918E130E9452
:10276000D76A65EA79E080918D1390918E130E946B
:10277000AF48409118135091191360E070E02AE0BF
:1027800080918D1390918E130E946F4760EA79E0DB
:1027900080918D1390918E130E94D34867E879E061
:1027A00080918D1390918E130E94AF4880910F13EA
:1027B0008436C8F460E879E080918D1390918E138F
:1027C0000E94AF4860910F1380918D1390918E13EA
:1027D0000E94D76A6EE779E080918D1390918E13F5
:1027E0000E94D34803C080E00E940E5765E679E05E
:1027F00080918D1390918E130E94AF488091101399
:102800008436C8F46EE579E080918D1390918E1333
:102810000E94AF486091101380918D1390918E1398
:102820000E94D76A6CE579E080918D1390918E13A8
:102830000E94D34803C080E00E940E5763E479E011
:1028400080918D1390918E130E94AF482091A7071D
:1028500080918D1390918E13222319F06CE379E00F
:1028600002C062E379E00E94D34869E179E0809197
:102870008D1390918E130E94AF4860910513709153
:102880000613072E000C880B990B0E9471C120E0E3
:1028900030E04AE754E40E9476C3AB01BC0121E07A
:1028A00080918D1390918E130E94D14764E179E05D
:1028B00080918D1390918E130E94D3486BEF78E036
:1028C00080918D1390918E130E94AF4860910713F1
:1028D00070910813072E000C880B990B0E9471C190
:1028E00020E030E04AE754E40E9476C3AB01BC012B
:1028F00021E080918D1390918E130E94D14766EF55
:1029000078E080918D1390918E130E94D3486DEDE5
:1029100078E080918D1390918E130E94AF48609162
:10292000091370910A13072E000C880B990B0E9453
:1029300071C120E030E04AE754E40E9476C3AB0165
:10294000BC0121E080918D1390918E130E94D1479C
:1029500068ED78E080918D1390918E130E94D3489A
:102960006FEB78E080918D1390918E130E94AF48A9
:1029700090910E13913011F09430F9F480910B1373
:102980000E94005780910B13882329F16BEB78E0AC
:1029900080918D1390918E130E94AF4860910C131B
:1029A00080918D1390918E130E94D76A69EB78E025
:1029B00080918D1390918E130CC020918D133091C6
:1029C0008E13953019F46CEA78E002C067E978E07C
:1029D000C9010E94AF4880918D1390918E130E947F
:1029E000B74780910E138230C1F46EE778E0809192
:1029F0008D1390918E130E94AF48609111138091B6
:102A00008D1390918E130E94D76A6CE778E08091C5
:102A10008D1390918E130E94D34863E678E08091E5
:102A20008D1390918E130E94AF4890910E132FEF4B
:102A3000290F80918D1390918E13223028F460918C
:102A400012070E94C06A04C06EE478E00E94D34876
:102A500065E378E080918D1390918E130E94AF48CA
:102A600080911B130E94005780911B13882341F112
:102A700063E278E080918D1390918E130E94AF48AD
:102A800060911C1380918D1390918E130E94D76AD0
:102A90006BE078E080918D1390918E130E94AF4887
:102AA00060911D1380918D1390918E130E94D76AAF
:102AB00069E078E080918D1390918E130E94AF4869
:102AC00080918D1390918E130E94B7470E94E997D1
:102AD00080918D1390918E13DC01ED91FC91068015
:102AE000F781E02D199580918D1390918E130E949E
:102AF000B7470E943F5762E27BE080918D1390912F
:102B00008E130E94D3480E943F5761E07BE0809182
:102B10008D1390918E130E94AF488091CC12843611
:102B2000C8F46AEF7AE080918D1390918E130E9421
:102B3000AF486091CC1280918D1390918E130E94BA
:102B4000D76A68EF7AE080918D1390918E130E947E
:102B5000D34803C080E00E940E5767ED7AE0809171
:102B60008D1390918E130E94AF488091CB128436C2
:102B7000C8F460ED7AE080918D1390918E130E94DD
:102B8000AF486091CB1280918D1390918E130E946B
:102B9000D76A6EEC7AE080918D1390918E130E942B
:102BA000D34803C080E00E940E576DEA7AE080911E
:102BB0008D1390918E130E94AF486091D91270913D
:102BC000DA121616170614F500918D1310918E1354
:102BD000072E000C880B990B0E9471C120E030E099
:102BE0004AE754E40E9476C3AB01BC0122E0C8016D
:102BF0000E94D147C8010E94B74768EA7AE08091F5
:102C00008D1390918E130E94D34803C080E00E94E0
:102C10000E570E94E99780918D1390918E13DC01DD
:102C2000ED91FC910680F781E02D199580918D132F
:102C300090918E130E94B7470E943F5769E47CE051
:102C400080918D1390918E130E94D3480E943F571C
:102C50002091E61280918D1390918E13FE01319692
:102C60006F01211103C067E27CE0C7C160E17CE035
:102C70000E94AF48E091EF12E3300CF0E3E08BE507
:102C80009BE09A83898387E49BE09C838B838AE320
:102C90009BE09E838D8382E39BE098878F83EE0F7A
:102CA000FF0BEC0DFD1D6081718180918D13909162
:102CB0008E130E94D348FF24F3948091EF12811168
:102CC00001C0F12C69EF7BE080918D1390918E1300
:102CD0000E94AF486091F01280918D1390918E13F5
:102CE000611105C065EF7BE00E94D3481AC00E94C5
:102CF000D76A6CEE7BE080918D1390918E130E94C9
:102D0000AF488091F407811108C066ED7BE08091A7
:102D10008D1390918E130E94AF4885ED99E00E942B
:102D2000B7476091E7127091E812072E000C880BEC
:102D3000990B0E9471C120E030E04FE753E40E94FC
:102D400076C320E030E048EC52E40E94D0C120E09D
:102D500030E040E05FE30E9412C30E94DEC3E62E33
:102D6000262F372F8901A090F112B090F2126FEB4D
:102D70007BE080918D1390918E130E94AF488E2D31
:102D80000E94F156043611053CF40E942F570A3078
:102D9000110514F40E942F5783E00E940B95FF2029
:102DA00001F10E947195B501BB0C880B990B0E9433
:102DB00071C120E030E04FE753E40E9476C320E089
:102DC00030E048EC52E40E94D0C120E030E040E026
:102DD0005FE30E9412C30E94DEC3862F0E94F15659
:102DE00004C00E9469950E9461950E9429576091D4
:102DF000E9127091EA12072E000C880B990B0E94C1
:102E000071C120E030E04FE753E40E9476C320E038
:102E100030E048EC52E40E94D0C120E030E040E0D5
:102E20005FE30E9412C30E94DEC3E62E262F372FD7
:102E30008901A090F312B090F41268EA7BE08091CF
:102E40008D1390918E130E94AF488E2D0E94F156E3
:102E5000043611053CF40E942F570A30110514F472
:102E60000E942F5783E00E940B95FF2001F10E94E2
:102E70007195B501BB0C880B990B0E9471C120E0C4
:102E800030E04FE753E40E9476C320E030E048ECA6
:102E900052E40E94D0C120E030E040E05FE30E94B5
:102EA00012C30E94DEC3862F0E94F15604C00E9406
:102EB00069950E9461950E9429576091EB1270916B
:102EC000EC12072E000C880B990B0E9471C120E0B8
:102ED00030E04FE753E40E9476C320E030E048EC56
:102EE00052E40E94D0C120E030E040E05FE30E9465
:102EF00012C30E94DEC3E62E262F372F8901A09031
:102F0000F512B090F61261E97BE080918D139091FB
:102F10008E130E94AF488E2D0E94F1560436110583
:102F20003CF40E942F570A30110514F40E942F57C9
:102F300083E00E940B95FF2001F10E947195B5017D
:102F4000BB0C880B990B0E9471C120E030E04FE769
:102F500053E40E9476C320E030E048EC52E40E9443
:102F6000D0C120E030E040E05FE30E9412C30E9445
:102F7000DEC3862F0E94F15604C00E9469950E940C
:102F800061950E9429576AE77BE080918D139091AB
:102F90008E130E94AF486091ED127091EE12009175
:102FA0008D1310918E136115710521F461E77BE09B
:102FB000C80123C0072E000C880B990B0E9471C119
:102FC00020E030E04FE753E40E9476C320E030E099
:102FD00048EC52E40E94D0C120E030E040E05FE3E2
:102FE0000E9412C30E94DEC3C8010E94876C6FE674
:102FF0007BE080918D1390918E130E94D3480E94A4
:10300000E99780918D1390918E13DC01ED91FC91E5
:103010000680F781E02D199580918D1390918E1384
:103020000E94B7470E943F5765EB7DE080918D136A
:1030300090918E130E94D3480E943F5720913207EF
:1030400080918D1390918E13222309F4B7C166E805
:103050007DE00E94AF480E944E7B0E940E570E9466
:103060004E7B20918D1330918E13882389F063E776
:103070007DE0C9010E94AF48809135070E943499D4
:10308000BC0180918D1390918E130E94D3484BC048
:1030900060E67DE0C9010E94AF48809132070E943E
:1030A0003499BC0180918D1390918E130E94AF488A
:1030B00080913307882389F168E57DE080918D1345
:1030C00090918E130E94AF48E0913307E4300CF0EA
:1030D000E0E08EEA93E09A8389838CEA93E09C8314
:1030E0008B838AEA93E09E838D8388EA93E09887B6
:1030F0008F83EE0FFF0BEC0DFD1D608171818091C0
:103100008D1390918E130E94AF4866E57DE080910B
:103110008D1390918E130E94AF4880918D139091E2
:103120008E130E94B74763E47DE080918D139091E8
:103130008E130E94AF488091340700918D13109137
:103140008E13882321F00E943499BC0102C06FE3E2
:103150007DE0C8010E94D3486CE27DE080918D1330
:1031600090918E130E94AF488091350700918D1386
:1031700010918E13882321F00E943499BC0102C063
:1031800068E27DE0C8010E94D34865E17DE080915E
:103190008D1390918E130E94AF488091370788233A
:1031A000E1F06FE07DE080918D1390918E130E948D
:1031B000AF48809136070E943499BC0180918D13ED
:1031C00090918E130E94AF4865EC76E080918D134C
:1031D00090918E130E94BA4703C080E00E940E5760
:1031E0006CEF7CE080918D1390918E130E94AF481C
:1031F000809138078823E1F066EF7CE080918D13A1
:1032000090918E130E94AF48809136070E943499A6
:10321000BC0180918D1390918E130E94AF4865EC94
:1032200076E080918D1390918E130E94BA4703C06F
:1032300080E00E940E5763EE7CE080918D139091A8
:103240008E130E94AF48E0913907E3300CF0E3E0C1
:103250008BE89CE09A8389838FE79CE09C838B8337
:103260008AE79CE09E838D8382E79CE098878F832A
:10327000EE0FFF0BEC0DFD1D6081718180918D13B0
:1032800090918E130E94D34860ED7CE080918D1365
:1032900090918E130E94AF48E0912B07E4300CF020
:1032A000E4E08BE69CE09A83898385E69CE09C833E
:1032B0008B838EE59CE09E838D8388E59CE09887D8
:1032C0008F8380E59CE09A878987EE0FFF0BEC0DDA
:1032D000FD1D6081718180918D1390918E130E94EC
:1032E000D3486EEC7CE080918D1390918E130E94F8
:1032F000AF486091300780918D1390918E130E949A
:10330000D76A6FEB7CE080918D1390918E130E94B1
:10331000AF4880912B07811110C0609131078091D7
:103320008D1390918E130E94D76A64EB7CE080919C
:103330008D1390918E130E94AF4860912C0770916D
:103340002D07072E000C880B990B0E9471C120E0FD
:1033500030E04AE754E40E9476C3AB01BC0121E0AF
:1033600080918D1390918E130E94D14766EA7CE084
:1033700080918D1390918E130E94AF4860912E071B
:1033800070912F07072E000C880B990B0E9471C1BA
:1033900020E030E04AE754E40E9476C3AB01BC0170
:1033A00021E080918D1390918E130E94D14767E99F
:1033B0007CE080918D1390918E1302C069E97DE0CD
:1033C0000E94D3480E94E99780918D1390918E13AB
:1033D000DC01ED91FC910680F781E02D199580913B
:1033E0008D1390918E130E94B7470E943F5763E35D
:1033F0007EE080918D1390918E130E94D3480E949D
:103400003F5766E27EE080918D1390918E130E946B
:10341000AF48E0912413E6300CF0E6E08EE0D601F0
:103420001D928A95E9F784E19EE09A8389838DEF66
:103430009DE09C838B838BEE9DE09E838D838CED42
:103440009DE098878F8389EC9DE09A87898781EC3E
:103450009DE09C878B87EE0FFF0BEC0DFD1D6081BF
:10346000718180918D1390918E130E94D3480E9498
:10347000E99780918D1390918E13DC01ED91FC9171
:103480000680F781E02D19952CEE3EE841E05527A6
:103490002BAB3CAB4DAB5EAB80918D1390918E13FB
:1034A0000E94B7470E943F5768E470E180918D13F6
:1034B00090918E130E94D3480E943F576FE270E1B3
:1034C00080918D1390918E130E94AF482091F10B43
:1034D00080918D1390918E13222319F06BE270E18D
:1034E00002C066E270E10E94D3488091F10B88230C
:1034F00049F16DE070E180918D1390918E130E94DF
:10350000AF486091221370912313072E000C880B93
:10351000990B0E9471C120E030E04AE754E40E9418
:1035200076C3AB01BC0122E080918D1390918E1384
:103530000E94D14768E070E180918D1390918E13C5
:103540000E94D3489DE4E92E92E1F92E29E2622EF1
:103550003AE0232E312C44E6842E912CD7012C9175
:10356000222309F4FFC1F70132970081118101156F
:10357000110509F4F7C186E49EE8A1E0BB27820F9C
:10358000911DA11DB11DABBFFC01879177247394E0
:10359000811101C0712C20918D1330918E13C801BF
:1035A0000197849790F568EE7FE0C9010E94AF48CB
:1035B00009500C3148F4E02FF0E0EE0FFF1FE15E00
:1035C000FD4F6081718102C06EE37EE080918D13BA
:1035D00090918E130E94AF480C3130F4E02FF0E050
:1035E000E95AFD4F808101C080E090E08252904F07
:1035F000092E000CAA0BBB0BABBFFC0187919EE010
:10360000981B892F09F053C154C1C80184569109F0
:103610008438934008F03FC06EEC7FE0C9010E94FF
:10362000AF48C801B4010E94A9C46130710531F0EE
:103630006230710559F46AEC7FE002C06CEC7FE007
:1036400080918D1390918E130E94AF480E9437573E
:10365000A0908D13B0908E137720B1F0C8010E9416
:10366000F295811107C066EC7FE0C5010E94AF486A
:1036700087E01DC1813009F01CC163EC7FE0C5010A
:103680000E94AF4888E013C16AEB7FE0C5010E9449
:10369000AF4882E00CC1C801885E934080359644F3
:1036A00008F05CC0C80168EE73E00E94A9C45B0129
:1036B0006DEA7FE0C9010E94AF48FAE0AF16B1049D
:1036C00010F40E942F57B50180918D1390918E13A5
:1036D0000E94876C0E94375740908D1350908E1334
:1036E0007720B1F1C8010E94F295782E68EA7FE058
:1036F000C2010E94AF48672D80918D1390918E1367
:103700000E94D76A62EA7FE080918D1390918E13B8
:103710000E94AF4828E13CEFA29EC001A39E900DFD
:10372000B29E900D1124800F911FB1010E94BDC463
:10373000772780918D1390918E130E94876C60EA99
:103740007FE080918D1390918E130E94AF48B1C09D
:1037500067E97FE0C2010E94AF4861C0F801E85309
:10376000FA44E83E43E0F40708F046C0EC30F105C7
:1037700008F09FC08827EE58FF4F8F4F0C94D0C49D
:1037800068E87FE019C06DE77FE0C9010E94AF489B
:1037900083E18DC06BE67FE027C06BE57FE016C05C
:1037A0006EE47FE055C062E47FE0C9010E94AF484B
:1037B00082E17DC063E37FE0C9010E94AF488FE0F2
:1037C00076C064E27FE0F8CF64E17FE0C9010E9447
:1037D000AF488EE06CC061E07FE0C9010E94AF4855
:1037E0008BE065C06FEE7EE0C9010E94AF488CE0BF
:1037F0005EC062EE7EE02CC0C80180529E44883ECE
:10380000934078F400526BEC7EE0C9010E94AF480F
:103810000A3010F40E942F57802F0E94F15684E046
:1038200046C0C80188509245883E934020F4085015
:1038300064EB7EE0EACF013FB5E51B0719F463EACC
:103840007EE01CC0023FE5E51E0739F466E97EE034
:10385000C9010E94AF4881E12AC0033FF5E51F0777
:1038600039F468E87EE0C9010E94AF4880E11FC0DA
:10387000043F45E5140739F467E77EE0C9010E947B
:10388000AF488DE014C0053F55E5150739F46FE5E5
:103890007EE0C9010E94AF4886E009C0063F154599
:1038A00041F466E47EE0C9010E94AF4885E00E94D1
:1038B0000B9563E070E180918D1390918E130E94BF
:1038C000AF4868EF7FE080918D1390918E130E9436
:1038D000AF48D7016C9170E080918D1390918E1359
:1038E0000E94876CF70180818A3020F482E00E9478
:1038F0000B9504C0843610F40E942F570E9437574E
:10390000D7014C91649EA0011124052E000C660B7A
:10391000770B8BA99CA9ADA9BEA9480F591F6A1F97
:103920007B1FD6018A019B010F5F1F4F2F4F3F4F17
:103930006BBFFA0187918D93B901A8018111F2CF74
:10394000B60180918D1390918E130E94BA47809199
:103950008D1390918E13DC01ED91FC910680F7811F
:10396000E02D1995B3E0EB0EF11CE5ECEE16E2E16B
:10397000FE0609F0F3CD0E94E99780918D13909196
:103980008E13DC01ED91FC910680F781E02D1995F5
:1039900080918D1390918E130E94B7470E943F57DC
:1039A00069EA70E180918D1390918E130E94D34843
:1039B0000E943F5766E970E180918D1390918E13BC
:1039C0000E94AF480E94CB7320E030E040E050E41A
:1039D0000E946BC120918D1330918E1387FF3FC0E1
:1039E00063E970E1C90159C0F090F8120091FB122F
:1039F00011E00C94711265E37AE080918D1390913F
:103A00008E130E94AF4860919B1480918D1390910A
:103A10008E130E94D76A63E37AE080918D139091B0
:103A20008E130E94AF480C94FA126AEE79E08091EE
:103A30008D1390918E130E94AF4860919D148091D8
:103A40008D1390918E130E94D76A68EE79E0809171
:103A50008D1390918E130E94AF480C9459136FE808
:103A600070E1C9010E94D3486CE770E180918D1329
:103A700090918E130E94AF480E94CB73AB01BC01A2
:103A800022E080918D1390918E130E94D1476AE7B6
:103A900070E180918D1390918E130E94D34867E658
:103AA00070E180918D1390918E130E94AF488091A8
:103AB0006E130E94005720916E1380918D13909188
:103AC0008E13222379F064E670E10E94AF480E94D1
:103AD0004A956AE570E180918D1390918E130E9452
:103AE000D34802C00E94B7470E94E99780918D1386
:103AF00090918E13DC01ED91FC910680F781E02D11
:103B0000199580918D1390918E130E94B7470E9452
:103B10003F5761E071E180918D1390918E130E9467
:103B2000D3480E943F576DEE70E180918D139091C4
:103B30008E130E94AF4840915E1350915F136091C5
:103B400060137091611380918D1390918E130E9478
:103B5000746C69ED70E180918D1390918E130E94C9
:103B6000AF4840916613509167136091681370914C
:103B7000691380918D1390918E130E94746C65EC83
:103B800070E180918D1390918E130E94AF48409107
:103B90006213509163136091641370916513809167
:103BA0008D1390918E130E94746C61EB70E1809183
:103BB0008D1390918E130E94AF4840916A135091DB
:103BC0006B1360916C1370916D1380918D139091B4
:103BD0008E130E94746C0E94E99780918D139091CE
:103BE0008E13DC01ED91FC910680F781E02D199593
:103BF00080918D1390918E130E94B7470E943F577A
:103C0000E6960FB6F894DEBF0FBECDBFDF91CF9121
:103C10001F910F91FF90EF90DF90CF90BF90AF90EA
:103C20009F908F907F906F905F904F903F902F90DC
:103C300008952F923F924F925F926F927F928F9250
:103C40009F92AF92BF92CF92DF92EF92FF920F932B
:103C50001F93CF93DF93CDB7DEB7AB970FB6F89432
:103C6000DEBF0FBECDBF8DED91E00E949CC2603FD4
:103C70007F4B8105910519F00E94688F08C041EEC5
:103C800051E060E070E086EA91E10E9484C240E089
:103C900052EC61E070E085ED99E00E945B8140911B
:103CA000621350916313609164137091651388E3FC
:103CB00099E00E945B814091661350916713609177
:103CC0006813709169138BE998E00E945B814091C1
:103CD0006A1350916B1360916C1370916D138EEF9A
:103CE00097E00E945B818BEA9EE09093F8078093B7
:103CF000F7078CE69CE09093F6078093F50711E0B8
:103D00001093AD0E85ED99E09093AB148093AA14B7
:103D10001092AC141092B10E1092AE0E1092B00E22
:103D20001092AF0E10930B140E9459608091821371
:103D30008093AE0710928F131092800082E08093E0
:103D400081008FE286BB10926F0010928500109266
:103D500084009BE29093A00099E09093A10089BB1E
:103D6000109272001092A5001092A4001092A90067
:103D70001092A8001092AB001092AA001092AD0011
:103D80001092AC0099EA90932001109321018ABB14
:103D900010927300109225011092240110922901B3
:103DA0001092280110922B0110922A0110922D01DD
:103DB00010922C01809143129091441280934307FA
:103DC00090934407813001F58FE38093140C109297
:103DD000150C61E00E94094B8AE09CE00E9425934B
:103DE0001092160C1092190C1092180C8091440726
:103DF000882329F08AE09CE00E94F89411C08AE0B0
:103E00009CE00E94D1940CC080914407882311F05B
:103E100062E001C060E08FE30E94094B0E94D17410
:103E200080914512909146128093490790934A07DA
:103E3000813001F58EE38093450C1092460C61E0D1
:103E40000E94094B8BE39CE00E9425931092470C43
:103E500010924A0C1092490C80914A07882329F04D
:103E60008BE39CE00E94F89411C08BE39CE00E94DD
:103E7000D1940CC080914A07882311F062E001C000
:103E800060E08EE30E94094B0E949E7460E085E42E
:103E90000E94094B62E08CE30E94094B62E08BE3D5
:103EA0000E94094B62E080E40E94094B62E081E4D9
:103EB0000E94094B62E082E40E94094B62E081E2C9
:103EC0000E94094B62E084E40E94094B61E089E3AF
:103ED0000E94094B61E08AE30E94094B0E945F72D5
:103EE0000E94967261E085E30E94094B61E085E0E3
:103EF0000E94094B61E070E085E00E94454B61E063
:103F000084E00E94094B61E087E00E94094B61E078
:103F100089E20E94DA4A61E089E20E94094B519AE3
:103F200060E085E30E94DA4A60E085E00E94DA4AB8
:103F300060E084E00E94DA4A60E087E00E94DA4AAA
:103F4000599861E088E00E94094B80E090E09C0174
:103F50002A553E4EF901E955FF4F40814F3629F46D
:103F6000329720813181232B31F4039688379105D4
:103F700071F760E001C061E088E00E94DA4A61E028
:103F80008DE20E94094B61E08EE20E94094B61E0E4
:103F90008CE20E94094B61E08BE20E94094B60E0D9
:103FA0008BE20E94DA4A0E9496720E94056C809110
:103FB000FA0B813009F058C08091FD0B9091FE0BF7
:103FC000A091FF0BB091000C4091010C5091020C9C
:103FD0006091030C7091040C841B950BA60BB70B1E
:103FE00084379E40A105B10500F30E94688F0E94AE
:103FF00029570E9429570E943F576FE071E1809135
:104000008D1390918E130E94AF4801E010E00E9442
:1040100063720E9496726EEE72E080E090E00E9401
:10402000504C6CE071E180918D1390918E130E9441
:10403000AF480E945F720E9492720530110531F004
:1040400064EF71E080E090E00E94504C0F5F1F4FE2
:1040500006301105E1F60E9429570E943F570E9441
:1040600029570E94295702C081119FCF80916F006C
:10407000826080936F0080918400909185008056CB
:10408000904F90938900809388000E94692C8DE660
:104090009CE09093BF148093BE1410911D13209147
:1040A0001C1380910B1390910D1330910E133093CC
:1040B000FD07909312078093130730E0AFEFB0E055
:1040C0000E9402C324E630E040E050E00E94B4C207
:1040D00020939F14612F70E080E090E00E946FC1F8
:1040E00020ED34E448E55BE30E94D0C126E636E6E5
:1040F00046E25FE30E9412C36093F9077093FA07E8
:104100008093FB079093FC0710939E1410929500E8
:1041100010929400109290008CE08093910084EFB4
:1041200090E0909399008093980081E088BB82E0B2
:1041300080937100809100020E94F45F80912413AB
:10414000863040F01092241360E070E08EE791E03A
:104150000E94986B10912413123009F444C008F5A2
:10416000112309F466C0113009F05BC08CE090E0C7
:104170000E94E4C42BE433E0DC0111963C932E93BF
:104180002BE938E01B963C932E931A979093AB073C
:104190008093AA071093270F10932A0F10932D0FC7
:1041A00067C0133009F45EC01430D9F586E090E0A2
:1041B0000E94E4C48C0125EB33E0DC012D933D9398
:1041C000CD0141E06DE67CE00E94527E87E792E0FF
:1041D000F801918380831093AB070093AA0781E0D5
:1041E0008093270F41C086E090E00E94E4C421EE56
:1041F00032E0FC01318320839093AB078093AA07C0
:104200008FB7F8942CED35E03093E6102093E5104D
:104210001092EB108FBF81E08093270F80932A0FBD
:1042200025C01092241360E070E08EE791E00E94B8
:10423000986B86E090E00E94E4C48C0125EB33E0AB
:10424000DC012D933D93CD0140E06DE67CE00E94C2
:10425000527E87E792E0F801918380831093AB0749
:104260000093AA071092270F10922A0F10922D0F79
:104270008091AA079091AB07DC01ED91FC91019030
:10428000F081E02D199580911B0F81111FC0809145
:104290001E0F81111BC08091210F811117C08091C9
:1042A000240F811113C08091270F81110FC08091BD
:1042B0002A0F81110BC080912D0F811107C081E061
:1042C0000E945560882309F419C311C3A12CB12C95
:1042D000912C1DA2412C512C612C712C812C03E6B8
:1042E00016E0EE24EA94A3E0FA2ECC24CA94DD244E
:1042F000D39487E5282E86E0382EC5018A559E4E38
:10430000FC01E955FF4FE081EE2309F4E7C2DC012F
:10431000AB55BF4F8D919C91892B09F4DFC28E2F35
:1043200090E0FC01F797EB32F10508F0D7C288273F
:10433000E258FF4F8F4F0C94D0C480911B0F8823FD
:1043400009F4CCC28110CAC289E190E00E94E4C4A1
:104350009C01FC011183008387E090E093838283BA
:1043600015821482F782E682D186C086108EC9013A
:104370002AA73BA70E940F422AA53BA5E7E3F4E04A
:10438000D901ED93FC9330930C0F20930B0FC901CF
:104390000E94FC8B7DC180911E0F882309F49EC270
:1043A00071109CC289E190E00E94E4C49C01DC0190
:1043B00011961C930E93E6E0F0E01396FC93EE93B7
:1043C000129715961C921E9214971796FC92EE92D5
:1043D00016971996DC92CE92189758961C922AA797
:1043E0003BA70E940F422AA53BA5E7E3F4E0D901D1
:1043F000ED93FC9330930E0F20930D0FC9010E9493
:10440000FC8B74C18091210F882309F467C261106D
:1044100065C289E190E00E94E4C49C01DC01119630
:104420001C930E93E5E0F0E01396FC93EE93129745
:1044300015961C921E9214971796FC92EE92169760
:104440001996DC92CE92189758961C922AA73BA7F1
:104450000E940F422AA53BA5E7E3F4E0D901ED93C2
:10446000FC933093100F20930F0FC9010E94FC8B17
:104470006BC18091240F882309F430C251102EC2E1
:1044800089E190E00E94E4C49C01DC0111961C9338
:104490000E93E4E0F0E01396FC93EE9312971596DA
:1044A0001C921E9214971796FC92EE9216971996EC
:1044B000DC92CE92189758961C922AA73BA70E948E
:1044C0000F422AA53BA5E7E3F4E0D901ED93FC9365
:1044D0003093120F2093110FC9010E94FC8B62C10F
:1044E0008091270F882309F4F9C14110F7C189E1B0
:1044F00090E00E94E4C49C01DC0111961C930E9391
:10450000E2E0F0E01396FC93EE93129715961C925E
:104510001E9214971796FC92EE9216971996DC92BB
:10452000CE92189758961C922AA73BA70E940F423A
:104530002AA53BA5E7E3F4E0D901ED93FC93309382
:10454000140F2093130FC9010E94FC8B59C1809155
:104550002A0F882309F4C2C12DA12111BFC189E10D
:1045600090E00E94E4C49C01DC0111961C930E9320
:10457000E1E0F0E01396FC93EE93129715961C92EF
:104580001E9214971796FC92EE9216971996DC924B
:10459000CE92189758961C922AA73BA70E940F42CA
:1045A0002AA53BA5E7E3F4E0D901ED93FC93309312
:1045B000160F2093150FC9010E94FC8B59C18091E1
:1045C0002D0F882309F48AC1911088C189E190E0F8
:1045D0000E94E4C49C01DC0111961C930E93139677
:1045E0001C921E92129715961C921E921497179663
:1045F000FC92EE9216971996DC92CE9218975896E6
:104600001C922AA73BA70E940F422AA53BA587E33D
:1046100094E0F901918380833093180F2093170F52
:10462000C9010E94FC8B58C180911B0F882309F49B
:1046300055C1811053C18CE190E00E94E4C49C01FB
:10464000DC0111961C930E93E7E0F0E01396FC93C7
:10465000EE93129715961C921E9214971796FC9241
:10466000EE9216971996DC92CE92189758961C9255
:104670002AA73BA70E940F422AA53BA5D9012D924C
:104680003C9230931A0F2093190FC9010E949C8C01
:104690008824839423C180911E0F882309F41EC1AE
:1046A00071101CC18CE190E00E94E4C49C01FC01EB
:1046B0001183008386E090E09383828315821482C5
:1046C000F782E682D186C086108EC9012AA73BA751
:1046D0000E940F422AA53BA5D9012D923C9230930E
:1046E0001D0F20931C0FC9010E949C8C772473948A
:1046F000F5C08091210F882309F4F0C06110EEC04D
:104700008CE190E00E94E4C49C01FC0111830083D1
:1047100085E090E09383828315821482F782E6829B
:10472000D186C086108EC9012AA73BA70E940F42DE
:104730002AA53BA5D9012D923C923093200F2093BE
:104740001F0FC9010E949C8C66246394C7C080918E
:10475000240F882309F4C2C05110C0C08CE190E03E
:104760000E94E4C49C01FC011183008384E090E07A
:104770009383828315821482F782E682D186C08673
:10478000108EC9012AA73BA70E940F422AA53BA56C
:10479000D9012D923C923093230F2093220FC9010F
:1047A0000E949C8C5524539499C08091270F882394
:1047B00009F494C0411092C08CE190E00E94E4C4DE
:1047C0009C01FC011183008382E090E0938382834B
:1047D00015821482F782E682D186C086108EC901C6
:1047E0002AA73BA70E940F422AA53BA5D9012D92DB
:1047F0003C923093260F2093250FC9010E949C8C78
:10480000442443946BC080912A0F882309F466C026
:104810002DA1211163C08CE190E00E94E4C49C01B1
:10482000DC0111961C930E93E1E0F0E01396FC93EB
:10483000EE93129715961C921E9214971796FC925F
:10484000EE9216971996DC92CE92189758961C9273
:104850002AA73BA70E940F422AA53BA5D9012D926A
:104860003C923093290F2093280FC9010E949C8C01
:1048700021E02DA333C080912D0F882379F1911071
:104880002DC08CE190E00E94E4C49C01DC011196F3
:104890001C930E9313961C921E92129715961C92BF
:1048A0001E9214971796FC92EE9216971996DC9228
:1048B000CE92189758961C922AA73BA70E940F42A7
:1048C0002AA53BA5F9013182208230932C0F209339
:1048D0002B0FC9010E949C8C99249394F3E0AF0E96
:1048E000B11C28E7A216B10409F007CDE8CC82E09C
:1048F0000E945560882311F01FA216C081E00E941B
:104900005560882329F082E00E94396081119CC79C
:104910008CE30E94B24A892B09F087C78CE30E947E
:10492000B24A892B09F087C786E0E4E5F3E1DE01AE
:10493000549601900D928A95E1F780914D139091D4
:104940005D13B0904E1300914F131091501370915E
:104950005113609152135091531340915A13209167
:104960005B1330915C13E091AA07F091AB07FEA3B3
:10497000EDA3A091450FB091460FB9A7A8A79090BD
:10498000801360907B13E0907413F0907513809007
:104990007E1370907D13C090D912D090DA1250908F
:1049A000DC124090D7123090D812BFA1BB8B8A8FF7
:1049B0009B8FBC8E0D8F1E8F7F8F68A359A34AA338
:1049C0003CA32BA3F2E1AF2EFE017396DE011196FC
:1049D00001900D92AA94E1F7EDE6FCE0F0931C073C
:1049E000E0931B07EFA1E98388879987BA860B8735
:1049F0001C877D876E875F87488B3A8B298B22E1E6
:104A0000FE013196ABE2B7E001900D922A95E1F7F5
:104A1000992321F0863011F0109233073092E3137E
:104A20004092E4135092DA13D092D313C092D2136F
:104A30006092470F7092D7138092D613F092D513DD
:104A4000E092D4139092E21388A599A59093D9137C
:104A50008093D8138DA19EA190931E0780931D076C
:104A600087E08093F60A1092F70A61E00E94094BF2
:104A70008CEE9AE00E9425931092F80A1092FB0A9D
:104A80001092FA0A80913607811102C010923707FE
:104A900090913207911105C0811103C01092E10B72
:104AA00098C08091DC0B9091DD0B0E94799581E09C
:104AB0008093E10B80912B07882359F1813071F0AD
:104AC0008330C1F488E293E290932D0780932C0702
:104AD00089E08093300780E197E217C088EB9BE084
:104AE00090932D0780932C0783E08093300788E90B
:104AF0009AE30BC088E893E190932D0780932C07ED
:104B000086E08093300780EE9EE290932F0780939B
:104B10002E07809132078823E9F180913607609152
:104B2000300770E08823C9F0809138078823A9F006
:104B300080E090E00E946FC19B01AC0160E070E0FA
:104B400088EC92E40E9476C360931F07709320075D
:104B5000809321079093220725C080E090E00E9477
:104B60006FC19B01AC0160E070E088EC92E40E94B0
:104B700076C360931F07709320078093210790935B
:104B8000220710921607109217071092180710921A
:104B900019071FC010921F071092200710922107BB
:104BA000109222076091310770E080E090E00E944F
:104BB0006FC19B01AC0160E070E088EC92E40E9460
:104BC00076C3609316077093170780931807909326
:104BD00019071092A5111092230710921A0710922C
:104BE00024071092250710922607109227070E948B
:104BF0008B815098589AE898809169008C7F8093B7
:104C000069008091E413882321F08091690082601B
:104C100003C080916900836080936900E8980E94D6
:104C2000378480E090E040E09C012A553E4EF90137
:104C3000E955FF4F5081552331F032972081318162
:104C4000232B09F04F5F03968837910569F740934E
:104C50003E07ABE4B7E020E030E084E7282E86E5AD
:104C6000382E95EC492E9BE5592E4AE9642E4BE5EA
:104C7000742E5DEA852E5BE5952E67E7A62E66E528
:104C8000B62E44E954E50AE714E577E8E72E74E523
:104C9000F72EE4ECCE2EE3E5DE2EC9018A559E4EBA
:104CA000FC01E955FF4F6081662309F4B0C38B55C1
:104CB0009F4FFC0180819181892B09F4A8C370E08A
:104CC000FB013197E53AF10508F0A1C38827E755C4
:104CD000FF4F8F4F0C94D0C483E79BE511969C93B4
:104CE0008E9395C382E79BE511969C938E938FC319
:104CF00080E79BE511969C938E9389C38AE69BE59A
:104D000011969C938E9383C388E69BE511969C93A2
:104D10008E937DC381EE9AE511969C938E9377C313
:104D200082EE9AE511969C938E9371C384EC9AE57A
:104D300011969C938E936BC380EB9AE511969C938E
:104D40008E9365C381EA9AE511969C938E935FC317
:104D500085E49AE511969C938E9359C38BEE98E562
:104D600011969C938E9353C388E39AE511969C9376
:104D70008E934DC385EC99E511969C938E9347C312
:104D80008FE29AE511969C938E9341C387E39AE54F
:104D900011969C938E933BC381E39AE511969C9365
:104DA0008E9335C388EF99E511969C938E932FC30C
:104DB00080E29AE511969C938E9329C389E19AE546
:104DC00011969C938E9323C388EE99E511969C933C
:104DD0008E931DC386EE99E511969C938E9317C30F
:104DE00084EE99E511969C938E9311C384ED99E519
:104DF00011969C938E930BC382ED99E511969C932B
:104E00008E9305C383EC99E511969C938E93FFC214
:104E100083EB99E511969C938E93F9C281EB99E50A
:104E200011969C938E93F3C28FEA99E511969C9309
:104E30008E93EDC285E697E511969C938E93E7C21B
:104E400083E697E511969C938E93E1C281E697E500
:104E500011969C938E93DBC283EC90E711969C9302
:104E60008E93D5C28DEA99E511969C938E93CFC20D
:104E70008DE999E511969C938E93C9C286E198E5D8
:104E800011969C938E93C3C287EF97E511969C93DE
:104E90008E93BDC28BE999E511969C938E93B7C210
:104EA0008CE699E511969C938E93B1C285E699E5BF
:104EB00011969C938E93ABC284E399E511969C93D3
:104EC0008E93A5C282E995E911969C938E939FC219
:104ED00089EE98E511969C938E9399C287EE98E59A
:104EE00011969C938E9393C284EE98E511969C93B1
:104EF0008E938DC280EC98E511969C938E9387C219
:104F00008CE998E511969C938E9381C281EE98E589
:104F100011969C938E937BC28DEB98E511969C9392
:104F20008E9375C289E998E511969C938E936FC212
:104F30008EED98E511969C938E9369C28AEB98E565
:104F400011969C938E9363C286E998E511969C9383
:104F50008E935DC28BED98E511969C938E9357C20C
:104F600087EB98E511969C938E9351C283E998E55F
:104F700011969C938E934BC288ED98E511969C9365
:104F80008E9345C284EB98E511969C938E933FC215
:104F900080E998E511969C938E9339C285ED98E54A
:104FA00011969C938E9333C281EB98E511969C9356
:104FB0008E932DC28DE898E511969C938E9327C20F
:104FC00082ED98E511969C938E9321C28EEA98E526
:104FD00011969C938E931BC28AE898E511969C9338
:104FE0008E9315C28FEC98E511969C938E930FC209
:104FF0008BEA98E511969C938E9309C287E898E511
:1050000011969C938E9303C28CEC98E511969C9319
:105010008E93FDC188EA98E511969C938E93F7C113
:1050200084E898E511969C938E93F1C189EC98E5FC
:1050300011969C938E93EBC185EA98E511969C930B
:105040008E93E5C181E898E511969C938E93DFC11C
:1050500086EC98E511969C938E93D9C182EA98E5E7
:1050600011969C938E93D3C18EE798E511969C93ED
:105070008E93CDC183EC98E511969C938E93C7C116
:105080008FE998E511969C938E93C1C18BE798E5C3
:1050900011969C938E93BBC18BE897E511969C93D8
:1050A0008E93B5C187E798E511969C938E93AFC117
:1050B00083E798E511969C938E93A9C18FE698E5B6
:1050C00011969C938E93A3C18BE698E511969C93C1
:1050D0008E939DC187E698E511969C938E9397C118
:1050E00083E698E511969C938E9391C18FE598E5A0
:1050F00011969C938E938BC18BE598E511969C93AA
:105100008E9385C182E897E511969C938E937FC11B
:105110008FE597E511969C938E9379C18DE597E580
:1051200011969C938E9373C185E398E511969C9399
:105130008E936DC185EA97E511969C938E9367C116
:1051400089E797E511969C938E9361C187E797E570
:1051500011969C938E935BC185E797E511969C937E
:105160008E9355C18BEC96E511969C938E934FC10F
:1051700089E796E511969C938E9349C18FE795E553
:1051800011969C938E9343C184E395E511969C936D
:105190008E933DC187EF9BE511969C938E9337C10B
:1051A00083EE9BE511969C938E9331C18FEC9BE52A
:1051B00011969C938E932BC18BED95E911969C9340
:1051C0008E9325C184E496E511969C938E931FC11E
:1051D00087E396E511969C938E9319C181E296E53B
:1051E00011969C938E9313C18FEF95E511969C9326
:1051F0008E930DC18FE196E511969C938E9307C116
:1052000081E096E511969C938E9301C182EB93E524
:1052100011969C938E93FBC088E693E511969C9320
:105220008E93F5C08AE893E511969C938E93EFC018
:105230008AE793E511969C938E93E9C08CE993E5F8
:1052400011969C938E93E3C080E493E511969C9312
:105250008E93DDC080E393E511969C938E93D7C027
:1052600082E593E511969C938E93D1C088E295E5F3
:1052700011969C938E93CBC08CE195E511969C93EF
:105280008E93C5C080E195E511969C938E93BFC027
:1052900084E095E511969C938E93B9C088EF94E5D0
:1052A00011969C938E93B3C08CEE94E511969C93CB
:1052B0008E93ADC080EE94E511969C938E93A7C01B
:1052C00080E394E511969C938E93A1C08EE194E5C2
:1052D00011969C938E939BC08CE094E511969C93C1
:1052E0008E9395C08AEF93E511969C938E938FC011
:1052F00088EE93E511969C938E9389C086ED93E595
:1053000011969C938E9383C01196DC92CE927FC0AF
:105310001196FC92EE927BC011961C930E9377C06F
:105320008AEB94E511969C938E9371C011965C93D1
:105330004E936DC01196BC92AE9269C011969C922C
:105340008E9265C011967C926E9261C011965C92AD
:105350004E925DC011963C922E9259C0E1E7F6E55F
:105360001196FC93EE9353C088E696E511969C93B4
:105370008E934DC0E5E6F6E51196FC93EE9347C09B
:1053800082E696E511969C938E9341C0EFE5F6E593
:105390001196FC93EE933BC08CE596E511969C9399
:1053A0008E9335C0E1E5F6E51196FC93EE932FC0A0
:1053B0008AE596E511969C938E9329C0E3E5F6E580
:1053C0001196FC93EE9323C08CE594E511969C9383
:1053D0008E931DC0EFE4F4E51196FC93EE9317C095
:1053E00082E494E511969C938E9311C0ECEDF5E563
:1053F0001196FC93EE930BC08AEC95E511969C9365
:105400008E9305C0EEEEF5E51196FC93EE932D5FBD
:105410003F4F12962837310509F03FCC10923F07D5
:1054200080914307811114C080E090E0FC01E55BAE
:10543000FD4E20813181245631092436310528F072
:1054400003968837910591F703C081E080933F0769
:105450001092450780914907811114C080E090E0C7
:10546000FC01E55BFD4E20813181285C3109243649
:10547000310528F003968837910591F703C081E044
:10548000809345078091AA079091AB07DC01ED91CD
:10549000FC91EE5AFF4F2091271330912813409131
:1054A0002513509126130190F081E02D61E01995AC
:1054B0008091AA079091AB07DC01ED91FC91EE5A27
:1054C000FF4F20912B1330912C13409129135091B1
:1054D0002A130190F081E02D62E019958091AA07CE
:1054E0009091AB07DC01ED91FC91EE5AFF4F2091BA
:1054F0002F133091301340912D1350912E130190A2
:10550000F081E02D63E019958091AA079091AB0797
:10551000DC01ED91FC91EE5AFF4F20913A1330914E
:105520003B1340913813509139130190F081E02DD5
:1055300064E019958091AA079091AB07DC01ED9189
:10554000FC91EE5AFF4F20913E1330913F13409152
:105550003C1350913D130190F081E02D65E01995C9
:105560008091AA079091AB07DC01ED91FC91EE5A76
:10557000FF4F2091421330914313409140135091BB
:1055800041130190F081E02D66E019958091AA0702
:105590009091AB07DC01ED91FC91EC5AFF4F01902B
:1055A000F081E02D4091311361E019958091AA07B7
:1055B0009091AB07DC01ED91FC91EC5AFF4F01900B
:1055C000F081E02D4091321362E019958091AA0795
:1055D0009091AB07DC01ED91FC91EC5AFF4F0190EB
:1055E000F081E02D4091331363E019958091AA0773
:1055F0009091AB07DC01ED91FC91EC5AFF4F0190CB
:10560000F081E02D4091441364E019958091AA0740
:105610009091AB07DC01ED91FC91EC5AFF4F0190AA
:10562000F081E02D4091451365E019958091AA071E
:105630009091AB07DC01ED91FC91EC5AFF4F01908A
:10564000F081E02D4091461366E019958091AA07FC
:105650009091AB07DC01ED91FC9102ACF3ADE02D34
:105660006091351319958091AA079091AB07DC01E1
:10567000ED91FC9106ACF7ADE02D60914A131995C0
:105680008091AA079091AB07DC01ED91FC9100A8F5
:10569000F1A9E02D6091361319958091AA07909198
:1056A000AB07DC01ED91FC9106A8F7A9E02D609114
:1056B000371319958091AA079091AB07DC01ED9102
:1056C000FC91E65BFF4F0190F081E02D40914B1380
:1056D00060E019958091AA079091AB07DC01ED91EC
:1056E000FC91E65BFF4F0190F081E02D40914C135F
:1056F00061E0199580E090E09C012A553E4EF90149
:10570000E955FF4F4081423731F432972081318192
:10571000232B09F09FC003968837910569F70E94F3
:10572000ED968091AA079091AB07DC01ED91FC9179
:10573000EC59FF4F0190F081E02D40E0609147135C
:1057400019958091AA079091AB07DC01ED91FC912E
:10575000EC59FF4F0190F081E02D41E06091491339
:1057600019958091AA079091AB07DC01ED91FC910E
:10577000EC59FF4F0190F081E02D42E06091481319
:1057800019952091721330E0AFEFB0E00E9402C390
:1057900024E630E040E050E00E94B4C2209397132A
:1057A0008091711381110E94EF720E9495A20E9454
:1057B000B3846B017C0110E011110FC08091AE0722
:1057C000882359F029E634E540ED57E060E070E0C9
:1057D0008DE69CE00E94543F11E00E94C48E882315
:1057E00051F00E9409730E94725C0E9496720E949E
:1057F000518E0E9426720E9454A1029711F00E94BD
:10580000A5640E94E9970E9454A10297A9F60E94FC
:10581000B384DC01CB018C199D09AE09BF098C3B17
:105820009240A105B10540F218C082E00E94556087
:1058300081110DC073C882E00E943960882309F489
:1058400073C8A3E0AFA370C881E08FA36DC892E0D6
:105850009FA36AC80E94E19664CF0E94CF7A0E94FB
:1058600096728091F50B811102C00E940C6D0E940E
:1058700027A186E30E940C4CBC01990F880B990B61
:10588000611571058105910511F00E94ECC02BE2B4
:1058900033E548EE53E060E070E08DE69CE0AB96C7
:1058A0000FB6F894DEBF0FBECDBFDF91CF911F9131
:1058B0000F91FF90EF90DF90CF90BF90AF909F90AF
:1058C0008F907F906F905F904F903F902F900C94AF
:1058D000543F5F926F927F928F929F92AF92BF924E
:1058E000CF92DF92EF92FF920F931F93CF93DF93AC
:1058F00081E080931B0F80931E0F8093210F809374
:10590000240F8093300F8093330F90910E1391509A
:10591000963040F080930E1361E070E088E691E0ED
:105920000E94986B90910E132DEF290F8091C31256
:10593000233008F011C28A3079F03CF4883009F441
:1059400063C0893009F4C0C1B6C18B3009F4A4C06A
:105950008C3009F4E6C0AFC184E290E00E94E4C458
:10596000FC018091811328E030E033832283882476
:10597000839499249A9495828482AA24AA94B12C1F
:10598000B782A68211861086108ED3E87D2E718E86
:105990009BE9C92E98E0D92ED38EC28E27E6E22E3F
:1059A00024E0F22EF182E082C6E6D3E1D1A3C0A3C7
:1059B00012A283A3F093A107E093A007CF010E9456
:1059C000264D84E290E00E94E4C4FC0180918113A2
:1059D00029E030E03383228395828482B782A682D5
:1059E00011861086108E718ED38EC28EF182E08267
:1059F000D1A3C0A312A283A3F0939F07E0939E07B5
:105A0000CF010E94264D0EC380E290E00E94E4C4C4
:105A1000FC0188E090E09383828388248394992416
:105A20009A9495828482AA24AA94B12CB782A682E1
:105A300011861086108E7AE0D72ED18EABE9EA2E31
:105A4000A8E0FA2EF38EE28ECFE4D4E0D183C083B7
:105A5000F093A107E093A007CF010E948F4C80E252
:105A600090E00E94E4C4FC0189E090E0938382838B
:105A700095828482B782A68211861086108ED18E7E
:105A8000F38EE28ED183C083F0939F07E0939E074D
:105A9000CF010E948F4CC6C289E190E00E94E4C40D
:105AA000FC0188E090E093838283CC24C394DD24BE
:105AB000DA94D582C482EE24EA94F12CF782E6824D
:105AC00011861086108EC3E4D4E0D183C083F09396
:105AD000A107E093A007CF010E94C68C1092300F5F
:105AE00080910E13843009F09DC289E190E00E94FC
:105AF000E4C4FC0189E090E093838283D582C48270
:105B0000F782E68211861086108ED183C083F093CF
:105B10009F07E0939E07CF010E94C68C1092330F1F
:105B200081C2943009F04BC089E190E00E94E4C446
:105B3000EC01B3E68B2EB6E09B2E9982888287E03B
:105B400090E09B838A83AA24A394BB24BA94BD8249
:105B5000AC82CC24CA94D12CDF82CE8219861886DE
:105B6000188ECE010E940F4227E3E22E24E0F22E8F
:105B7000F982E882D093A107C093A007CE010E94CA
:105B8000FC8B10921B0F89E190E00E94E4C4EC01B1
:105B90009982888286E090E09B838A83BD82AC8272
:105BA000DF82CE8219861886188ECE010E940F429F
:105BB000F982E882D0939F07C0939E074DC095302D
:105BC00009F050C089E190E00E94E4C4EC0173E662
:105BD000872E76E0972E9982888287E090E09B83DB
:105BE0008A83AA24A394BB24BA94BD82AC82CC2419
:105BF000CA94D12CDF82CE8219861886188ECE01E7
:105C00000E940F42A7E3EA2EA4E0FA2EF982E8826E
:105C1000D0939F07C0939E07CE010E94FC8B1092E9
:105C20001B0F89E190E00E94E4C4EC019982888214
:105C300086E090E09B838A83BD82AC82DF82CE8245
:105C400019861886188ECE010E940F42F982E882CA
:105C5000D093A107C093A007CE010E94FC8B1092A5
:105C60001E0FE0C189E190E00E94E4C4EC0183E6EC
:105C700096E09983888387E090E09B838A8381E024
:105C80009FEF9D838C838FEF90E09F838E83198697
:105C90001886188ECE010E940F4287E394E0998304
:105CA0008883D093A107C093A007CE010E94FC8BEC
:105CB00010921B0FB7C189E08093C31269E070E0B6
:105CC0008DE191E00E94986B80E290E00E94E4C434
:105CD000FC0188E090E09383828388248394992454
:105CE0009A9495828482AA24AA94B12CB782A6821F
:105CF00011861086108E50E8D52ED18E6BE9E62ED7
:105D000068E0F62EF38EE28ECBE5D4E0D183C0833B
:105D1000F093A107E093A007CF010E94D14C80E24D
:105D200090E00E94E4C4FC0189E090E093838283C8
:105D300095828482B782A68211861086108ED18EBB
:105D4000F38EE28ED183C083F0939F07E0939E078A
:105D5000CF010E94D14C66C18A3009F458C03CF48E
:105D6000883009F4A2C0893009F405C1FBC08B302A
:105D700009F4BEC08C3009F0F5C089E190E00E94C2
:105D8000E4C4EC0183E6882E86E0982E998288820E
:105D900087E090E09B838A83AA24A394BB24BA94CF
:105DA000BD82AC82CC24CA94D12CDF82CE821986EB
:105DB0001886188ECE010E940F4237E3E32E34E09E
:105DC000F32EF982E882D093A307C093A20789E15A
:105DD00090E00E94E4C4EC019982888286E090E021
:105DE0009B838A83BD82AC82DF82CE82198618862D
:105DF000188ECE010E940F42F982E882D093A50747
:105E0000C093A40710921B0F10921E0FF5C084E2DE
:105E100090E00E94E4C4FC017090811360901A131A
:105E200088E090E0938382838824839499249A94D1
:105E300095828482AA24AA94B12CB782A682118664
:105E40001086108E83E8582E518E9BE9C92E98E05B
:105E5000D92ED38EC28E27E6E22E24E0F22EF182D6
:105E6000E082C6E6D3E1D1A3C0A362A273A2F093FD
:105E7000A307E093A20784E290E00E94E4C4FC013F
:105E800089E090E09383828395828482B782A682A0
:105E900011861086108E518ED38EC28EF182E082D2
:105EA000D1A3C0A362A273A2A3C080E290E00E942B
:105EB000E4C4FC0188E090E0938382838824839487
:105EC00099249A9495828482AA24AA94B12CB782A8
:105ED000A68211861086108EAAE0DA2ED18EBBE93A
:105EE000EB2EB8E0FB2EF38EE28ECFE4D4E065C05B
:105EF00089E190E00E94E4C4FC0188E090E0938393
:105F00008283CC24C394DD24DA94D582C482EE2427
:105F1000EA94F12CF782E68211861086108EC3E493
:105F2000D4E0D183C083F093A307E093A20789E173
:105F300090E00E94E4C4FC0189E090E093838283B6
:105F4000D582C482F782E68211861086108ED183B4
:105F5000C083F093A507E093A4071092300F10922E
:105F6000330F4AC089E08093C31269E070E08DE18D
:105F700091E00E94986B80E290E00E94E4C4FC01F2
:105F800088E090E0938382838824839499249A9470
:105F900095828482AA24AA94B12CB782A682118603
:105FA0001086108EA0E8DA2ED18EBBE9EB2EB8E079
:105FB000FB2EF38EE28ECBE5D4E0D183C083F09349
:105FC000A307E093A20780E290E00E94E4C4FC01F2
:105FD00089E090E09383828395828482B782A6824F
:105FE00011861086108ED18EF38EE28ED183C083FF
:105FF000F093A507E093A4078091A4079091A507CB
:10600000DC01ED91FC910280F381E02D19958091E6
:10601000A2079091A307DC01ED91FC910280F3812E
:10602000E02D199580910E13833039F0823009F0FC
:106030006CC08091C3128C3051F189E190E00E94D4
:10604000E4C4EC0183E696E09983888386E090E0DF
:106050009B838A8381E09FEF9D838C838FEF90E009
:106060009F838E8319861886188ECE010E940F4258
:1060700087E394E099838883D0939C07C0939B0720
:10608000CE010E94FC8B10921E0FC6E029C089E150
:1060900090E00E94E4C4EC0183E696E09983888353
:1060A00084E090E09B838A8381E09FEF9D838C83D3
:1060B0008FEF90E09F838E8319861886188ECE010D
:1060C0000E940F4287E394E099838883D0939C07D2
:1060D000C0939B07CE010E94FC8B1092240FC4E05A
:1060E0006091D2127091D3128C2F0E94284160913E
:1060F000D4127091D5128C2F0E9424418091D61217
:10610000E0919B07F0919C07808FE091C4128E2F45
:10611000EE0F990BAA0BBB0BFC013897E830F10589
:1061200008F0BBC08827E25BFE4F8F4F0C94D0C4B1
:1061300084E290E00E94E4C4FC018091811328E095
:1061400030E03383228321E03FEF358324832FEF38
:1061500030E03783268311861086108E94E8918F65
:106160002BE938E0338F228F27E634E03183208318
:1061700026E633E131A320A312A283A31EC080E24E
:1061800090E00E94E4C4FC0188E090E09383828365
:1061900081E09FEF958384838FEF90E097838683E0
:1061A00011861086108E87E8818F8BE998E0938F97
:1061B000828F8BE594E091838083F093A907E0932D
:1061C000A80799C080E290E00E94E4C4FC0188E046
:1061D00090E09383828381E09FEF958384838FEFA8
:1061E00090E09783868311861086108E8DE0818FD4
:1061F0008BE998E0938F828F8FE494E0DCCF89E184
:1062000090E00E94E4C4FC0188E090E093838283E4
:1062100081E09FEF958384838FEF90E0978386835F
:1062200011861086108E83E494E091838083F0932E
:10623000A907E093A8071092300F5DC08CE190E0B1
:106240000E94E4C4EC0183E696E09983888385E0AC
:1062500090E09B838A8381E09FEF9D838C838FEF07
:1062600090E09F838E8319861886188ECE010E9437
:106270000F4287E596E037C089E190E00E94E4C4D0
:10628000FC011382128215821482178216821186F3
:106290001086108E8FE194E08ECF8CE08093C41234
:1062A0006CE070E08EE191E00E94986B89E190E0F3
:1062B0000E94E4C4EC0183E696E09983888385E03C
:1062C00090E09B838A8381E09FEF9D838C838FEF97
:1062D00090E09F838E8319861886188ECE010E94C7
:1062E0000F4287E394E099838883D093A907C093F2
:1062F000A8071092210F8091A8079091A907DC01AF
:10630000ED91FC910280F381E02D19958091CC12E2
:10631000843658F4853608F084E664E6681B80917C
:10632000A8079091A9070E94CE4D8091C4128C506D
:106330008230A8F46091CD127091CE1285E00E9457
:106340005A406091CF127091D01285E00E943F4078
:106350008091D112E091A807F091A907808F209138
:10636000C512822F022E000C990BAA0BBB0BFC014D
:106370003897E830F10508F089C08827EA5AFE4FBF
:106380008F4F0C94D0C484E290E00E94E4C4FC01DE
:106390008091811329E030E03383228321E03FEFB5
:1063A000358324832FEF30E03783268311861086D0
:1063B000108E94E8918F2BE938E0338F228F27E6F7
:1063C00034E03183208326E633E131A320A312A2F7
:1063D00083A357C080E290E00E94E4C4FC0189E0FE
:1063E00090E09383828381E09FEF958384838FEF96
:1063F00090E09783868311861086108E87E8818FC0
:106400008BE998E0938F828F8BE594E038C080E22F
:1064100090E00E94E4C4FC0189E090E093838283D1
:1064200081E09FEF958384838FEF90E0978386834D
:1064300011861086108E8DE0818F8BE998E0938F06
:10644000828F8FE494E01BC080910E13823009F09C
:10645000C9C28091C3128C3009F0C4C21FC089E147
:1064600090E00E94E4C4FC0113821282158214821F
:106470001782168211861086108E8FE194E0918328
:106480008083F093AD07E093AC075EC080910E135C
:10649000823061F58091C3128C3041F58BE080939E
:1064A000C5126BE070E08FE191E00E94986B89E18A
:1064B00090E00E94E4C4FC0189E090E09383828331
:1064C00081E09FEF958384838FEF90E097838683AD
:1064D00011861086108E83E494E091838083F0937C
:1064E000AD07E093AC071092330F2EC08CE0809381
:1064F000C5126CE070E08FE191E00E94986B89E139
:1065000090E00E94E4C4EC0183E696E099838883DE
:1065100084E090E09B838A8381E09FEF9D838C835E
:106520008FEF90E09F838E8319861886188ECE0198
:106530000E940F4287E394E099838883D093AD074C
:10654000C093AC071092240F8091AC079091AD07D7
:10655000DC01ED91FC910280F381E02D1995809191
:10656000CB12843658F4853608F084E664E6681B5E
:106570008091AC079091AD070E94CE4D8091C512DD
:106580008C50823000F56091C6127091C71284E081
:106590000E945A406091C8127091C91284E00E9412
:1065A0003F408091CA12E091AC07F091AD07808F17
:1065B0008091C5128D3039F48091CA12E091AE13EA
:1065C000F091AF13808F8EE190E00E94E4C4EC0163
:1065D000D090DB12A090DF12B090E0128090DD121C
:1065E0009090DE1283E696E09983888383E090E0C2
:1065F0009B838A8381E09FEF9D838C83EE24EA94C2
:10660000F12CFF82EE8219861886188ECE010E9428
:106610000F428BE294E0998388839A8E898EBC8E98
:10662000AB8EDD8ED093460FC093450F6091E11283
:106630007091E21283E00E945A406091E3127091DF
:10664000E41283E00E943F408091DB12E091450F0D
:10665000F091460F808F8091DB120E94636B8091D6
:10666000450F9091460FDC01ED91FC910280F38182
:10667000E02D19958091E6128823A1F18BE390E03B
:106680000E94E4C4FC018091F0129091EF122091DD
:10669000F5123091F6124091F3125091F41260917C
:1066A000F1127091F212A091EB12B091EC12C09124
:1066B000E912D091EA12C090E712D090E81211824C
:1066C0001082F382E28215821482D4A2C3A2D6A3DE
:1066D000C5A3B0A7A7A372A761A754A743A736A7CE
:1066E00025A72FC08BE390E00E94E4C4FC018091B9
:1066F000F0129091EF122091F5123091F612409124
:10670000F3125091F4126091F1127091F212A09173
:10671000E912B091EA12C091E712D091E812118209
:106720001082F382E28215821482D4A3C3A3B6A39B
:10673000A5A370A767A352A741A734A723A7F6A6CE
:10674000E5A62BE938E030AB27A726E633E132ABEC
:1067500021AB93AB84ABF0932A07E0932907C09158
:106760002907D0912A072FA138A54BA15CA18DA1A3
:106770009EA1421753071CF4821793077CF0281739
:1067800039071CF44817590764F0241735075CF4DF
:106790008417950744F4142F052F05C0122F032FDB
:1067A00002C0182F092F1F821E82188709871B8697
:1067B0001A861D861C861E870F87198A188A2DA5A2
:1067C0003EA549A55AA58BA59CA5421753071CF4C5
:1067D000821793077CF0281739071CF448175907CC
:1067E00064F0241735075CF48417950744F4142FDC
:1067F000052F05C0122F032F02C0182F092F1B8A47
:106800001A8A1C8B0D8B1F8A1E8A198E188E1A8F5E
:106810000B8F1D8E1C8E1AAE19AE18A28BA981305B
:1068200069F08230E9F0811183C061E08CE20E945E
:10683000094B10922D0110922C017AC061E08CE27C
:106840000E94094B10922D0110922C0161E088E00A
:106850000E94094B60E070E088E00E94454B68C0F0
:10686000E9A9FAA980819181A281B3818115964914
:10687000A105B10509F457C040E056E960E070E0B9
:106880008FA598A90E945B8164E170E080E090E0B0
:106890000E94504CE9A9FAA980819181A281B3811B
:1068A00081152BE49207A105B105E9F068F4803663
:1068B00029E09207A105B105A1F080389542A10514
:1068C000B105C1F442E012C0811521EE9207A10585
:1068D000B10559F08115924CA140B10559F445E03C
:1068E00005C041E003C043E001C046E06FE0CE01D7
:1068F0000E94C23C8FA598A9DC01ED91FC91068015
:10690000F781E02D1995E9A9FAA9408151816281A9
:1069100073818FA598A90E945B8164E170E080E09B
:1069200090E00E94504C4AE06EE0CE010E94C23CD2
:106930008091F0128093F4078091300F8823F9F052
:1069400089E190E00E94E4C4FC0188E090E0938338
:106950008283158214828FEF93E0978386838FEF73
:1069600091E091878087108E83E494E09183808307
:10697000F0932F0FE0932E0FCF010E94C68C8091D1
:10698000330F882309F478C089E190E00E94E4C4C1
:10699000FC0189E090E093838283158214828FEF5B
:1069A00093E0978386838FEF91E091878087108EA5
:1069B00083E494E091838083F093320FE093310F6E
:1069C000CF01DF91CF911F910F91FF90EF90DF905A
:1069D000CF90BF90AF909F908F907F906F905F907F
:1069E0000C94C68C2C3009F48ACD8CE190E00E9486
:1069F000E4C4EC0193E6692E96E0792E79826882F0
:106A000024E0822E912C9B828A82AA24A394BB2408
:106A1000BA94BD82AC82CC24CA94D12CDF82CE82BF
:106A200019861886188ECE010E940F4257E5E52E72
:106A300056E0F52EF982E882D093AD07C093AC07FB
:106A40008CE190E00E94E4C4EC01798268829B8230
:106A50008A82BD82AC82DF82CE8219861886188E29
:106A60000E940F42F982E882D093AF13C093AE1315
:106A7000CE010E949C8C66CDDF91CF911F910F912A
:106A8000FF90EF90DF90CF90BF90AF909F908F904E
:106A90007F906F905F9008952F923F924F925F92F8
:106AA0006F927F928F929F92AF92BF92CF92DF921E
:106AB000EF92FF920F931F93CF93DF93CDB7DEB783
:106AC000CE5AD1090FB6F894DEBF0FBECDBFCDB6FA
:106AD000DEB6C455DF4F1882CC5AD040C555DF4FC3
:106AE0001882CB5AD0408091B20E8B3709F4E8C19E
:106AF00080F4873709F4D7C238F48F3109F445C5DB
:106B0000863709F4E0C107C68937B9F008F4DAC25C
:106B100034C0803809F472C438F48C3709F4E1C207
:106B20008E3709F42DC3F7C5823809F408C508F477
:106B30001DC5833809F4E6C4EEC50E9422440E94B4
:106B4000B3842B013C010E9454A1029709F428C58B
:106B50000E94B384DC01CB0184199509A609B70909
:106B600080329340A105B10508F01AC50E94A564C2
:106B70000E9422440E94939FE6CF0E9454A1029754
:106B800029F060E084E80E9447A08BC18091F60B59
:106B9000823031F0833039F482E080937A0F03C081
:106BA00081E08093E20E81E08093BC0E8E0104555B
:106BB0001F4F2FE0AE0140575F4F68E871E90E9418
:106BC000D09F0E9427A1893058F0015011092FE071
:106BD000AE014F575F4F68E872E981E00E94D09F95
:106BE0001092BB0E772473940E943DA1882309F470
:106BF0003DC1198222961FAE22971091BB0E111132
:106C00000EC0BE0160577F4FCE018F5B9F4F0E9429
:106C100002C7C455DF4F0881CC5AD04011C0113093
:106C200071F4BE016F577F4FCE018F5B9F4F0E9463
:106C300002C7C555DF4F0881CB5AD04001C000E0E4
:106C4000ADB6BEB68091F20BEDB7FEB722E0829FE3
:106C5000E019F10911240FB6F894FEBF0FBEEDBF85
:106C60008DB79EB701967C016DE876E0CE018B551D
:106C70009F4F0E9437478091F60B823089F0833016
:106C800061F1813009F0A1C04091F20B50E0B701F1
:106C90008091C9149091CA140E94889E10E039C056
:106CA0002091F20B30E05FB7F89440E0842F90E041
:106CB0008217930774F4880F991FF701E80FF91FE3
:106CC000DC01AF53B14F8D919C91918380834F5FD5
:106CD000EDCF5FBF1092E10E1CC02091F20B30E0AF
:106CE0005FB7F89440E0842F90E08217930774F424
:106CF000880F991FF701E80FF91FDC01AD56B04F5F
:106D00008D919C91918380834F5FEDCF5FBF1092F7
:106D1000C6146DE270E0CE018B559F4F0E943A463B
:106D20002091F20B293048F0112321F0113021F489
:106D300018E004C028E001C020E010E0121758F568
:106D4000F701E10FF11DE10FF11D608171814AE052
:106D5000CE0181569F4FC355DF4F2883CD5AD04077
:106D60000E94E046BE0161567F4FCE018B559F4F7A
:106D70000E946146CE0181569F4F0E94DB46CE01A4
:106D80008B559F4F0E94CA6E1F5FC355DF4F2881EE
:106D9000CD5AD040D3CF40E450E0BE016F5F7F4F6B
:106DA000CE018B559F4F0E94C26EC755DF4F188191
:106DB000C95AD040CE018B559F4F0E94DB460FB67B
:106DC000F894BEBE0FBEADBE0BC0CE018B559F4F1B
:106DD0000E94DB460FB6F894BEBE0FBEADBE10E0FB
:106DE000BE016F5F7F4FCE018F5B9F4F0E9402C736
:106DF000010F10E0E1E4F0E0EC0FFD1FE00FF11FE8
:106E00001082BE016F5B7F4F8091AA149091AB14EA
:106E10000E94AE48B801CE018F5B9F4F0E94B09F89
:106E2000BC018091AA149091AB140E94876C6AE017
:106E30008091AA149091AB140E94CA478091AA1421
:106E40009091AB14DC01ED91FC910680F781E02D6F
:106E500019950E9427A1893048F08091BB0E8111BD
:106E600003C07092BB0E02C01092BB0E0E9422445F
:106E70000E94939F0E94528D81110EDE8091B10E6F
:106E800081110FC08091BC0E882359F08091AC1401
:106E9000811107C08091AF0E9091B00E0A970CF44B
:106EA000A3CE8091F60B823039F0833009F033C4E1
:106EB00081E080937A0F2FC481E08093E20E2BC48F
:106EC0001092BC0E5FC31091B50E8FEF810F85300D
:106ED00028F060E089E80E9447A01DC4133079F0D3
:106EE00018F41230F9F004C0143079F0153099F02C
:106EF00040E6442E49E0542E612C712C19C0412CDF
:106F00003BE4532E612C712C13C0412C26E9522EE8
:106F1000612C712C0DC0412C92EC592E6624639487
:106F2000712C06C080E8482E85E2582E612C712C09
:106F300000E0E12EF12C5701BFE8AB0EB11C1501AA
:106F4000E89427F83324E6E9EE0EF11CE894E7F81C
:106F5000FF24023091F018F4013051F004C00330E6
:106F600089F00430A1F040E659E060E070E013C021
:106F700040E855E260E070E00EC040E05BE460E0B5
:106F800070E009C040E056E960E070E004C040E015
:106F900052EC61E070E08BE998E00E945B818BE944
:106FA00098E00E944A450E94B3844B015C01F2E3E1
:106FB0008F0E911CA11CB11C0E94539F0E94B38490
:106FC000681579058A059B05B8F360E870E08BE9E0
:106FD00098E00E94438F6FE070E08BE998E00E9498
:106FE000438F612F8BE998E00E940445B1018BE942
:106FF00098E00E94438F0E94B3844B015C012AE019
:10700000820E911CA11CB11C0E94539F0E94B3844C
:10701000681579058A059B05B8F367E870E08BE988
:1070200098E00E94438F6FE070E08BE998E00E9447
:10703000438F612F8BE998E00E940445B7018BE9EB
:1070400098E00E94438F8BE998E00E944A450E9495
:10705000B3844B015C013EE5830E31E0931EA11C1D
:10706000B11C0E94539F0E94B384681579058A055C
:107070009B05B8F30F5F053009F06BCFB301A20198
:107080008BE998E00E945B814092661350926713EF
:107090006092681370926913B301A20180EC91E0D1
:1070A0000E94FD6E6FC283E090E00E94E4C42AE07B
:1070B000DC012C932BE938E012963C932E93119728
:1070C0006AE00CC083E090E00E94E4C42DE0FC0183
:1070D00020832BE938E0328321836DE00E94CF6664
:1070E00051C24091B50E5091B60E0091B70E10915D
:1070F000B80E6091B30E7091B40ECE010196C355D7
:10710000DF4F4883CD5AD040C255DF4F5883CE5A07
:10711000D0400E940B92C355DF4F4881CD5AD040DA
:10712000C255DF4F5881CE5AD040892BE9F08D816E
:10713000873050F4853080F48130B0F0642F8B813B
:107140009C810E94F26C0DC0893070F4B8018B8173
:107150009C810E94FD6E05C0BA018B819C810E94BA
:10716000986B0E94C2A004C061E085E80E9447A01D
:107170008091AE0E8111CFC281E08093AE0ECBC262
:10718000B090B30EE090B40EC156DF4F1882CF59C5
:10719000D0406DE876E0CE018F579F4F0E94374771
:1071A0006B2D7E2DCE0180579F4F0E940B92892B15
:1071B00009F4BEC0CC56DF4FE881C459D0404E2FF1
:1071C00050E0FA013197E830F10508F0B1C08827A6
:1071D000E25AFE4F8F4F0C94D0C4CE56DF4F8881B9
:1071E0009981C259D0400E9494C24AE0682FCE01D2
:1071F00001960E940B471BC0CE56DF4F88819981B4
:10720000C259D0400E9494C2682F880F770B4AE081
:107210000AC0CE56DF4F88819981C259D0400E9462
:10722000A1C24AE0BC01CE0101960E94E046BE0127
:107230006F5F7F4FCE018F579F4F0E940146CE0157
:10724000019663C0CE56DF4F88819981C259D040E4
:107250000E94A1C223961FAE1EAE239725961FAE95
:107260001EAE259727961FAE1EAE27974AE0BE0199
:107270006F5F7F4F0E9442C135C0CE56DF4F88817D
:107280009981C259D0400E949CC223961FAE1EAE67
:10729000239725961FAE1EAE259727961FAE1EAECE
:1072A00027972AE0AE014F5F5F4F0E9409C11AC0C5
:1072B000CE56DF4F88819981C259D0400E949CC22E
:1072C00023961FAE1EAE239725961FAE1EAE2597A2
:1072D00027961FAE1EAE27972AE0AE014F5F5F4F85
:1072E0000E9417C1BE016F5F7F4FCE018F5B9F4F22
:1072F0000E94BB46BE016F5B7F4FCE018F579F4FF1
:107300000E940146CE018F5B9F4F0E94DB464FE0FB
:1073100050E0BE016F5B7F4FCE018F579F4F0E94A1
:10732000C26ECB57DF4FF880C558D04011E002C085
:10733000F12C10E0CE018F579F4F0E94DB461123A6
:1073400009F4C7CD8E0101561F4F20E4AE014F5FF7
:107350005F4F68E87B2D8E2D0E94D09FBE016F5B32
:107360007F4FCE0101960E9402C7C156DF4F888130
:10737000CF59D040F80E81E08F0DC156DF4F888382
:10738000CF59D040E1E0F0E0EC0FFD1FEF0DF11D13
:107390009CE79083E1E0F0E0EC0FFD1FE80FF11DAA
:1073A0001082BE016F5F7F4F8091AA149091AB1441
:1073B0000E94AE48C156DF4F6881CF59D04070E07F
:1073C000CE0101960E94B09FBC018091AA149091B9
:1073D000AB140E94876C6AE08091AA149091AB1460
:1073E0000E94CA478091AA149091AB14DC01ED91E0
:1073F000FC910680F781E02D19958DC18091B30E27
:107400009091B40E8038910509F085C18E01005726
:107410001F4F20E4AE014F5F5F4F68E870E880E0E7
:107420000E94D09F6BE676E0CE018F579F4F0E945F
:107430003747CE018F579F4F0E94CA6EC057DF4F0C
:107440002881C059D040CB57DF4F88819981C558DA
:10745000D040820F911DC057DF4F8883C059D04064
:1074600022961FAE22974FE050E0BE016F5B7F4F28
:10747000CE018F579F4F0E949F6EBE016F5B7F4F63
:10748000CE0101960E9402C7C057DF4F8881C059C4
:10749000D040E1E0F0E0EC0FFD1FE80FF11D10829D
:1074A000BE016F5F7F4F8091AA149091AB140E9430
:1074B000AE48C057DF4F6881C059D04070E0CE0160
:1074C00001960E94B09FBC018091AA149091AB14C8
:1074D0000E94876C6AE08091AA149091AB140E947C
:1074E000CA478091AA149091AB14DC01ED91FC91F4
:1074F0000680F781E02D1995CE018F579F4F0E948E
:10750000DB4609C18091B30E9091B40E833891058A
:1075100009F001C18E0100571F4F20E4AE014F5FFB
:107520005F4F68E873E880E00E94D09F4AE0609176
:10753000AD0ECE018F579F4F0E940B477ACF80919F
:10754000B30E9091B40E8238910509F0E4C08E011B
:1075500000571F4F20E4AE014F5F5F4F68E872E8AD
:1075600080E00E94D09F63E876E05ECF8091B30E0A
:107570009091B40E8138910509F0CDC08091BC0E78
:107580008111C9C00E94C2A0C6C08091B30E909163
:10759000B40E4F9709F0BFC081E08093B10EBBC01D
:1075A0000E9454A1029719F060E084E894CC809185
:1075B000F50B811102C00E940C6D0E9427A1F82ECC
:1075C0006DE876E0CE0180579F4F0E943747C15645
:1075D000DF4F1882CF59D0408E0101561F4F20E453
:1075E000AE014F5F5F4F68E879E780E00E94D09F6F
:1075F000CF57DF4F19821882C158D040CD57DF4F87
:1076000019821882C358D040CB57DF4F1982188295
:10761000C558D0406F2D70E080E090E02AE0AE01C8
:107620004F5B5F4F0E9409C1BE016F5B7F4FCE0170
:107630008F579F4F0E94BB46BE016F577F4FCE01B1
:1076400080579F4F0E940146CE018F579F4F0E9447
:10765000DB464FE050E0BE016F5B7F4FCE018057AD
:107660009F4F0E949F6ECC56DF4F1881C459D04067
:10767000BE016F5B7F4FCE0101960E9402C7C156CB
:10768000DF4F8881CF59D040810F91E0980FC156CC
:10769000DF4F9883CF59D040E1E0F0E0EC0FFD1FC1
:1076A000E80FF11D8CE78083E1E0F0E0EC0FFD1FB7
:1076B000E90FF11D1082BE016F5F7F4F8091AA1408
:1076C0009091AB140E94AE48C156DF4F6881CF59EC
:1076D000D04070E0CE0101960E94B09FBC01809125
:1076E000AA149091AB140E94876C6AE08091AA144E
:1076F0009091AB140E94CA478091AA149091AB1448
:10770000DC01ED91FC910680F781E02D1995CE0109
:1077100080579F4FF4CE0FB6F894DEBE0FBECDBE9D
:10772000C255DF4F0FB6F894DEBF0FBECDBFDF915D
:10773000CF911F910F91FF90EF90DF90CF90BF906E
:10774000AF909F908F907F906F905F904F903F9001
:107750002F900895FC0182810895482F50E095E113
:10776000899FF0011124EC51FF4E218132818085E7
:107770009185280F391F838194818217930728F000
:107780008581968128173907E8F485E1849FF00107
:10779000859FF00D1124EC51FF4E858196812817AD
:1077A000390728F52581368185E1849FF001859F81
:1077B000F00D1124EC51FF4E8285823019F41186B0
:1077C0001086128685E1849FF001859FF00D1124BB
:1077D000EC51FF4E3283218380918400909185008B
:1077E000280F391F309389002093880008958381E2
:1077F000948182179307C0F623813481D5CF62E349
:107800000C94238A61E30C94238A60E30C94238A0A
:1078100064E50C94238A6FE20C94238A6DE20C9445
:10782000238A6CE20C94238A77FF03C071956195DB
:10783000710920E0462F6EE20C94DD89462F20E08E
:107840006DE40C94DD89FC016283611105C020E0C8
:1078500040E06BE40C94DD89089577FF03C07195D7
:107860006195710920E0462F6BE40C94DD894F92FD
:107870005F926F927F928F929F92AF92BF92CF92C0
:10788000DF92EF92FF920F931F93CF93DF936C01E0
:10789000A4ECCA1AADEFDA0AD601ED91FC917E97FD
:1078A0000CF05DC0FC01E858FF4F812C912CA19198
:1078B000B191AB2B21F42115310549F450C0BFEF34
:1078C0008B1A9B0AAEE18A16910489F748C0EC0135
:1078D0005401AA0CBB1CAA0CBB1CAC0EBD1EF501AE
:1078E000EC54FF4F40835183628373837401EE0C29
:1078F000FF1CEC0EFD1EF701E858FF4F318320837B
:10790000EC54FF4F11830083BE01680D791DFB010C
:10791000EC55FE4F81E080830E94B384F5016083C3
:10792000718382839383C65CDD4F88819981F701DF
:10793000E250FE4F91838083D6012D913C911197A7
:107940002F5F3F4F2D933C939C012F5F3F4F1216AB
:10795000130614F021E030E03983288302C08FEF52
:107960009FEFDF91CF911F910F91FF90EF90DF90EC
:10797000CF90BF90AF909F908F907F906F905F90CF
:107980004F9008950F931F93CF93DF938C01C62FD1
:10799000D42F65E870E0DC019F968D919C91D09783
:1079A0000E94438FF80187A590A9DC01ED91FC911D
:1079B0000190F081E02D6C2F1995F80187A590A911
:1079C000DC01ED91FC910190F081E02D6D2F199576
:1079D0002C2F30E0B9016B577F4F6D0F711D6F7702
:1079E0007727F80187A590A9DF91CF911F910F917B
:1079F0000C94438F262F2B7FA1F49A014F3F510502
:107A000019F014F02FEF30E0A90141302FEF5207A9
:107A100014F441E05FEF57FF03C0519541955109C0
:107A2000B1CF0895CF93DF93EC0189AD9AAD892B47
:107A300011F01AAE19AECE010E9433818BA98130AC
:107A400029F0823069F0811117C005C060E070E054
:107A500088E00E94454B10922D0110922C0108C025
:107A600040E064E0CE018EDF40E060E0CE018ADFDE
:107A70001AA219A21F8E1E8E0E94B3846DAB7EAB1C
:107A80008FAB98AFDF91CF9108958F929F92AF9275
:107A9000BF92CF92DF92EF92FF920F931F93DC0180
:107AA00014968D919C9115975696CD90DC90579792
:107AB0006817790709F455C09096FC9090974C018F
:107AC000092E000CAA08BB088B01072E000C220B04
:107AD000330B861797073CF41296ED91FC911397A0
:107AE000FF2031F014C0ED91FC911197FF2079F047
:107AF0000D2C000CEE08FF08A9019801281939097E
:107B00004A095B0954966D917C9155970EC00D2CD6
:107B1000000CEE08FF08A9019801281939094A0943
:107B20005B0952966D917C915397CB01770FAA0B0D
:107B3000BB0BBC01CD016C197D098E099F090E9408
:107B40009AC48F01FF0F220B330BA901980128194A
:107B500039094A095B090E94B4C2C20ED31EE41E51
:107B6000F51EC6011F910F91FF90EF90DF90CF900F
:107B7000BF90AF909F908F9008958F929F92AF92F9
:107B8000BF92CF92DF92EF92FF920F931F93DC018F
:107B900014968D919C9115971A96CD90DC901B9719
:107BA0006817790709F455C09096FC9090974C019E
:107BB000092E000CAA08BB088B01072E000C220B13
:107BC000330B861797073CF41296ED91FC911397AF
:107BD000FF2031F014C0ED91FC911197FF2079F056
:107BE0000D2C000CEE08FF08A9019801281939098D
:107BF0004A095B0918966D917C9119970EC00D2C5E
:107C0000000CEE08FF08A9019801281939094A0952
:107C10005B0916966D917C911797CB01770FAA0B94
:107C2000BB0BBC01CD016C197D098E099F090E9417
:107C30009AC48F01FF0F220B330BA9019801281959
:107C400039094A095B090E94B4C2C20ED31EE41E60
:107C5000F51EC6011F910F91FF90EF90DF90CF901E
:107C6000BF90AF909F908F900895EF92FF920F93E7
:107C70001F93CF93DF93EC0189AD9AAD892B11F05F
:107C80001AAE19AE8BA98130B1F0823059F1811151
:107C900043C0CB0177FF03C0919581959109BC0149
:107CA000CE016BDF90932D0180932C019AA389A3C1
:107CB0009F8F8E8F31C08B0177FF03C01195019587
:107CC0001109B801CE0159DF7C01B801CE01DDDE1A
:107CD0008C01B70188E00E94454B10932D01009361
:107CE0002C0116C08B0177FF03C011950195110976
:107CF000B801CE0142DF7C01B801CE01C6DE8C01A5
:107D0000A70164E0CE0176DEA80160E0CE0172DE5C
:107D1000FAA2E9A21F8F0E8F0E94B3846DAB7EABD7
:107D20008FAB98AFDF91CF911F910F91FF90EF90A4
:107D30000895CF93DF93EC0189AD9AAD892B11F0B3
:107D40001AAE19AE2FA138A58DA19EA19F838E8357
:107D5000398728879B878A872DA53EA58BA59CA55B
:107D60009B8B8A8B3D8B2C8B9F8B8E8B60E070E086
:107D7000CE017BDF0E94B3846DAB7EAB8FAB98AF3F
:107D8000DF91CF910895CF93DF93EC0189AD9AAD48
:107D9000892B11F01AAE19AE2FA138A58BA19CA189
:107DA0009F838E83398728879B878A872DA53EA549
:107DB00089A59AA59B8B8A8B3D8B2C8B9F8B8E8B59
:107DC00060E070E0CE0151DF0E94B3846DAB7EAB0A
:107DD0008FAB98AFDF91CF910895DC01A250BE4FD9
:107DE00020E030E04D915D914617570739F4280F98
:107DF000391FF901EC55FE4F808108952F5F3F4FE9
:107E00002E31310579F780E00895CF93DF93EC01AF
:107E1000C45CDD4FA881B981109709F442C0FC0110
:107E2000E250FE4F20E030E0419151914617570754
:107E300099F5A901440F551F480F591FFA01E85839
:107E4000FF4F60817181672B61F111821082FC010B
:107E5000E20FF31FEC55FE4F1082FA01EE53FE4F76
:107E600011821082235D3F4F220F331F220F331FD9
:107E7000FC01E20FF31F1082118212821382FA01B9
:107E8000E859FE4F11821082EA56FF4F118210828C
:107E90001197B983A88305C02F5F3F4F2E3131055D
:107EA00019F6DF91CF9108950F931F9301E010E031
:107EB000DEDC1F910F9108950F931F9300E010E0F7
:107EC000D6DC1F910F9108952F923F924F925F92AF
:107ED0006F927F928F929F92AF92BF92CF92DF92DA
:107EE000EF92FF920F931F93CF93DF9300D000D0B8
:107EF000CDB7DEB78C010E94B38498012E533E4F5C
:107F00003C832B831E830D83D801AC55BE4FBA83AF
:107F1000A9831801B2E02B1ABEEF3B0AF901AA248B
:107F2000A394B12C32E0832E912C118210829F01F8
:107F30002A543140D9012D913C91232B09F44DC095
:107F4000AD81BE812D913D914D915C9113977D0145
:107F5000B4EBEB0EF11CD701CD90DD90ED90FC90D1
:107F60002B013C01421A530A640A750A4C145D0441
:107F70006E047F0490F1C20ED31EE41EF51EAD8187
:107F8000BE81CD92DD92ED92FC921397A981BA81C8
:107F90002C91222311F19F0126593109D9012D91EC
:107FA0003C912115310519F4B182A08216C07F01E0
:107FB000BAE5EB1AF108D7014D915C911197421780
:107FC00053075CF4B182A0824F5F5F4F4D935C9387
:107FD0004217530714F09182808232962D813E81A0
:107FE0002C5F3F4F3E832D83A981BA811196BA83BE
:107FF000A983E215F30509F098CFEB81FC8181910B
:108000009191FC83EB838130910599F00297C9F43B
:10801000EB81FC81EC54F1400190F081E02D199549
:10802000AB81BC81DA966D917C91DB97C801EDDE66
:1080300008C0EB81FC81EC54F1400190F081E02D0F
:1080400019952B813C8122153305B9F626960FB67A
:10805000F894DEBF0FBECDBFDF91CF911F910F917E
:10806000FF90EF90DF90CF90BF90AF909F908F9058
:108070007F906F905F904F903F902F9008956E3E4D
:1080800022E0720738F06B3C98E0790728F06AEC40
:1080900078E002C06EEE72E0660F771F9FB7F8942B
:1080A00025E1829FF0011124EC51FF4E748363831C
:1080B0009FBF08956E3E22E0720738F06B3C98E057
:1080C000790728F06AEC78E002C06EEE72E0660F85
:1080D000771F9FB7F89425E1829FF0011124EC519E
:1080E000FF4E768365839FBF0895660F771F282F05
:1080F00030E095E1899FF0011124EC51FF4E85811C
:1081000096816817790718F46581768107C08381A5
:1081100094818617970710F4638174818FB7F89460
:1081200095E1929FF001939FF00D1124EC51FF4EC9
:10813000728361838FBF0895982F8FB7F89425E1DC
:10814000929FF0011124EC51FF4E21E027838FBF55
:1081500041B121E030E0B90102C0660F771F9A9566
:10816000E2F7CB01842B81B908958A3058F49FB788
:10817000F89425E1829FF0011124EC51FF4E118605
:1081800010869FBF08951F93CF93DF9325E1829FB1
:10819000C0011124EC01CC51DF4E8A8581110FC042
:1081A0001FB7F89481E08A8789899A899A8389839D
:1081B0000E94B3846B877C878D879E871FBFDF916A
:1081C000CF911F910895CF93DF938A30D0F562331A
:1081D000710538F061369DE6790728F060E67DE6A6
:1081E00002C062E370E0D42FC82F80E090E00E94CC
:1081F0006FC120E030E04AE754E40E9476C320E0FB
:1082000030E04CE852E40E94D0C19B01AC0160E038
:1082100070E08AEF94E40E9476C30E94DEC39B0163
:10822000DD2321F022273327261B370B8FB7F89445
:1082300095E1C99FF0011124EC51FF4E3187208751
:108240008FBFDF91CF9108958A3008F418CF089539
:108250008A3008F42FCF08958A3058F495E1899F29
:10826000F0011124EC51FF4E818192819695879502
:10827000089580E090E008958A3008F436CF08959C
:108280001F920F920FB60F9211240BB60F920F93FD
:108290001F932F933F934F935F936F937F938F938E
:1082A0009F93AF93BF93CF93EF93FF938091040F6E
:1082B000893048F01092040F80919311882399F02F
:1082C00080918C110DC0E091040FE15025E1E29FF7
:1082D000F0011124EC51FF4E8781882321F0808129
:1082E00092B1892782B9E091040F85E1E89FF001FE
:1082F0001124EC51FF4E8781882321F0808192B1B7
:10830000892B82B9E091040FC5E1CE9FF0011124C1
:10831000EC51FF4E80859185892B09F04DC0E0918D
:10832000040FCE9FF0011124EC51FF4E8285813065
:1083300009F060C00E94B384E091040FCE9FF00169
:108340001124EC51FF4E0385148525853685E09177
:10835000040FCE9FF0011124EC51FF4E0784F089E9
:10836000E02DAB01BC01401B510B620B730BCF0125
:10837000A0E0B0E084179507A607B707D8F5E0910D
:10838000040FA091040FCA9FD0011124AC51BF4E1D
:1083900053968D919C915497CE9FF0011124EC51EE
:1083A000FF4E91878087E091040FCE9FF00111244A
:1083B000EC51FF4E82E082878091040FCED98091EC
:1083C000040F8F5F8093040FFF91EF91CF91BF91C6
:1083D000AF919F918F917F916F915F914F913F915D
:1083E0002F911F910F910F900BBE0F900FBE0F900A
:1083F0001F901895E091040F809184009091850062
:1084000025E1E29FF0011124EC51FF4E21813281E0
:10841000820F931F9093890080938800D0CF1F9381
:10842000CF93DF938091030F811173C01092040FDB
:108430009FB7F89485E128EB3BE04CED55E064E90B
:1084400071E1A1E0B0E0E091040FE93008F052C022
:10845000E091040F8E9FF0011124EC51FF4E328306
:108460002183E091040F8E9FF0011124EC51FF4E07
:1084700056834583E091040F8E9FF0011124EC5147
:10848000FF4E74836383E091040FF091040FED01BC
:1084900001C0CC0FFA95EAF78E9FF0011124EC5140
:1084A000FF4EC083E091040F8E9FF0011124EC5128
:1084B000FF4E1782E091040F8E9FF0011124EC51C2
:1084C000FF4E11861086E091040F8E9FF00111245B
:1084D000EC51FF4E1286E091040F8E9FF0011124A3
:1084E000EC51FF4E148A138AE091040FEF5FE09382
:1084F000040FA9CF9FBF8FB7F89420EA3FE03093D5
:108500008E1120938D1110928C118FBF81E080937A
:10851000030FDF91CF911F9108950F931F93CF9376
:10852000DF938C01C62FD42FDC0111968D919C9185
:108530001297DC01ED91FC910190F081E02DD801C2
:108540006C911995F80181819281DC01ED91FC918A
:108550000190F081E02D6C2F1995F80181819281B5
:10856000DC01ED91FC910190F081E02D6D2F1995CA
:10857000F80180816C2F70E0680F711D6D0F711D07
:108580006F77772781819281DF91CF911F910F9132
:108590000C94438F0F931F93CF93DF938C01C62FBF
:1085A000D42FDC0111968D919C911297DC01ED91F5
:1085B000FC910190F081E02DD8016C911995F801A2
:1085C00081819281DC01ED91FC910190F081E02D9F
:1085D0006C2F1995F80181819281DC01ED91FC915C
:1085E0000190F081E02D6D2F1995F80180816C2F9D
:1085F00070E0680F711D6D0F711D6F777727818196
:108600009281DF91CF911F910F910C94438F4F92E4
:108610005F926F927F92AF92BF92CF92DF92EF9272
:10862000FF921F93CF93DF93DD24D39445E0C42EB4
:10863000C2E0D0E053E0E52EF12CAA24A394B12CA3
:108640008091E70E9091E80EDC01ED91FC910084A1
:10865000F185E02D1995892B09F4D1C010913001D5
:108660008091E70E9091E80EDC01ED91FC9102847F
:10867000F385E02D199596B3B39A2091840030913B
:1086800085002059384E30938D0020938C00212F87
:108690002C7119F01092020F2AC093FB992790F9C0
:1086A000E091020FE11116C0992351F28F3041F68B
:1086B000D092020F8093E90E8091E50E9091E60E24
:1086C000892B09F0BDCFB092E60EA092E50E109274
:1086D000E40EB6CF992381F01092020F1092E40EAF
:1086E0008091E50E9091E60E029709F0A9CFF092E5
:1086F000E60EE092E50EA4CF91E09E0F9093020F5C
:10870000F0E0E751F14F8083993109F099CF811161
:1087100073C08091000F82FF05C0F092E60EE092D8
:10872000E50E6AC083FDF9CF8091E50E9091E60ECB
:10873000019761F48091E40E8F5F8093E40E8430A2
:1087400058F0D093E60EC093E50E06C0D093E60E27
:10875000C093E50E1092E40E8091E30E8F5F80933C
:10876000E30E9091E20E981708F044C0D092E10E0B
:10877000A1ECBEE0EAEEFEE040E050E0BA0110E01D
:10878000CF01FC011B3098F401964080512C612CE4
:10879000712C012E04C0440C551C661C771C0A94D5
:1087A000D2F74429552966297729185FEACF9A011B
:1087B0003770205E3340C29EC001C39E900D1124CD
:1087C00097FD079623E0959587952A95E1F78452C2
:1087D0009A4F8D939D931B503BE0769567955795E7
:1087E00047953A95D1F78EE0A13EB80749F6109229
:1087F000E30E02C01092E10E1092020F21CFDF9122
:10880000CF911F91FF90EF90DF90CF90BF90AF90EE
:108810007F906F905F904F9008958091F60B83301A
:1088200031F48091BF0E9091C00E0C9491990895EF
:108830008091F60B823029F48091BD0E9091BE0E8E
:10884000E6CE0895F5DFE9CF1092BD101092C71063
:108850001092D1101092DB101092651080E090E021
:10886000FC01E859FF4E1182079684359105C1F746
:1088700008950895CF92DF92EF92FF920F931F9386
:10888000CF93DF936C017A018B01C0E0D0E0CE156D
:10889000DF0589F0D8016D918D01D601ED91FC9134
:1088A0000190F081E02DC6011995892B11F47E010C
:1088B00002C02196ECCFC701DF91CF911F910F919C
:1088C000FF90EF90DF90CF900895FC01A089B189CF
:1088D0008C91A689B78982FD0FC09C91818D8F5F95
:1088E0008F73228D821749F0218DDF01A20FB11DF8
:1088F0005D969C93818F08958C910895089580E0F2
:1089000090E00895FC01538D448D252F30E0842F95
:1089100090E0821B930B541710F0CF9608950197A7
:108920000895FC01918D828D981761F0828DDF0191
:10893000A80FB11D5D968C91928D9F5F9F73928F52
:1089400090E008958FEF9FEF0895FC01918D828D47
:10895000981731F0828DE80FF11D858D90E0089514
:108960008FEF9FEF0895FC01918D228D892F90E06C
:10897000805C9F4F821B91098F73992708958EEF1A
:1089800097E0F1DF21E0892B09F420E0822F0895A0
:108990008BE998E0E8DF21E0892B09F420E0822FC1
:1089A000089588E399E0DFDF21E0892B09F420E0D6
:1089B000822F089585ED99E0D6DF21E0892B09F417
:1089C00020E0822F0895FC01848DDF01A80FB11DE6
:1089D000A35ABF4F2C91848D90E001968F739927F5
:1089E000848FA689B7892C93A089B1898C918064E2
:1089F0008C93938D848D981306C00288F389E02DA3
:108A000080818F7D80830895EF92FF920F931F9353
:108A1000CF93DF93EC0181E0888F9B8D8C8D981331
:108A200005C0E889F989808185FD23C0F62E0B8D6C
:108A300010E00F5F1F4F0F731127E02E8C8DE8128F
:108A40000BC00FB607FCFACFE889F989808185FF52
:108A5000F5CFCE01B8DFF2CF8B8DFE01E80FF11D0F
:108A6000E35AFF4FF0820B8FEA89FB898081806295
:108A700007C0EE89FF896083E889F9898081806475
:108A8000808381E090E0DF91CF911F910F91FF9063
:108A9000EF900895CF93DF93EC01888D8823C1F088
:108AA000EA89FB89808185FD05C0A889B9898C91F7
:108AB00086FD0EC00FB607FCF5CF808185FFF2CF93
:108AC000A889B9898C9185FFEDCFCE017CDFE8CFF5
:108AD000DF91CF91089580E090E0892B19F06ADF53
:108AE000811116C080E090E0892B19F05ADF8111C6
:108AF00012C080E090E0892B19F04ADF81110EC08E
:108B000080E090E0892B79F03ADF81110AC0089566
:108B10000E940000E7CF0E940000EBCF0E940000FF
:108B2000EFCF0C940000089590E0FC013197E23102
:108B3000F10508F04EC08827EA59FE4F8F4F0C947C
:108B4000D0C4809180008F7703C0809180008F7D9A
:108B500080938000089580918000877FF9CF84B54D
:108B60008F7702C084B58F7D84BD08958091B00059
:108B70008F7703C08091B0008F7D8093B0000895FF
:108B8000809190008F7707C0809190008F7D03C007
:108B900080919000877F8093900008958091A0003D
:108BA0008F7707C08091A0008F7D03C08091A000C7
:108BB000877F8093A0000895809120018F7707C060
:108BC000809120018F7D03C080912001877F809359
:108BD000200108950E94F5C66115710579F0FB0129
:108BE00001900020E9F73197AF01461B570BDC01DC
:108BF000ED91FC910280F381E02D199480E090E0EA
:108C000008950F931F93CF93DF938C01EB01FC0129
:108C1000808191810097B1F068817981611571053A
:108C200079F0428153812C813D814217530740F0F6
:108C30000E940DC78C819D81F8019583848313C0A8
:108C40000E9479C588819981F801918380838A8106
:108C50009B81938382838C819D81958384831982F8
:108C600018821B821A821D821C82DF91CF911F9174
:108C70000F9108950F931F93CF93DF93EC01888199
:108C80009981009729F02A813B812617370788F4BC
:108C90008B016F5F7F4F0E9411C6009761F099832F
:108CA00088831B830A832C813D81232B11F4FC01D3
:108CB000108281E001C080E0DF91CF911F910F9180
:108CC0000895EF92FF920F931F93CF93DF93FB01D1
:108CD00024813581E080F180FC0104811581E1145B
:108CE000F10411F480E016C02115310591F0EC017A
:108CF000020F131FB801BEDF8823A1F32881398139
:108D00008C819D81B701820F931F0E940DC71D8327
:108D10000C8381E0DF91CF911F910F91FF90EF9035
:108D20000895EF92FF920F931F93CF93DF93EC017F
:108D30007B018A01BA019EDF2881398181110DC032
:108D40002115310519F0C9010E9479C519821882CF
:108D50001D821C821B821A8206C01D830C83B701F0
:108D6000C9010E940DC7CE01DF91CF911F910F91D4
:108D7000FF90EF900895CF93DF93EC01611571059B
:108D800051F0FB0101900020E9F73197AF01461B3C
:108D9000570BC7DF0CC088819981009711F00E94A2
:108DA00079C5198218821D821C821B821A82CE010B
:108DB000DF91CF910895FC01808191810C9479C558
:108DC0000F931F93CF93DF93CDB7DEB762970FB6A4
:108DD000F894DEBF0FBECDBF8C01CB01F80111822C
:108DE0001082138212821582148250E0BE016F5FDE
:108DF0007F4F0E94F5C0BE016F5F7F4FC801BBDF90
:108E000062960FB6F894DEBF0FBECDBFDF91CF9153
:108E10001F910F9108950F931F93CF93DF93CDB7B9
:108E2000DEB729970FB6F894DEBF0FBECDBF8C0119
:108E3000862FF80111821082138212821582148209
:108E400050E0BE016F5F7F4F90E00E9438C1BE01CD
:108E50006F5F7F4FC8018FDF29960FB6F894DEBF92
:108E60000FBECDBFDF91CF911F910F910895FC01EF
:108E7000118210821382128215821482611571058B
:108E800049F0FB0101900020E9F73197AF01461B43
:108E9000570B47CF0895CF93DF9300D01F92CDB7E4
:108EA000DEB7611571058105910579F09B01AC0173
:108EB00069833A834B835C830E94E9C029813A81AC
:108EC0004B815C810E94B4C203C060E070E0CB01C2
:108ED0000F900F900F900F90DF91CF9108954F92C8
:108EE0005F926F927F92EF92FF920F931F93CF93B7
:108EF000DF93CDB7DEB7A1970FB6F894DEBF0FBEF4
:108F0000CDBF7C01FA01CB0119A2223008F42AE07E
:108F10008E010F5D1F4F422E512C612C712CBF0111
:108F2000A30192010E94E0C2F901CA010150110996
:108F30006A3014F4605D01C0695CD8016C93232B26
:108F4000242B252B61F7B801C70146DEA1960FB689
:108F5000F894DEBF0FBECDBFDF91CF911F910F916F
:108F6000FF90EF907F906F905F904F9008956BE827
:108F700076E032CE0F931F93CF93DF93EC012CDE7C
:108F80008C01CE01F4DF800F911FDF91CF911F91F3
:108F90000F910895DC01ED91FC910190F081E02D9D
:108FA00019944F925F926F927F928F929F92AF929D
:108FB000BF92CF92DF92EF92FF92CF93DF93EC01BB
:108FC0006A017B01B22E9A01AB01C701B6010E9472
:108FD00019C4882319F06EE876E027C0260137010E
:108FE000E89477F82FEF3FEF4FE75FE7C301B20157
:108FF0000E9419C481110DC02FEF3FEF4FE75FE7CB
:10900000C301B2010E946BC118161CF462E976E03C
:109010000CC02FEF3FEF4FE75FE4C701B6010E949E
:109020000FC4181694F466E976E0CE01DF91CF9173
:10903000FF90EF90DF90CF90BF90AF909F908F9078
:109040007F906F905F904F90C7CD2FEF3FEF4FE72E
:109050005FECC701B6010E946BC187FDE4CF20E041
:1090600030E0A901C701B6010E946BC187FF09C0AA
:109070006DE2CE018FDF4C01F7FAF094F7F8F0942F
:1090800002C0812C912CA12C60E070E080E09FE375
:10909000AB1441F020E030E040E251E40E9476C39E
:1090A000A394F6CF9B01AC01C701B6010E9412C385
:1090B0002B013C010E94E3C36B017C010E946FC144
:1090C0009B01AC01C301B2010E9411C32B013C0101
:1090D0002AE0B701A601CE0102DF7C01E80CF91CF1
:1090E000BB2029F06EE2CE0155DFE80EF91EDB2C25
:1090F000DD2021F120E030E040E251E4C301B20183
:109100000E94D0C12B013C010E94E3C34B01A12C62
:10911000B12C2AE0B501A401CE01E1DEE80EF91E72
:10912000C501B4010E946FC19B01AC01C301B20132
:109130000E9411C32B013C01DA94DACFC701DF9101
:10914000CF91FF90EF90DF90CF90BF90AF909F9026
:109150008F907F906F905F904F9008953DCDEF92EC
:10916000FF920F931F93CF93DF938C017B01C0E09D
:10917000D0E0F701EC0FFD1F6491662361F0D80188
:10918000ED91FC910190F081E02DC8011995892B9A
:1091900011F02196EECFCE01DF91CF911F910F916B
:1091A000FF90EF9008950F931F93CF93DF93EC01FF
:1091B000D6DF8C01CE01DBDE800F911FDF91CF91D6
:1091C0001F910F9108951F920F920FB60F921124C5
:1091D0000BB60F922F933F934F935F936F937F93B1
:1091E0008F939F93AF93BF93EF93FF938EEF97E08F
:1091F000EADBFF91EF91BF91AF919F918F917F91AA
:109200006F915F914F913F912F910F900BBE0F90F7
:109210000FBE0F901F9018951F920F920FB60F92CE
:1092200011240BB60F922F933F934F935F936F933D
:109230007F938F939F93AF93BF93EF93FF938EEFA3
:1092400097E043DBFF91EF91BF91AF919F918F9199
:109250007F916F915F914F913F912F910F900BBE36
:109260000F900FBE0F901F9018951F920F920FB680
:109270000F9211240BB60F922F933F934F935F934E
:109280006F937F938F939F93AF93BF93EF93FF93CE
:109290008BE998E098DBFF91EF91BF91AF919F919F
:1092A0008F917F916F915F914F913F912F910F908F
:1092B0000BBE0F900FBE0F901F9018951F920F922C
:1092C0000FB60F9211240BB60F922F933F934F932B
:1092D0005F936F937F938F939F93AF93BF93EF931E
:1092E000FF938BE998E0F1DAFF91EF91BF91AF9195
:1092F0009F918F917F916F915F914F913F912F91AE
:109300000F900BBE0F900FBE0F901F9018951F92DD
:109310000F920FB60F9211240BB60F922F933F931B
:109320004F935F936F937F938F939F93AF93BF936D
:10933000EF93FF9388E399E046DBFF91EF91BF91B4
:10934000AF919F918F917F916F915F914F913F91DD
:109350002F910F900BBE0F900FBE0F901F9018957E
:109360001F920F920FB60F9211240BB60F922F93EC
:109370003F934F935F936F937F938F939F93AF939D
:10938000BF93EF93FF9388E399E09FDAFF91EF910A
:10939000BF91AF919F918F917F916F915F914F910D
:1093A0003F912F910F900BBE0F900FBE0F901F900B
:1093B00018951F920F920FB60F9211240BB60F92B1
:1093C0002F933F934F935F936F937F938F939F93CD
:1093D000AF93BF93EF93FF9385ED99E0F4DAFF919C
:1093E000EF91BF91AF919F918F917F916F915F911D
:1093F0004F913F912F910F900BBE0F900FBE0F908A
:109400001F9018951F920F920FB60F9211240BB652
:109410000F922F933F934F935F936F937F938F930D
:109420009F93AF93BF93EF93FF9385ED99E04DDA50
:10943000FF91EF91BF91AF919F918F917F916F912C
:109440005F914F913F912F910F900BBE0F900FBEE8
:109450000F901F901895CF93DF93EC01E881F9816D
:109460000680F781E02D1995EA89FB8980818F7E3E
:109470008083EA89FB898081877F8083EA89FB89F1
:1094800080818F778083EA89FB8980818F7D8083CB
:109490008A8D898FDF91CF910895CF92DF92EF92DD
:1094A000FF921F93CF93DF93EC016A017B01122F90
:1094B000E889F98982E080834115514E6105710583
:1094C000B1F060E079E08DE390E0A70196010E94A1
:1094D000E0C2DA01C9010197A109B109B695A795C2
:1094E00097958795AC01411580E15807A8F0E88968
:1094F000F989108260E874E88EE190E0A701960196
:109500000E94E0C2BA01A9014150510961097109E3
:109510007695679557954795EC85FD855083EE8543
:10952000FF854083188EEC89FD891083EA89FB89C9
:10953000808180618083EA89FB8980818860808363
:10954000EA89FB89808180688083EA89FB89808140
:109550008F7D8083DF91CF911F91FF90EF90DF90FF
:10956000CF900895CF93DF93282F30E0F901E75093
:10957000FE4E8491F901ED54FE4ED491F901E35968
:10958000FE4EC491CC2389F08111CEDAEC2FF0E0AD
:10959000EE0FFF1FED5AFE4EA591B491EC91ED2315
:1095A00081E090E021F480E002C080E090E0DF9173
:1095B000CF9108951F93CF93DF93282F30E0F901C7
:1095C000E750FE4E8491F901ED54FE4ED491F9011D
:1095D000E359FE4EC491CC23C1F0162F8111A4DAB9
:1095E000EC2FF0E0EE0FFF1FE75CFE4EA591B4916B
:1095F0008FB7F894111105C09C91ED2FE095E923E8
:1096000002C0EC91ED2BEC938FBFDF91CF911F91B6
:109610000895CF93DF9390E0FC01ED54FE4E24912A
:10962000FC01E359FE4E8491882361F190E0880F9C
:10963000991FFC01E15EFE4EC591D491FC01E75CEF
:10964000FE4EA591B491611109C09FB7F89488812D
:10965000209582238883EC912E230BC0623061F425
:109660009FB7F8943881822F809583238883EC916B
:109670002E2B2C939FBF06C08FB7F894E8812E2B1A
:1096800028838FBFDF91CF9108951F93CF93DF93EE
:10969000182FEB0161E0BDDF209711F460E004C0FA
:1096A000CF3FD10531F461E0812FDF91CF911F9140
:1096B00081CFE12FF0E0E750FE4EE4914E2F50E0D5
:1096C000FA013197E231F10508F09DC08827E8588A
:1096D000FE4F8F4F0C94D0C484B5806884BDC7BD45
:1096E00097C084B5806284BDC8BD92C0809180005F
:1096F000806880938000D0938900C093880088C0E0
:1097000080918000806280938000D0938B00C09312
:109710008A007EC080918000886080938000D09312
:109720008D00C0938C0074C08091B00080688093DD
:10973000B000C093B3006CC08091B0008062809391
:10974000B000C093B40064C08091900080688093A2
:109750009000D0939900C09398005AC080919000D7
:10976000806280939000D0939B00C0939A0050C079
:1097700080919000886080939000D0939D00C0936A
:109780009C0046C08091A00080688093A0008091DA
:10979000A0008F7B8093A000D093A900C093A80065
:1097A00037C08091A00080628093A000D093AB006E
:1097B000C093AA002DC08091A00088608093A00073
:1097C000D093AD00C093AC0023C08091200180688D
:1097D00080932001D0932901C093280119C0809162
:1097E0002001806280932001D0932B01C0932A0135
:1097F0000FC080912001886080932001D0932D01BB
:10980000C0932C0105C0C038D1050CF04CCF46CF19
:10981000DF91CF911F910895863308F08653909180
:109820007B00282F2870977F922B90937B00877066
:10983000806480937C0080917A00806480937A00B9
:1098400080917A0086FDFCCF80917800209179008C
:1098500090E0922B08953FB7F8948091050F909176
:10986000060FA091070FB091080F26B5A89B05C061
:109870002F3F19F00196A11DB11D3FBFBA2FA92F8F
:10988000982F8827820F911DA11DB11DBC01CD010C
:1098900042E0660F771F881F991F4A95D1F70895F8
:1098A0008F929F92AF92BF92CF92DF92EF92FF92F0
:1098B0006B017C01D0DF4B015C01C114D104E104D8
:1098C000F104E9F0C8DFDC01CB0188199909AA0984
:1098D000BB09883E9340A105B10578F321E0C21A87
:1098E000D108E108F10888EE880E83E0981EA11CDB
:1098F000B11CC114D104E104F10421F7DECFFF90C3
:10990000EF90DF90CF90BF90AF909F908F90089591
:1099100008950895089508951092DA0B0895CF934D
:10992000DF93EC0180910A0F811109C06A8D7B8D54
:10993000CE0149960E94D66B81E080930A0F21E800
:109940003FEF3B872A878FE790E09D878C871F86B4
:109950001E86398B288B9B8B8A8B1D8A1C8ADF91F4
:10996000CF9108950F931F93CF93DF93EC011F8A3C
:109970001E8A8C01075E1F4F40E060E0C8010E9414
:10998000CA4240E064E0C8010E94CA420E94B38417
:109990006C8F7D8F8E8F9F8FDF91CF911F910F9155
:1099A00008950F931F93CF93DF93EC018091090FDC
:1099B000811112C00A8D1B8D6AEA70E0C8010E94F5
:1099C000438FD801ED91FC910680F781E02DC8010D
:1099D000199581E08093090F4AE06EE0CE01499627
:1099E0000E94CA4221E83FEF3B872A878FE790E039
:1099F0009D878C871F861E86398B288B9B8B8A8B35
:109A00001D8A1C8ADF91CF911F910F9108950F93AA
:109A10001F93CF93DF93EC011F8A1E8A8C01075E90
:109A20001F4F40E060E0C8010E948D4240E064E0CA
:109A3000C8010E948D420E94B3846C8F7D8F8E8FEF
:109A40009F8FDF91CF911F910F9108950F931F93D7
:109A5000CF93DF93EC01E8A1F9A180819181A281EC
:109A6000B3818E01075E1F4F81159649A105B1058F
:109A700009F450C040E056E960E070E08BE998E0FE
:109A80000E945B8164E170E080E090E009DFE8A182
:109A9000F9A180819181A281B38181152BE4920784
:109AA000A105B105E9F068F4803629E09207A10527
:109AB000B105A1F080389542A105B105C1F442E09D
:109AC00012C0811521EE9207A105B10559F081154B
:109AD000924CA140B10559F445E005C041E003C0F6
:109AE00043E001C046E06FE0C8010E948D428BE96F
:109AF00098E00E944A45E8A1F9A140815181628124
:109B000073818BE998E00E945B8164E170E080E002
:109B100090E0C6DE4AE06EE0C8010E948D4241E05E
:109B200067E1C8010E948D424AA168E1C8010E9414
:109B30008D424BA18FEF840F8E3108F04CE066E12F
:109B4000C8010E948D4221E83FEF3B872A878FE7BB
:109B500090E09D878C871F861E86398B288B9B8B78
:109B60008A8B1D8A1C8ADF91CF911F910F910895D6
:109B70000C944A8FCF93DF93CCE6DBE081E090E05A
:109B80009A8389831092DA0B66DE6C837D838E83E1
:109B90009F83E49AEC9ADF91CF910895EF92FF9220
:109BA0000F931F93CF93DF93EC016623E1F0262FF1
:109BB000653608F024E60A891B89E888F988D80107
:109BC000AE19BF0930E00E94DEC428EC30E040E06E
:109BD00050E00E94E0C2E20EF31EFB86EA86021B02
:109BE000130B1D870C87DF91CF911F910F91FF9071
:109BF000EF900895CF93DF93CDB7DEB7A4970FB65C
:109C0000F894DEBF0FBECDBF81310CF081E12AE1B7
:109C100033E13A83298322E133E13C832B832AE039
:109C200033E13E832D8322E033E138872F832AEF0F
:109C300032E13A87298722EF32E13C872B872AEEEF
:109C400032E13E872D8722EE32E1388B2F8724EDDB
:109C500032E13A8B298B22EC32E13C8B2B8B25EACB
:109C600032E13E8B2D8B20E932E1388F2F8B26E8B5
:109C700032E13A8F298F2CE732E13C8F2B8F2FE690
:109C800032E13E8F2D8F23E632E138A32F8F27E478
:109C900032E13AA329A32FE332E13CA32BA3E82F1F
:109CA000EE0FFF0BEC0FFD1F81819281A4960FB682
:109CB000F894DEBF0FBECDBFDF91CF9108958F9294
:109CC0009F92AF92BF92CF92DF92EF92FF920F934B
:109CD0001F93DC0118968D919C9119971E96CD903B
:109CE000DC901F976817790709F456C05896FC90C6
:109CF00058974C01092E000CAA08BB088B01072EAF
:109D0000000C220B330B861797073CF41696ED9147
:109D1000FC911797FF2039F015C01496ED91FC9136
:109D20001597FF2079F00D2C000CEE08FF08A90113
:109D30009801281939094A095B091C966D917C9193
:109D40001D970EC00D2C000CEE08FF08A90198010C
:109D5000281939094A095B091A966D917C911B975C
:109D6000CB01770FAA0BBB0BBC01CD016C197D0990
:109D70008E099F090E949AC48F01FF0F220B330B9B
:109D8000A9019801281939094A095B090E94B4C23E
:109D9000C20ED31EE41EF51EC6011F910F91FF9047
:109DA000EF90DF90CF90BF90AF909F908F900895ED
:109DB000EF92FF920F931F93CF93DF938C01FC01DF
:109DC000778B668B7CDFEC01F80182819381883090
:109DD000910531F57801F9E1EF0EF11CD7FF06C0CE
:109DE0006AE0C1388FEFD80754F001C068E02C2F2B
:109DF0009D2FC038D1052CF02FE790E002C021E85C
:109E00009FEF422F592F57FF03C05195419551099C
:109E1000C7010E946D9ECD2B69F54FE766E027C014
:109E2000099741F57801E9E1EE0EF11CD7FF06C074
:109E30006EE0C138FFEFDF0754F001C06CE02C2F5B
:109E40009D2FC038D1052CF02FE790E002C021E80B
:109E50009FEF422F592F57FF03C05195419551094C
:109E6000C7010E946D9ECD2B29F44FE767E0C70123
:109E70000E946D9E0E94B384F801648F758F868F57
:109E8000978FDF91CF911F910F91FF90EF900895E1
:109E9000CF93DF93EC017F8B6E8B11DF9C018A8166
:109EA0009B8188309105C1F437FF06C061E02138FD
:109EB0008FEF38074CF001C060E0A9012038310570
:109EC0002CF04FE750E002C041E85FEF57FF1FC0A2
:109ED0005195419551091BC00997E9F4922F832FA1
:109EE0002038310514F09FE780E0492F582F413882
:109EF0008FEF580714F441E85FEF57FF03C0519507
:109F000041955109632F661F6627661F6C5FCE015E
:109F100049960E94CA420E94B3846C8F7D8F8E8FB7
:109F20009F8FDF91CF9108950F931F93CF93DF936E
:109F3000EC010E94B3840C8D1D8D2E8D3F8DDC01B4
:109F4000CB01801B910BA20BB30B853F9140A10568
:109F5000B10540F06E897F89CE01DF91CF911F91CD
:109F60000F9196CFDF91CF911F910F910895CF93CD
:109F7000DF93EC017F8B6E8BA2DE9C018A819B813B
:109F800088309105C1F437FF06C061E021388FEFBA
:109F900038074CF001C060E0A901203831052CF0F1
:109FA0004FE750E002C041E85FEF57FF1FC05195F7
:109FB000419551091BC00997E9F4922F832F20384E
:109FC000310514F09FE780E0492F582F41388FEF7B
:109FD000580714F441E85FEF57FF03C051954195CE
:109FE0005109632F661F6627661F6C5FCE01499675
:109FF0000E948D420E94B3846C8F7D8F8E8F9F8FC5
:10A00000DF91CF9108950F931F93CF93DF93EC01CE
:10A010000E94B3840C8D1D8D2E8D3F8DDC01CB01F4
:10A02000801B910BA20BB30B853F9140A105B1059D
:10A0300040F06E897F89CE01DF91CF911F910F9102
:10A0400096CFDF91CF911F910F910895CF93DF931A
:10A05000EC0161E089E0DDDA60E089E0ABDA1092E2
:10A06000DF0A83E395E099838883DF91CF91089598
:10A07000CF92DF92EF92FF928091E00A833009F055
:10A0800061C08091E10A8130D1F488EE93E0A0E0D4
:10A09000B0E08093720A9093730AA093740AB0930D
:10A0A000750A80E797E1A0E0B0E08093760A90938C
:10A0B000770AA093780AB093790A32E001C030E0C1
:10A0C000E091E10AF0E0EE51F54F2081A0E1A30F0D
:10A0D00048EE53E060E070E088EBC82E8BE0D82EAD
:10A0E000E12CF12C832F90E0FC01EE0FFF1FEE0F0F
:10A0F000FF1FEE58F54F27FF10C0C082D182E282C9
:10A10000F382880F991F880F991FFC01EA58F54FB9
:10A1100040835183628373830FC040835183628382
:10A120007383880F991F880F991FFC01EA58F54F18
:10A13000C082D182E282F3823E5F220F3A13D2CFF5
:10A140003093DB0AFF90EF90DF90CF900895CF938C
:10A15000DF938091DF0A811151C01092DD0A1092C5
:10A16000DA0AC1E0C093DF0AD091DE0A61E089E03B
:10A1700050DA60E089E01EDA2D2F30E040E050E058
:10A1800060E47FE180E090E00E94B4C2C093B00040
:10A1900089E08093B1002093B3008BEA289F212DA2
:10A1A000112426952093B40080916F008B7F8093BB
:10A1B0006F008091B00080628093B0002091840095
:10A1C00030918500E091DA0A81E08E0F8093DA0AFF
:10A1D00084E0E89FF0011124EE58F54F80819181D1
:10A1E000A281B381820F931F90938B0080938A008A
:10A1F000B29A80916F00846080936F00DF91CF915D
:10A2000008954F925F926F927F928F929F92AF923A
:10A21000BF92CF92DF92EF92FF928AE18093DB0AA6
:10A220002093DC0A88E28093DE0A81E08093E10AD1
:10A230008093E20A8EE08093E00A80EC92E1A0E055
:10A24000B0E08093720A9093730AA093740AB0935B
:10A25000750A80EB94E0A0E0B0E08093760A9093DA
:10A26000770AA093780AB093790AA4E1440F551FA6
:10A27000661F771FAA95D1F722E030E0B0EBCB2E16
:10A28000B4E0DB2EE12CF12C80E6482E89E0582E3C
:10A29000612C712C90E4892E9CE9992EA12CB12C73
:10A2A000C901880F991F880F991FFC01EE58F54FBF
:10A2B00077FF05C0408251826282738204C0C082EF
:10A2C000D182E282F382C9010196880F991F880F1B
:10A2D000991FFC01EE58F54F283129F0C082D18238
:10A2E000E282F38204C080829182A282B382440F10
:10A2F000551F661F771F2E5F3F4F2A31310581F6AC
:10A30000FF90EF90DF90CF90BF90AF909F908F9095
:10A310007F906F905F904F901ACF8F929F92AF92E5
:10A32000BF92CF92DF92EF92FF9282E18093DB0A9D
:10A3300086E08093DC0A96E29093DE0A91E09093A7
:10A34000E10A9093E20A8093E00A88ED90E4A0E0AD
:10A35000B0E08093720A9093730AA093740AB0934A
:10A36000750A8CE19CE0A0E0B0E08093760A9093BF
:10A37000770AA093780AB093790A742F6627552735
:10A38000442722E030E0ACE1CA2EACE0DA2EE12C2A
:10A39000F12CB8E38B2EB8E19B2EA12CB12CC90176
:10A3A000880F991F880F991FFC01EE58F54F77FF12
:10A3B00005C080829182A282B38204C0C082D18211
:10A3C000E282F382F901EE0FFF1FEE0FFF1FEA5842
:10A3D000F54FC082D182E282F382440F551F661F7F
:10A3E000771F2E5F3F4F22313105C9F68CE199E886
:10A3F000A0E0B0E08093B60A9093B70AA093B80AA1
:10A40000B093B90AFF90EF90DF90CF90BF90AF90DC
:10A410009F908F909CCE1F920F920FB60F92112497
:10A420000BB60F922F933F934F935F936F937F934E
:10A430008F939F93AF93BF93EF93FF939091DA0A1B
:10A440008091DB0A981316C01092DA0A8091E10A13
:10A450008F5F8093E10A9091E10A8091E20A891767
:10A4600040F481E08093E10A8091DD0A8F5F809360
:10A47000DD0AFEDD9091DD0A8091DC0A98130DC0A3
:10A480008091B0008F7D8093B00080916F008B7FB2
:10A4900080936F001092DF0A27C08091B00085FF83
:10A4A00004C08091B0008F7D03C08091B0008062B5
:10A4B0008093B0002091840030918500E091DA0A09
:10A4C00081E08E0F8093DA0A84E0E89FF001112486
:10A4D000EE58F54F80819181A281B381820F931F45
:10A4E00090938B0080938A00FF91EF91BF91AF9181
:10A4F0009F918F917F916F915F914F913F912F919C
:10A500000F900BBE0F900FBE0F901F9018951F92CB
:10A510000F920FB60F9211240BB60F921F932F9329
:10A520003F934F935F936F937F938F939F93AF93DB
:10A53000BF93EF93FF93CF93DF9300D01F92CDB7DC
:10A54000DEB780916C0B0ED811E0892B09F010E07A
:10A5500082D969837A838B839C8389819A81AB8139
:10A56000BC814091700B5091710B6091720B709196
:10A57000730B841B950BA60BB70B20916D0B3091C1
:10A580006E0B2430310509F44CC02530310521F023
:10A5900021303105E9F414C020916F0B222339F0EA
:10A5A0002091DA0B20FF02C0289A01C028981123BD
:10A5B00079F0813E2EE29207A105B10548F02BC04B
:10A5C000112379F125E030E030936E0B20936D0B71
:10A5D00020916D0B30916E0B2530310511F5E09116
:10A5E000DA0BF0E0EE0FFF1FEC58F44F91838083FD
:10A5F00089819A81AB81BC818093700B9093710BA0
:10A60000A093720BB093730B8091DA0B8F5F8093E2
:10A61000DA0B833330F084E090E090936E0B8093FC
:10A620006D0B0F900F900F900F90DF91CF91FF91D6
:10A63000EF91BF91AF919F918F917F916F915F91BA
:10A640004F913F912F911F910F900BBE0F900FBE16
:10A650000F901F9018958091AE0780938F130895E7
:10A660008091330F882359F08091310F9091320FF0
:10A67000DC01ED91FC910480F581E02D19940895A1
:10A680008091330F882369F08091310F9091320FC0
:10A69000DC01ED91FC910190F081E02D6FEF73E012
:10A6A000199408958091330F882389F080913E0F8B
:10A6B000882321F080E090E0D3DF03C080E090E0C9
:10A6C000DFDF90913E0F81E0892780933E0F089550
:10A6D0002091330F222369F0A091310FB091320FF6
:10A6E000ED91FC9111970190F081E02DBC01CD011D
:10A6F000199408958091300F882359F080912E0F7E
:10A7000090912F0FDC01ED91FC910480F581E02DFB
:10A71000199408958091300F882369F080912E0F4D
:10A7200090912F0FDC01ED91FC910190F081E02DD3
:10A730006FEF73E0199408958091300F882389F0AA
:10A7400080913D0F882321F080E090E0D3DF03C0AB
:10A7500080E090E0DFDF90913D0F81E089278093DA
:10A760003D0F08952091300F222369F0A0912E0F04
:10A77000B0912F0FED91FC9111970190F081E02D98
:10A78000BC01CD011994089520912D0F222369F069
:10A79000A0912B0FB0912C0FED91FC91119701908E
:10A7A000F081E02DBC01CD011994089520912A0F6C
:10A7B000222369F0A091280FB091290FED91FC910F
:10A7C00011970190F081E02DBC01CD0119940895FD
:10A7D0002091270F222369F0A091250FB091260F19
:10A7E000ED91FC9111970190F081E02DBC01CD011C
:10A7F000199408952091240F222369F0A091220F2B
:10A80000B091230FED91FC9111970190F081E02D13
:10A81000BC01CD01199408952091210F222369F0E4
:10A82000A0911F0FB091200FED91FC911197019015
:10A83000F081E02DBC01CD011994089520911E0FE7
:10A84000222369F0A0911C0FB0911D0FED91FC9196
:10A8500011970190F081E02DBC01CD01199408956C
:10A8600020911B0F222369F0A091190FB0911A0FAC
:10A87000ED91FC9111970190F081E02DBC01CD018B
:10A88000199408958091AA079091AB07DC01ED918E
:10A89000FC91EE59FF4F0190F081E02D19948091C9
:10A8A000AA079091AB07DC01ED91FC91E05AFF4FB4
:10A8B0000190F081E02D19948091AA079091AB0747
:10A8C000DC01ED91FC91E25AFF4F0190F081E02D07
:10A8D00019948091AE07882361F00E9454A10297D9
:10A8E00041F06EE074E180918D1390918E130C9481
:10A8F000D348089580918F13882341F060E673E177
:10A9000080918D1390918E130C94D348089580916B
:10A910008F13882341F060E573E180918D1390914E
:10A920008E130C94D3480895CF93DF932091410F59
:10A930003091420F28173907D1F09093420F80933E
:10A94000410F20918F13222391F0EC016FED73E101
:10A9500080918D1390918E130E94AF48BE0180911B
:10A960008D1390918E13DF91CF910C941A68DF9123
:10A97000CF910895CF93DF9320913F0F3091400FF7
:10A9800028173907D1F09093400F80933F0F209103
:10A990008F13222391F0EC0165EC73E180918D130C
:10A9A00090918E130E94AF48BE0180918D139091BB
:10A9B0008E13DF91CF910C941A68DF91CF91089597
:10A9C00020912D0F222339F0BC018091170F909117
:10A9D000180F0C944A8F089520912A0F222339F0E2
:10A9E000BC018091150F9091160F0C944A8F089519
:10A9F0002091270F222339F0BC018091130F9091F1
:10AA0000140F0C944A8F08952091240F222339F0BB
:10AA1000BC018091110F9091120F0C944A8F0895F0
:10AA20002091210F222339F0BC0180910F0F9091CA
:10AA3000100F0C944A8F089520911E0F222339F095
:10AA4000BC0180910D0F90910E0F0C944A8F0895C8
:10AA500020911B0F222339F0BC0180910B0F9091A4
:10AA60000C0F0C944A8F0895CF92DF92EF92FF92D1
:10AA700020910002213019F42091FB1204C02230F1
:10AA8000C9F5209101132223A9F19C01211584E02D
:10AA9000380710F02FEF33E0ADE0B0E00E9402C3C2
:10AAA0002FEF33E040E050E00E94B4C269017A0128
:10AAB0008FEFC81AD80AE80AF80A80919D148C15FD
:10AAC000C9F0C0929D1480918F13882399F06EEA8B
:10AAD00073E180918D1390918E130E94AF486C2D7D
:10AAE00080918D1390918E13FF90EF90DF90CF9017
:10AAF0000C94C06AFF90EF90DF90CF900895CF92B2
:10AB0000DF92EF92FF9220910002213019F4209100
:10AB1000F81204C02230C9F52091FE122223A9F1B7
:10AB20009C01211584E0380710F02FEF33E0ADE0F1
:10AB3000B0E00E9402C32FEF33E040E050E00E94FB
:10AB4000B4C269017A018FEFC81AD80AE80AF80A74
:10AB500080919B148C15C9F0C0929B1480918F1327
:10AB6000882399F067E973E180918D1390918E139A
:10AB70000E94AF486C2D80918D1390918E13FF90A1
:10AB8000EF90DF90CF900C94C06AFF90EF90DF9031
:10AB9000CF90089583E08093A70781E0FAD6809153
:10ABA0008F13882341F06AE873E180918D139091AF
:10ABB0008E130C94D348089582E08093A70781E018
:10ABC000E8D680918F13882341F060E773E180918C
:10ABD0008D1390918E130C94D348089581E0809347
:10ABE000A707A9D680918F13882341F06DE773E101
:10ABF00080918D1390918E130C94D34808950C94EA
:10AC00000C978091350F81110BC081E09091F0126B
:10AC1000911101C080E08093340F81E08093350F63
:10AC20008091340F882329F00E94F9961092340FF6
:10AC300008950E940C9781E08093340F08950C943E
:10AC4000F9968091E612811111C0809129079091A7
:10AC50002A07FC0121A132A1121613061CF460E0A0
:10AC600070E002C06FEF70E00C94353E0895809163
:10AC7000E612811108C060E070E080912907909190
:10AC80002A070C94353E08958091E612811108C080
:10AC90006FEF70E08091290790912A070C94353E60
:10ACA00008950C94CC978091010281110C94B29775
:10ACB0000C94CC970C94B29784E60C94515F89E184
:10ACC0000C94515F82E30C94515F8BE40C94515FC0
:10ACD00080910002813011F482E001C081E00C9487
:10ACE000F45F82E00C94F45F81E00C94F45F0C94C8
:10ACF000D90ECF93DF93CDB7DEB765970FB6F89433
:10AD0000DEBF0FBECDBF8091491290914A122091B3
:10AD10004712309148123A8329839C838B8381E0C8
:10AD20008D8B82E08F938DB79EB745970FB6F894C1
:10AD30009EBF0FBE8DBFADB7BEB7119685E1FE01B8
:10AD4000319601900D928A95E1F78BE39CE00E9489
:10AD500039930FB6F894DEBF0FBECDBF80918F132D
:10AD6000882381F065E373E180918D1390918E13B8
:10AD700065960FB6F894DEBF0FBECDBFDF91CF91C1
:10AD80000C94D34865960FB6F894DEBF0FBECDBFC6
:10AD9000DF91CF91089580914A07882339F08BE3A2
:10ADA0009CE00E94D1942EEE31E706C08BE39CE03C
:10ADB0000E94F8942EEA31E74CE251E060E070E046
:10ADC0008DE69CE00E94543F80918F13882341F0D0
:10ADD00062E273E180918D1390918E130C94D348AD
:10ADE0000895682F80918D1390918E130E94D76AD9
:10ADF0006CE074E180918D1390918E130C94AF48A8
:10AE000020918D1330918E13882319F062E078E041
:10AE100002C066E078E0C9010C94AF48F1DF809190
:10AE20008D1390918E130C94B74720918D13309110
:10AE30008E13882319F061E074E102C066E074E1CA
:10AE4000C9010E94AF4880918D1390918E130C948C
:10AE5000B74780918D1390918E130C94B7476FEF85
:10AE600073E180918D1390918E130C94AF486BEF2A
:10AE700073E180918D1390918E130C94AF48CF9312
:10AE8000CDE269EF73E180918D1390918E130E9452
:10AE9000AF48C150B1F780918D1390918E130E94ED
:10AEA000B74780918D1390918E13DC01ED91FC9149
:10AEB0000680F781E02DCF9119940C94CE710C94FB
:10AEC0000A720C94F2700C942D7180914F0F8823AC
:10AED00019F00E94F27002C00E942D7190914F0FE4
:10AEE00081E0892780934F0F08950C94AE710C94E4
:10AEF000EE718BE39CE00E94E49481110C94AE719E
:10AF00000C94EE718AE09CE00E94E49481110C9410
:10AF1000CE710C940A728091AA079091AB07DC0164
:10AF2000ED91FC91EA5BFF4F0190F081E02D1995C6
:10AF300080918F13882341F06AE975E180918D1328
:10AF400090918E130C94D3480895CF93DF93CDB78F
:10AF5000DEB765970FB6F894DEBF0FBECDBF809108
:10AF6000491290914A1220914712309148123A8327
:10AF700029839C838B8381E08D8B82E08F938DB7B7
:10AF80009EB745970FB6F8949EBF0FBE8DBFADB765
:10AF9000BEB7119685E1FE01319601900D928A951A
:10AFA000E1F78AE09CE00E9439930FB6F894DEBF87
:10AFB0000FBECDBF80918F13882381F062EC75E1C5
:10AFC00080918D1390918E1365960FB6F894DEBF25
:10AFD0000FBECDBFDF91CF910C94D34865960FB6CD
:10AFE000F894DEBF0FBECDBFDF91CF9108950E94D0
:10AFF000F270409174135091751360E070E02DE28F
:10B0000031E78DE69CE00E94543F9093701480934A
:10B010006F1480918F13882341F06DE475E1809166
:10B020008D1390918E130C94D34808950E942D7126
:10B03000409174135091751360E070E022EF30E797
:10B040008DE69CE00E94543F9093701480936F149F
:10B0500080918F13882341F06AE375E180918D130D
:10B0600090918E130C94D3480895809144078823BF
:10B0700039F08AE09CE00E94D1942AE032E706C0D1
:10B080008AE09CE00E94F8942EEC31E74CE251E01B
:10B0900060E070E08DE69CE00E94543F80918F1349
:10B0A000882341F06FEA75E180918D1390918E13A2
:10B0B0000C94D348089569E081E00C94279668E0E9
:10B0C00081E00C94279667E081E00C94279661E07C
:10B0D00081E00C94279669E080E00C94279668E064
:10B0E00080E00C94279667E080E00C94279661E05E
:10B0F00080E00C9427968CE00C9474968BE00C9472
:10B1000074968AE00C94749689E00C94749688E0A6
:10B110000C94749687E00C94749686E00C94749664
:10B1200085E00C94749684E00C94749683E00C94FF
:10B13000749682E00C94749681E00C9474968CE082
:10B140000C949B968BE00C949B968AE00C949B96B7
:10B1500089E00C949B9688E00C949B9687E00C9475
:10B160009B9686E00C949B9685E00C949B9684E0DD
:10B170000C949B9683E00C949B9682E00C949B9697
:10B1800081E00C949B968CE00C94C2968BE00C941E
:10B19000C2968AE00C94C29689E00C94C29688E02C
:10B1A0000C94C29687E00C94C29686E00C94C296EA
:10B1B00085E00C94C29684E00C94C29683E00C94D3
:10B1C000C29682E00C94C29681E00C94C2960C94D4
:10B1D000E1960C94ED960F931F93CF93DF9300911C
:10B1E0004A0F10914B0FC0911B07D0911C07B8015B
:10B1F000CE010E94ED3E882379F0B801CE010E9475
:10B20000053F80911D0790911E07DC01ED91FC9197
:10B2100002A0F3A1E02D19950091480F1091490F5C
:10B22000C0911B07D0911C07B801CE010E94ED3ED2
:10B23000882321F0B801CE010E94053F59988091E2
:10B240008F13882361F06CED74E180918D139091E0
:10B250008E13DF91CF911F910F910C94D348DF9102
:10B26000CF911F910F910895CF93DF9380916E142A
:10B27000882321F110926E1460E088E00E94DA4A7F
:10B28000C0916F14D0917014BE018DE69CE00E94B5
:10B29000ED3E882329F0BE018DE69CE00E94053F2B
:10B2A00080918F13882371F061E875E180918D138F
:10B2B00090918E13DF91CF910C94D348DF91CF9171
:10B2C0000C941F95DF91CF91089580916E14811198
:10B2D00002C00C941F950895CF93DF938091711451
:10B2E000882311F10E94F27010927114C0916F14B2
:10B2F000D0917014BE018DE69CE00E94ED3E882343
:10B3000029F0BE018DE69CE00E94053F80918F13DD
:10B31000882371F068E675E180918D1390918E130A
:10B32000DF91CF910C94D348DF91CF910C9442716F
:10B33000DF91CF9108950C9442718091500F882332
:10B3400019F00E94F27002C00E94C5729091500FD5
:10B3500081E089278093500F08950C94C5720C9456
:10B36000D8720C94EF7280914E0F882319F00E94CE
:10B37000D87202C00E94EF7290914E0F81E089272F
:10B3800080934E0F08950C943A730E943A73809103
:10B39000AA079091AB07DC01ED91FC9106A0F7A103
:10B3A000E02D19940C94777380914D0F882319F038
:10B3B0000E943A7302C00E94777390914D0F81E012
:10B3C000892780934D0F08950C9493730C94AF7359
:10B3D00080914C0F882319F00E94937302C00E9441
:10B3E000AF7390914C0F81E0892780934C0F0895A3
:10B3F0000E94A78680918F138823D1F020914D134E
:10B4000080918D1390918E13211107C020915013BC
:10B41000211103C064EE74E109C02091E10B2223E5
:10B4200019F063E275E102C06FE075E10C94D34856
:10B4300008958091E10B81110C949F860C94A7864E
:10B440000E949F8680918F13882341F06EE275E100
:10B4500080918D1390918E130C94D34808950C9481
:10B460007EA28091E3138111BAC60C947EA2B7C666
:10B470000E947E718091AA079091AB07DC01ED914B
:10B48000FC9104A0F5A1E02D1994CF93DF93C09116
:10B490001B07D0911C0760914A0F70914B0FCE0192
:10B4A0000E94ED3E811129C04091470F50E060E0BD
:10B4B00070E02EE531E8CE010E945C3F90934B0F87
:10B4C00080934A0F80911D0790911E07DC01ED913A
:10B4D000FC9100A0F1A1E02D1995809137078823F8
:10B4E00061F06091480F7091490F80911B07909116
:10B4F0001C070E94ED3E882371F080918F138823F2
:10B50000E9F063ED74E180918D1390918E13DF91DA
:10B51000CF910C94D3480E945A842AE534E844E63B
:10B5200050E060E070E080911B0790911C070E9442
:10B530005C3F9093490F8093480FDFCFDF91CF910D
:10B5400008950E94BD8680918F13882341F068EA98
:10B5500074E180918D1390918E130C94D3480895CB
:10B56000E091450FF091460F82810E94C340809187
:10B570008F13882341F06AE874E180918D139091D4
:10B580008E130C94D34808958091E413882319F006
:10B590000E94278702C00E94118780918F13882301
:10B5A00079F02091D71280918D1390918E132223E0
:10B5B00019F06EE474E102C067E674E10C94D348BC
:10B5C0000895B9C1CF938091E20B882309F47EC01E
:10B5D0000E944E7B9091E00B882341F0911176C040
:10B5E00080913D07882309F45AC070C091116EC044
:10B5F00080918F138823D1F06FE274E180918D13D5
:10B6000090918E130E94AF488091E10B882341F006
:10B6100064E274E180918D1390918E130E94AF4883
:10B6200080918D1390918E130E94B7470E94F77BF3
:10B6300081E08093280780911B13882309F446C07A
:10B640008091E313882349F18091D712882379F000
:10B6500029E432EA42E350E060E070E08DE69CE0ED
:10B660000E945C3F9093440F8093430F2FC08091C2
:10B670000702813059F54091D9125091DA1214160F
:10B6800015065CF4052E000C660B770B2FE83BE5E6
:10B690008DE69CE0CF910C94543FCF9140C082E066
:10B6A00080933D0780918F13882341F06BE374E111
:10B6B00080918D1390918E130E94D348C1E0C09366
:10B6C000871339D10E94F77BC0932807CF91089543
:10B6D00081E05FC18091881381112DC181E059C142
:10B6E0000C94DE6A53C28091911381110C94DE6A2E
:10B6F0004DC28091AA079091AB07DC01ED91FC91BE
:10B700000084F185E02D19958091AA079091AB07EF
:10B71000DC01ED91FC910480F581E02D199480917C
:10B720000702813019F485E0809307020895109292
:10B73000A607089580911307882371F010921307CC
:10B7400080918F13882341F067EC77E180918D130E
:10B7500090918E130C94D348089580910E138330EA
:10B7600099F08091130781110FC081E08093130736
:10B7700080918F13882341F062EB77E180918D13E4
:10B7800090918E130C94D3480895809113078823C9
:10B7900019F080E090E0CECF80E090E0DECF8091A5
:10B7A0001207833079F083E08093120780918F1322
:10B7B000882341F061EA77E180918D1390918E1397
:10B7C0000C94D348089580911207823079F082E07A
:10B7D0008093120780918F13882341F060E977E10D
:10B7E00080918D1390918E130C94D348089580917D
:10B7F0001207813079F081E08093120780918F13D6
:10B80000882341F06FE777E180918D1390918E133B
:10B810000C94D348089580919113882371F00E946D
:10B82000DE6A80918F13882341F06FE377E1809186
:10B830008D1390918E130C94D348089580910E131C
:10B84000833059F02CF48130E9F08230D9F030C0E7
:10B85000863044F08630B1F02BC08091A0079091E3
:10B86000A1071FC08091A0079091A107DC01ED9175
:10B87000FC910480F581E02D199580919E079091AF
:10B880009F070FC08091A4079091A507DC01ED915F
:10B89000FC910480F581E02D19958091A20790918B
:10B8A000A307DC01ED91FC910480F581E02D199551
:10B8B0008091AA079091AB07DC01ED91FC91E25BCE
:10B8C000FF4F0190F081E02D19958091AA0790918A
:10B8D000AB07DC01ED91FC910484F585E02D60E07F
:10B8E00070E01994ABDF0E947986809191138111E9
:10B8F0000E94DE6A8091AC079091AD07DC01ED916A
:10B90000FC910480F581E02D19958091A807909114
:10B91000A907DC01ED91FC910480F581E02D1995DA
:10B920008091E612882331F08091290790912A07AF
:10B930000C94123D089580919113882339F18091E0
:10B940008813882319F1109288130E9433978091ED
:10B950008713882319F0109287130CC08091AA07CF
:10B960009091AB07DC01ED91FC910288F389E02D09
:10B9700060E0199580918F13882341F068E677E1A4
:10B9800080918D1390918E130E94D348109288134A
:10B990000895CF93909191139923D1F19091E00B59
:10B9A000911136C090918813911132C0C82F81E057
:10B9B000809388138091770F882331F081E00E9473
:10B9C00082971092770F02C00E944297809187134E
:10B9D000882319F0109287130CC08091AA079091C8
:10B9E000AB07DC01ED91FC910288F389E02D61E069
:10B9F000199580918F13882359F0CC2349F064E581
:10BA000077E180918D1390918E13CF910C94D34850
:10BA1000CF91089581E0BDCFCF93DF93C091750F93
:10BA2000D091760FBE018DE69CE00E94ED3E88230A
:10BA300029F0BE018DE69CE00E94053F1092760F32
:10BA40001092750FDF91CF910895CF92DF92EF9210
:10BA5000FF920F931F93CF93DF93C0901313D09057
:10BA60001413E0901513F09016131C141D041E04FB
:10BA70001F040CF040C080919113882399F100912C
:10BA8000750F1091760FB8018DE69CE00E94ED3E97
:10BA90008823D9F0EBE6FEE0C0E0D0E081919191FF
:10BAA0008017910769F40E94B384CC0FDD1FCC0F7F
:10BAB000DD1FC359D34F688379838A839B831BC05F
:10BAC0002196CE31D10551F716C02BE03CE5B701E8
:10BAD000A6018DE69CE00E94543F9093760F8093E0
:10BAE000750F09C0DF91CF911F910F91FF90EF90DB
:10BAF000DF90CF9091CFDF91CF911F910F91FF9069
:10BB0000EF90DF90CF9008950F931F9380910C02D8
:10BB100081111EC00E94B3840091710F1091720FA9
:10BB20002091730F3091740FAB01BC01401B510B7E
:10BB3000620B730B8091071390910813A0E0B0E0A3
:10BB4000481759076A077B0718F081E080930C02B9
:10BB50001F910F9108958091071390910813892BDD
:10BB600089F080910C02882381F00E94B384609355
:10BB7000710F7093720F8093730F9093740F1092E4
:10BB80000C02089581E080930C020895CF92DF9219
:10BB9000EF92FF92CF93DF938091E00B81117AC1F6
:10BBA0008091A707823040F080918F13882309F499
:10BBB00071C16DEF76E191C08091EF12882309F495
:10BBC00098C08091F407882309F493C08091901362
:10BBD00081118FC08091F712882359F18091A111B2
:10BBE0009091A211A091A311B091A411892B8A2B3D
:10BBF0008B2BF9F00E94B384C090A111D090A211B8
:10BC0000E090A311F090A4119B01AC012C193D0907
:10BC10004E095F0969017A012091F71230E0A8EE20
:10BC2000B3E00E9402C3C616D706E806F90608F478
:10BC300060C0C0912907D0912A0789AD9AAD892BA0
:10BC400011F01AAE19AE8BA9813009F06FC08FEFD9
:10BC500090E090932D0180932C019F8F8E8F0E94F6
:10BC6000B3846DAB7EAB8FAB98AF8091AA079091F8
:10BC7000AB07DC01ED91FC910284F385E02D199571
:10BC800081E0809390132091F40730E0A8EEB3E0B8
:10BC90000E9402C3AB01BC0126EC3DE58DE69CE0B1
:10BCA0000E94543F90938C1380938B1380918F1339
:10BCB000882309F4EFC06BEC76E180918D139091AD
:10BCC0008E130E94AF486091F40780918D1390917C
:10BCD0008E130E94D76A62EC76E180918D13909169
:10BCE0008E13DF91CF91FF90EF90DF90CF900C9467
:10BCF000D3480ADF80910C02882309F4CBC08091DD
:10BD000091138111C7C081E08093911380930C023D
:10BD100022DF80918F138823A1F068E776E180917C
:10BD20008D1390918E130E94D3480BC0823009F07E
:10BD300096CF4FEF60E0CE010E94C23C8FEF90E0C3
:10BD40008CCF80919013811136C08091EF1288239F
:10BD500091F18091F407882371F18091F712882383
:10BD600051F18091A1119091A211A091A311B091D4
:10BD7000A411892B8A2B8B2BF1F00E94B384C090E5
:10BD8000A111D090A211E090A311F090A4119B01F9
:10BD9000AC012C193D094E095F0969017A01209116
:10BDA000F71230E0A8EEB3E00E9402C3C616D70631
:10BDB000E806F906D8F110929013809189139091BA
:10BDC0008A13806190938A13809389138091AA07C4
:10BDD0009091AB07DC01ED91FC910280F381E02DA5
:10BDE00019958091A70781111AC0409109135091AC
:10BDF0000A1381E0809387134115510561F060E0DB
:10BE000070E02AE03DE58DE69CE00E94543F80E032
:10BE10000E94829704C08093770F80E0BADDDF91A3
:10BE2000CF91FF90EF90DF90CF900FCE6DEA76E14B
:10BE300080918D1390918E130E94AF480E94B3841D
:10BE4000C090A111D090A211E090A311F090A41184
:10BE50006C197D098E099F0928EE33E040E050E01F
:10BE60000E94E0C2BA01A90121E080918D13909156
:10BE70008E130E946F4767E876E180918D13909151
:10BE80008E130E94AF4880918D1390918E130E9463
:10BE9000B74791CFDF91CF91FF90EF90DF90CF9098
:10BEA0000895AF92BF92CF92DF92EF92FF920F93DD
:10BEB0001F93CF93DF939091690F91110BC0209145
:10BEC000B3073091B4073093680F2093670F91E068
:10BED0009093690F90915F0F91110BC02091B10762
:10BEE0003091B20730935E0F20935D0F91E09093F5
:10BEF0005F0FA090670FB090680F00915D0F1091D9
:10BF00005E0FD0918F13843608F047C0C82F682F7A
:10BF100070E080E090E00E946FC120E030E048ECEB
:10BF200052E40E9476C36B017C01B501BB0C880B07
:10BF3000990B0E9471C19B01AC01C701B6010E941F
:10BF4000D0C10E94DEC37093B4076093B307B801F9
:10BF5000110F880B990B0E9471C19B01AC01C701A5
:10BF6000B6010E94D0C10E94DEC37093B2076093F5
:10BF7000B107DD2371F167E576E180918D13909132
:10BF80008E130E94AF486C2F80918D1390918E1369
:10BF90000E94D76A65E576E10CC0B092B407A09222
:10BFA000B3071093B2070093B107DD2391F069E660
:10BFB00076E180918D1390918E13DF91CF911F9137
:10BFC0000F91FF90EF90DF90CF90BF90AF900C94C7
:10BFD000D348DF91CF911F910F91FF90EF90DF90A9
:10BFE000CF90BF90AF900895CF93823069F4909135
:10BFF00002132091FF1230910313409100135091CE
:10C0000001136091FE120CC09091FC122091F91264
:10C010003091FD124091FA125091FB126091F8128A
:10C0200060939C145093991440939A1430939814ED
:10C0300020939B1490939D14909100028917B9F05E
:10C040008093000290918F13992389F0C82F6CE39D
:10C0500076E180918D1390918E130E94AF486C2FE2
:10C0600080918D1390918E13CF910C94C06ACF91D3
:10C070000895833079F030F4813051F0823091F4BA
:10C080008BE30BC0843041F0853061F482E405C05D
:10C090008CE303C080E401C081E40E94B24A21E045
:10C0A000892B09F420E0822F0895E3DF91E08927AE
:10C0B00008950F931F938091550F81110DC00E9419
:10C0C000B3846093510F7093520F8093530F9093EA
:10C0D000540F81E08093550F80910A028A3AF1F45F
:10C0E00085E0C7DF882371F088E399E09093AB1473
:10C0F0008093AA1490938E1380938D138FEF809367
:10C100000A020CC085ED99E09093AB148093AA14B9
:10C1100090938E1380938D1310920A020E94B38421
:10C120000091510F1091520F2091530F3091540FE5
:10C13000DC01CB01801B910BA20BB30BC397A105B4
:10C14000B10508F449C00E94B3846093510F709305
:10C15000520F8093530F9093540F85E08ADF88230A
:10C1600021F080910A02882349F085E082DF811165
:10C1700033C080910A028F3F79F518C088E399E0B7
:10C180009093AB148093AA1490938E1380938D1385
:10C1900080918F13882331F062E276E188E399E0A1
:10C1A0000E94D3488FEF80930A0216C085ED99E074
:10C1B0009093AB148093AA1490938E1380938D1355
:10C1C00080918F13882331F06DE076E185ED99E061
:10C1D0000E94D34810920A021F910F910895109265
:10C1E000E31380918F13882379F02091D7128091E7
:10C1F0008D1390918E13222319F06DED75E102C01D
:10C2000060EF75E10C94D348089581E08093ED0BC5
:10C21000089581E08093EE0B089581E08093EF0B09
:10C2200008952F923F924F925F926F927F928F92DA
:10C230009F92AF92BF92CF92DF92EF92FF920F93B5
:10C240001F93CF93DF9300D000D0CDB7DEB74DB6AC
:10C250005EB60E9418440E940D440E9454A10297A9
:10C2600009F0EFC20E943DA1882309F4E4C2C09006
:10C27000C014D090C114E090BE14F090BF14B60169
:10C28000C7010E94ED3E8823F1F0F701E250FE4F16
:10C2900000E010E0819191918C159D0571F40E9450
:10C2A000B384000F111F000F111FF701E00FF11FE2
:10C2B000608371838283938308C00F5F1F4F0E31A9
:10C2C000110541F702C00E942AA21092F00BEDB6B0
:10C2D000FEB64091F30B5091F40BCA01880F991FE1
:10C2E000ADB6BEB6A81AB90A0FB6F894BEBE0FBE58
:10C2F000ADBE0DB71EB70F5F1F4F8091F60B82309A
:10C3000069F0833029F1813009F071C0B801809162
:10C31000C9149091CA140E94889E33C03FB7F89404
:10C3200020E0822F90E08417950774F4880F991FFE
:10C33000F801E80FF91FDC01AF53B14F8D919C91CB
:10C34000918380832F5FEDCF3FBF1092E10E19C024
:10C350003FB7F89420E0822F90E08417950774F49B
:10C36000880F991FF801E80FF91FDC01AD56B04F97
:10C370008D919C91918380832F5FEDCF3FBF109271
:10C38000C61420E06AE071E0822F90E04091F30B48
:10C390005091F40B8417950754F5689FF001699F3D
:10C3A000F00D1124ED53F04FA085B1858C918823B9
:10C3B000E1F0A081B1813C91C801830F911D830FF1
:10C3C000911DDC0112978D919C91A281B3814D91B9
:10C3D0005C9111970480F581E02D4817590711F4FD
:10C3E000108203C070838D939C932F5FCDCF0FB6C7
:10C3F000F894FEBE0FBEEDBE8091BD10882321F0E3
:10C400008CEB90E10E9472A18091C710882321F0EB
:10C4100086EC90E10E9472A18091D110882321F0D6
:10C4200080ED90E10E9472A18091DB10882321F0C1
:10C430008AED90E10E9472A18091F10B882309F4AA
:10C4400065C08091D110811105C08091DB108823D7
:10C4500009F450C08091D4109091D510E091D8107B
:10C46000F091D910238134812817390724F480856D
:10C47000811109C00EC0218132818217930734F4E3
:10C480008085811106C088E090E005C080E190E0E1
:10C4900002C080E290E02091DE103091DF10E09148
:10C4A000E210F091E310438154814217530724F4C2
:10C4B0002085222349F00AC0418152812417350783
:10C4C0003CF42085222311F0816003C0846001C008
:10C4D000826020916310309164102817390719F495
:10C4E0001092651007C0909364108093631081E0F0
:10C4F000809365108091631090916410429709F4C5
:10C50000A4C181E08093DD108093D310A9E6B0E14F
:10C510006CE670E188EE682E83E0782E2224239466
:10C52000FD0131978081882309F47CC11496CD9058
:10C53000DC901597DE82CD82F6018781882309F48D
:10C5400071C18C91882309F46DC111964D915C9154
:10C55000129730847301E41AF50A1E141F042CF09C
:10C560007A01F8EEEF1AF3E0FF0A20E030E001E094
:10C5700010E0EFE0F7E290E0832C912CA32CB12C9B
:10C58000C12CD12CA982BA82CB82DC82650182E0E7
:10C59000C81AD108081519050CF04AC08BE0C81656
:10C5A000D104E0F5F6018827E657FE4F8F4F0C9433
:10C5B000D0C4F901E15BF94F27C0F901E75BF94FFE
:10C5C00023C0F901EF5BF94F1FC0F901E95CF94F96
:10C5D0001BC0F901E55DF94F17C0F901E35EF94FA2
:10C5E00013C0F901E35FF94F0FC0F901E550FA4FAD
:10C5F0000BC0F901E951FA4F07C0F901EF52FA4FA8
:10C6000003C0F901E754FA4F0280F381E02DE41BE7
:10C61000F50BF7FF03C0F195E195F109EE15FF0564
:10C6200014F4902F7F010F5F1F4F2E5F3F4FB2CF4B
:10C630009F5FED81FE818185882309F4EAC0032D87
:10C6400010E0F8013297EB30F10508F0E2C08827DE
:10C65000EB56FE4F8F4F0C94D0C4913009F0ACC014
:10C66000C3C0913009F4D4C0933009F0D2C0A4C043
:10C67000913009F4CBC0923009F4CAC0933009F468
:10C68000B3C0943009F0C5C097C0913009F4BCC064
:10C69000923009F4BBC0943009F4A6C0953009F07B
:10C6A000B8C08AC0913009F4ADC0923009F4ACC072
:10C6B000933009F4ABC0943009F4AAC0953009F462
:10C6C00093C0963009F0A5C077C0913009F498C0A6
:10C6D000923009F497C0933009F496C0953009F46C
:10C6E00097C0963009F480C0973009F092C064C0BA
:10C6F000913009F483C0923009F482C0933009F478
:10C7000081C0943009F480C0953009F47FC0963020
:10C7100009F47EC0973009F467C0983009F079C0F9
:10C720004BC0913009F468C0923009F467C093306F
:10C7300009F466C0943009F465C0963009F466C007
:10C74000973009F465C0983009F44EC0993009F06B
:10C7500060C032C0913009F44DC0923009F44CC031
:10C76000933009F44BC0943009F44AC0953009F471
:10C7700049C0963009F448C0973009F447C0983052
:10C7800009F446C0993081F19A3009F042C014C0D2
:10C79000913071F1923071F1933071F1943071F107
:10C7A000953071F1973081F1983081F1993081F1B4
:10C7B0009A30D1F09B3069F591E02BC09130B1F007
:10C7C0009230B1F09330B1F09430B1F09530B1F0D7
:10C7D0009630B1F09730B1F09830B1F09930B1F0B7
:10C7E0009A30B1F09B30A9F492E013C09CE011C0E4
:10C7F0009BE00FC09AE00DC099E00BC098E009C023
:10C8000097E007C096E005C095E003C094E001C042
:10C8100093E0FB018081891302C01C9203C02C921B
:10C82000FB0190831796695F7F4FF0E1AD3BBF0737
:10C8300009F076CE04C00E9424440E942AA281E01E
:10C8400066C00E94244480E062C0E0906610F090D0
:10C8500067101E141F040CF055C08091D210009177
:10C86000BE141091BF146091B20F7091B30F882362
:10C87000B1F081E08093D310C8010E94ED3E811198
:10C8800015C0A701FF0C660B770B24E231EAC80143
:10C890000E94543F9093B30F8093B20F07C0C8011A
:10C8A0000E94ED3E811102C01092D3108091DC10E5
:10C8B0000091BE141091BF146091B00F7091B10F30
:10C8C0008823D1F081E08093DD10C8010E94ED3E05
:10C8D00081111CCE4091661050916710052E000CFE
:10C8E000660B770B21E231EAC8010E94543F909316
:10C8F000B10F8093B00F0ACEC8010E94ED3E8111A6
:10C9000005CE02C01092D3101092DD10FFCD0FB6ED
:10C91000F8945EBE0FBE4DBE26960FB6F894DEBFED
:10C920000FBECDBFDF91CF911F910F91FF90EF9080
:10C93000DF90CF90BF90AF909F908F907F906F903F
:10C940005F904F903F902F900895CF938091AF0FBD
:10C95000C0910B02811101C1C23009F450C0C33033
:10C9600009F49DC0C13009F028C18091EF0B8111FD
:10C9700024C181E090E00E94E4C49093CA148093A3
:10C98000C91462E083E00E94094B1092900F10924C
:10C99000C3141092C2141092C71480E090E0FC01FE
:10C9A000EE0FFF1FE258F04F11821082019688307F
:10C9B0009105A9F710928F0F10928E0F80916A0047
:10C9C0008C6080936A00ED9A8FB7F8942091840070
:10C9D000309185003093790F2093780F8FBF2DE031
:10C9E00031E64AEF50E060E070E08091BE14909133
:10C9F000BF140E94543F81E08093AF0FDEC080914E
:10CA0000EE0B8111DAC081E090E00E94E4C49093C3
:10CA1000BE0E8093BD0E809104018E7F8093040131
:10CA2000809105018160809305018EEF97E09093DE
:10CA3000E80E8093E70E2EE240EA56E861E070E0EF
:10CA40000E944D4A809165008B7F80936500109213
:10CA5000350189E0809334018EE2809332018CEFBE
:10CA60008093300180E9809331011092E60E10929C
:10CA7000E50E1092E40E1092E30E1092E10EE1EC3E
:10CA8000FEE08CED95E0819391932EE0E13EF2077C
:10CA9000D1F7C1E0C093E20E29E031E651C08091A8
:10CAA000ED0B81118AC081E090E00E94E4C4909374
:10CAB000C00E8093BF0E809104018E7F809304018D
:10CAC000809105018160809305018EEF97E090933E
:10CAD000920F8093910F26E040E052EC61E070E00D
:10CAE0000E944D4A809165008B7F80936500109273
:10CAF000350180E18093340186E0809332018EEF2E
:10CB00008093300180E9809331011092C514109216
:10CB1000C41410927D0F10927C0F1092C614E3E99A
:10CB2000FFE08CED95E0819391932FE0EF3AF207CF
:10CB3000D1F710927B0FC1E0C0937A0F25E031E668
:10CB40004AEF50E060E070E08091BE149091BF1415
:10CB50000E94543FC093AF0F30C0C23069F0C33061
:10CB6000D1F0C13051F58091EF0B811126C0809139
:10CB7000C2149091C3141DC08091EE0B81111DC091
:10CB80008091BD0E9091BE0E0E9407438091E50EEC
:10CB90009091E60E0EC08091ED0B81110EC0809138
:10CBA000BF0E9091C00E0E9491998091C4149091F3
:10CBB000C514029711F4C093F60B80910B028230DA
:10CBC000A1F1833009F454C0813009F074C0809120
:10CBD000EF0B882309F46FC0ED98E59A1092900F3F
:10CBE0001092C8141092C3141092C2141092C71459
:10CBF00080E090E0FC01EE0FFF1FE258F04F118241
:10CC00001082019688309105A9F710928F0F10922B
:10CC10008E0F8091C9149091CA140E9479C5109208
:10CC2000AF0F1092EE0B82E044C08091EE0B882390
:10CC300009F441C08091E70E9091E80E0E942B4AC2
:10CC4000809131018F7780933101809131018F7E06
:10CC500080933101109230018091BD0E9091BE0EF3
:10CC60000E9479C51092AF0F1092ED0B83E021C0A6
:10CC70008091ED0B8823F9F08091910F9091920FA4
:10CC80000E942B4A809131018F77809331018091EE
:10CC900031018F7E80933101109230018091BF0E5F
:10CCA0009091C00E0E9479C51092AF0F1092EF0BB9
:10CCB00081E080930B028091BE149091BF14CF91BC
:10CCC0000C94643FAF92BF92CF92DF92EF92FF92AB
:10CCD0000F931F93CF93DF937C016B015A01D0E038
:10CCE000C0E08D2F90E0F701A181B2818A159B05EC
:10CCF000D0F4F601E80FF91F608102E819EA21E09B
:10CD00003327C6270C0F111D211D311D2BBFF80124
:10CD1000C791ED91FC9111970190F081E02DCD012B
:10CD20001995DF5FDECFED91FC9111970190F081B5
:10CD3000E02D6C2FCD01DF91CF911F910F91FF90CE
:10CD4000EF90DF90CF90BF90AF901994CF93DF9387
:10CD500000D01F921F92CDB7DEB7FE01319625E0BD
:10CD6000DF011D922A95E9F724E8298325E52C8324
:10CD70002AE22D836A834B8345E050E0BF01A2DFA6
:10CD800065E070E080E090E00E94504C80E00F9001
:10CD90000F900F900F900F90DF91CF910895EF9229
:10CDA000FF921F93CF93DF931F92CDB7DEB77C0125
:10CDB000162FFC0161817281F9D465E070E080E09A
:10CDC00090E00E94504C42E462E4C701BFDF412F73
:10CDD00060E0C701BBDF811163C040E061E0C701D3
:10CDE000B5DF81115DC040E062E0C701AFDF8111B6
:10CDF00057C046E062E0C701A9DF811151C040E0A1
:10CE000063E0C701A3DF81114BC040E064E0C701CC
:10CE10009DDF11E0811110E040E065E0C70196DF81
:10CE2000811101C01F5F40E066E0C7018FDF811103
:10CE300001C01F5F40E067E0C70188DF811101C0CA
:10CE40001F5F40E068E0C70181DF811101C01F5F03
:10CE500040E069E0C7017ADF811101C01F5F44E053
:10CE60006AE0C70173DF811101C01F5F44E06AE01F
:10CE7000C7016CDF811101C01F5F62E370E080E0D9
:10CE800090E00E94504C82E8898341E050E0BE016E
:10CE90006F5F7F4FC70116DF81E0183011F011116D
:10CEA00080E00F90DF91CF911F91FF90EF90089558
:10CEB000CF93DF93EC010E94B384688379838A83E4
:10CEC0009B83CE01DF91CF910895EF92FF921F9344
:10CED000CF93DF93CDB7DEB765970FB6F894DEBF7B
:10CEE0000FBECDBF182F7B018CEE9AE00E941393EA
:10CEF00081E080931A0B84E690E09093FD0A809382
:10CF0000FC0A84E6E816F10418F484E6E82EF12C15
:10CF1000C70164E670E00E94A9C470931C0B609383
:10CF20001B0B7093FF0A6093FE0A1093F90A8FEFB0
:10CF3000810F823010F41230D1F08CEE9AE00E9412
:10CF400025938091F70A882329F083EC95EFA8ECCC
:10CF5000BFE304C084EB98ECA6E9B0E48093160B21
:10CF60009093170BA093180BB093190B55C0809199
:10CF7000F70A882329F084EB98ECA6E9B0E404C012
:10CF800083EC95EFA8ECBFE38093160B9093170BFF
:10CF9000A093180BB093190B8CEE9AE00E942F937C
:10CFA00080911A0B8823C1F11092F90A8EE690E065
:10CFB0009A83898388E290E09C838B838CE390E062
:10CFC0009E838D831D8A83E08F938DB79EB745978F
:10CFD0000FB6F8949EBF0FBE8DBFADB7BEB711960A
:10CFE00085E1FE01319601900D928A95E1F78CEE74
:10CFF0009AE00E9439930FB6F894DEBF0FBECDBF02
:10D0000065960FB6F894DEBF0FBECDBFDF91CF910E
:10D010001F91FF90EF9008958CEE9AE065960FB601
:10D02000F894DEBF0FBECDBFDF91CF911F91FF906F
:10D03000EF903ECF0F931F93CF93DF93EC01AB01A3
:10D0400060E070E02AE00E946F478C01CE010E94F0
:10D05000B747800F911FDF91CF911F910F910895D6
:10D060008F929F92AF92BF92CF92DF92EF92FF92F8
:10D070000F931F93CF93DF931F921F92CDB7DEB70D
:10D08000082E000C990BAA0BBB0BFC013197EF305B
:10D09000F10508F066C28827E056FE4F8F4F0C94CA
:10D0A000D0C484E08093DB0A82E38093DC0A86E2CA
:10D0B0008093DE0A81E08093E10A8093E20A809304
:10D0C000E00A49E458E120E030E08091DB0A90E09A
:10D0D000281739070CF08CC1FA0185919491A0E0D2
:10D0E000B0E0880F991FAA1FBB1FF901EE0FFF1FA9
:10D0F000EE0FFF1FEE58F54F80839183A283B38319
:10D100002F5F3F4F4E5F5F4FE0CF84E08093DB0A9D
:10D1100082E38093DC0A86E28093DE0A81E08093DA
:10D12000E10A8093E20A82E08093E00A41E458E158
:10D1300020E030E08091DB0A90E0281739070CF0FE
:10D1400057C1FA0185919491A0E0B0E0880F991F32
:10D15000AA1FBB1FF901EE0FFF1FEE0FFF1FEE58B6
:10D16000F54F80839183A283B3832F5F3F4F4E5F40
:10D170005F4FE0CF84E08093DC0A85E28093DE0A93
:10D1800081E08093E10A88E08093E20A83E0809363
:10D19000E00A80E090E0FC01E75CF74EE491DC01FE
:10D1A000AD51B54FEC93019688309105A1F70E94DF
:10D1B00038501EC188E08093DB0A86E08093DC0A49
:10D1C00086E28093DE0A81E08093E10A8093E20A9E
:10D1D00084E08093E00A49E258E120E030E0809169
:10D1E000DB0A90E0281739070CF002C1FA0185919B
:10D1F0009491A0E0B0E0880F991FAA1FBB1FF9010E
:10D20000EE0FFF1FEE0FFF1FEE58F54F8083918347
:10D21000A283B3832F5F3F4F4E5F5F4FE0CF88E025
:10D220008093DB0A81E08093DC0A97E29093DE0A28
:10D230008093E10A8093E20A85E08093E00A49E165
:10D2400058E120E030E08091DB0A90E028173907B0
:10D250000CF0CEC0FA0185919491A0E0B0E0880F67
:10D26000991FAA1FBB1FF901EE0FFF1FEE0FFF1F33
:10D27000EE58F54F80839183A283B3832F5F3F4F96
:10D280004E5F5F4FE0CF82E18093DB0A81E08093C5
:10D29000DC0A97E29093DE0A8093E10A8093E20A27
:10D2A0008FE08093E00A45EF57E120E030E0809185
:10D2B000DB0A90E0281739070CF09AC0FA01859133
:10D2C0009491A0E0B0E0880F991FAA1FBB1FF9013D
:10D2D000EE0FFF1FEE0FFF1FEE58F54F8083918377
:10D2E000A283B3832F5F3F4F4E5F5F4FE0CFE0914C
:10D2F000460BF091470B74978081918140E550E097
:10D3000060E070E08A5B944F0E948D512AC182E1F7
:10D310008093DB0A85E08093DC0A82E28093DE0A58
:10D3200081E08093E10A8093E20A87E08093E00A3B
:10D3300080E993E3A0E0B0E08093720A9093730ACF
:10D34000A093740AB093750AF2E08F2E912C01E03D
:10D3500010E080E090E0A0E0BBE54CE454E060E049
:10D3600070E024EEC22E2CE0D22EE12CF12C98019C
:10D37000220F331F220F331F5401AA0CBB1CAA0C0F
:10D38000BB1C2E58354FF901B7FF0DC0C082D182AA
:10D39000E282F38295012E58354FF9014083518383
:10D3A000628373830CC040835183628373839501CE
:10D3B0002E58354FF901C082D182E282F382880F64
:10D3C000991FAA1FBB1F0E5F1F4FF2E08F0E911C0B
:10D3D00022E18216910459F688E79FEFA0E0B0E0C1
:10D3E0008093B60A9093B70AA093B80AB093B90A8B
:10D3F0000E94A750B6C0CE0101960E94265023E09D
:10D4000040E150E060E070E072C084E08093DB0AAD
:10D4100082E38093DC0A86E28093DE0A81E08093D7
:10D42000E10A8093E20A8AE08093E00A4DEE57E138
:10D4300020E030E08091DB0A90E028173907C4F63D
:10D44000FA0185919491A0E0B0E0880F991FAA1F7E
:10D45000BB1FF901EE0FFF1FEE0FFF1FEE58F54F38
:10D4600080839183A283B3832F5F3F4F4E5F5F4FD3
:10D47000E1CF84E08093DB0A80E28093DC0A86E2DD
:10D480008093DE0A81E08093E10A8093E20A8BE0D8
:10D490008093E00A45EE57E120E030E08091DB0A1E
:10D4A00090E0281739070CF0A3CFFA0185919491E9
:10D4B000A0E0B0E0880F991FAA1FBB1FF901EE0F73
:10D4C000FF1FEE0FFF1FEE58F54F80839183A2835D
:10D4D000B3832F5F3F4F4E5F5F4FE0CFCE0101968A
:10D4E0000E94265021E040E154E060E070E0CE016F
:10D4F00001960E94015135C084E08093DB0A83E0ED
:10D500008093DC0A86E28093DE0A81E08093E10A60
:10D510008093E20A8DE08093E00A4DED57E120E030
:10D5200030E08091DB0A90E0281739070CF060CFDB
:10D53000FA0185919491A0E0B0E0880F991FAA1F8D
:10D54000BB1FF901EE0FFF1FEE0FFF1FEE58F54F47
:10D5500080839183A283B3832F5F3F4F4E5F5F4FE2
:10D56000E0CF0F900F90DF91CF911F910F91FF901F
:10D57000EF90DF90CF90BF90AF909F908F900895E5
:10D580000F931F93CF93DF93EC01462F50E060E0A1
:10D5900070E02AE00E946F478C01CE010E94B747DD
:10D5A000800F911FDF91CF911F910F910895462F0A
:10D5B00050E060E070E02AE00C946F478091E00B4F
:10D5C000811180C00E94845D80910C02882321F02B
:10D5D00080919113811105C080919013882309F4E3
:10D5E00071C01092911381E080930C020E94AB5D98
:10D5F00080918F138823D1F06AE976E080918D13B2
:10D6000090918E130E94AE4880919013882341F030
:10D610006AEA76E080918D1390918E130E94AE4855
:10D6200080918D1390918E130E94B7478091901333
:10D63000882369F060918B1370918C13161617066E
:10D6400024F48DE69CE00E94053F10929013809197
:10D65000891390918A13806290938A13809389131F
:10D6600080918813882311F081E001C080E00E943E
:10D67000519781E0809387130E949B5C80912413D3
:10D6800081110FC08091A511882359F029E73BE54E
:10D6900044E650E060E070E08DE69CE00E94543F7C
:10D6A00002C00E94795B0E941E5C0E94255D0E9460
:10D6B000B3846093A1117093A2118093A3119093EE
:10D6C000A411089508952FB7F894882381F08091CC
:10D6D00026119091271190933511809334118091E8
:10D6E00036119091371118161906ACF00FC08091C1
:10D6F00028119091291190933511809334118091C4
:10D70000361190913711181619062CF480913611A4
:10D710009091371107C080913611909137119195F2
:10D720008195910990933711809336112FBF0895F9
:10D73000AF92BF92CF92DF92EF92FF920F931F931F
:10D74000CF93DF931F921F92CDB7DEB78C017A8300
:10D750006983CE0101966C01580192E0A90EB11CBB
:10D76000E12CF12CC8010E9494C2F60161916F0175
:10D77000861731F0C8010E94A6C2FFEFEF1AFF0A18
:10D780000F5F1F4F0A151B0569F781E0EF2809F4A9
:10D7900080E00F900F90DF91CF911F910F91FF903C
:10D7A000EF90DF90CF90BF90AF900895EF92FF92EF
:10D7B0000F931F93CF93DF931F921F92CDB7DEB7C6
:10D7C0008C017B018AEA8A8341E050E0BE016E5FF2
:10D7D0007F4FC80177DAD701ED91FC910680F78180
:10D7E000E02DC701199582E8898341E050E0BE0130
:10D7F0006F5F7F4FC80166DA0F900F90DF91CF9176
:10D800001F910F91FF90EF900895CF92DF92EF92CA
:10D81000FF920F931F930E94B3846B017C0160936E
:10D820009313709394138093951390939613809110
:10D83000F70B0E94B24A809392139091F90B9923AF
:10D8400029F091E0811190E0909392138091010C66
:10D850009091020CA091030CB091040C97018601E9
:10D86000081B190B2A0B3B0B4091050C5091060C21
:10D870006091070C7091080C9091FA0B0417150732
:10D880002607370760F4C092FD0BD092FE0BE092A2
:10D89000FF0BF092000C1092FC0B892F1EC090938E
:10D8A000FB0B809192138093FA0BC092FD0BD092E8
:10D8B000FE0BE092FF0BF092000C891761F0C09212
:10D8C000010CD092020CE092030CF092040C91E057
:10D8D0009093FC0B02C01092FC0B1F910F91FF90D4
:10D8E000EF90DF90CF9008950F931F93CF93DF9326
:10D8F000EC012AE00E946F478C01CE010E94B747DD
:10D90000800F911FDF91CF911F910F910895CF92BA
:10D91000DF92EF92FF920F931F93CF93DF936B01F0
:10D92000770FEE08FF08F7FE1BC0EC016DE20E94C6
:10D93000CA478C0144275527BA014C195D096E0965
:10D940007F092AE0CE010E946F47800F911FDF916F
:10D95000CF911F910F91FF90EF90DF90CF9008959E
:10D960002AE0B701A601DF91CF911F910F91FF909F
:10D97000EF90DF90CF900C946F47CF92DF92EF92B1
:10D98000FF920F931F93CF93DF938C016B01770F5F
:10D99000EE08FF08F7FE12C06DE20E94CA47EC01D4
:10D9A00044275527BA014C195D096E097F092AE001
:10D9B000C8010E946F47C80FD91F06C02AE0B701EF
:10D9C000A6010E946F47EC01C8010E94B7478C0F67
:10D9D0009D1FDF91CF911F910F91FF90EF90DF90EE
:10D9E000CF9008950F931F93CF93DF931F92CDB7DE
:10D9F000DEB78C0169830E9494C26981861729F081
:10DA0000C8010E94A6C281E001C080E00F90DF91B2
:10DA1000CF911F910F910895CF930E9427A184E089
:10DA200090E09093F40B8093F30B1092BC10109243
:10DA3000C6101092D0101092DA10E8E6F0E1DF0183
:10DA40001C92179680E1AC3BB807D1F787EA91E1C9
:10DA50009093C5108093C4101092BF108091F20B68
:10DA60009091A711891718F091E09093BC1020EBCA
:10DA700031E13093CF102093CE101092C9109091C5
:10DA8000B011891718F091E09093C61029EB31E19D
:10DA90003093D9102093D8101092D3109091B911CF
:10DAA000891718F091E09093D01022EC31E1309377
:10DAB000E3102093E2101092DD109091C2118917AB
:10DAC00018F091E09093DA101092F10B20E030E022
:10DAD000D901A55BBD4E4D915C9141505109443235
:10DAE000510520F491E09093F10B05C02D5F3F4F5D
:10DAF0002837310569F79091F10B992341F1209175
:10DB0000BA113091BB112D5D3F4F3093BB11209363
:10DB1000BA112091BC113091BD11235231093093BB
:10DB2000BD112093BC112091C3113091C4112D5D02
:10DB30003F4F3093C4112093C3112091C5113091F0
:10DB4000C611235231093093C6112093C51190910B
:10DB5000C4129F3049F49091C5129F3029F410925D
:10DB600067101092661008C0209122133091231381
:10DB7000309367102093661022E130E030936410F8
:10DB8000209363102091F30B3091F40BABECB1E1D7
:10DB900041E0B683A5839C91992329F0891718F059
:10DBA00040832F5F3F4F1A96379690E1EC3BF90781
:10DBB00081F73093F40B2093F30B2131310534F0CE
:10DBC00080E190E09093F40B8093F30B0E94244447
:10DBD00080EC90E19093C60F8093C50F8091C410A4
:10DBE0009091C5109093C40F8093C30F8DEB90E17B
:10DBF0009093C80F8093C70F8EEB90E19093CA0F5C
:10DC00008093C90F8CEB90E19093CC0F8093CB0F56
:10DC10008AEC90E19093D00F8093CF0F8091CE103B
:10DC20009091CF109093CE0F8093CD0F87EC90E121
:10DC30009093D20F8093D10F88EC90E19093D40F02
:10DC40008093D30F86EC90E19093D60F8093D50FFD
:10DC500084ED90E19093DA0F8093D90F8091D810E2
:10DC60009091D9109093D80F8093D70F81ED90E1C8
:10DC70009093DC0F8093DB0F82ED90E19093DE0FA9
:10DC80008093DD0F80ED90E19093E00F8093DF0FA4
:10DC90008EED90E19093E40F8093E30F8091E2107A
:10DCA0009091E3109093E20F8093E10F8BED90E160
:10DCB0009093E60F8093E50F8CED90E19093E80F41
:10DCC0008093E70F8AED90E19093EA0F8093E90F3C
:10DCD0002091F30B3091F40B2450310960E07AE08D
:10DCE000C7E0462F50E04217530724F5CA010496B7
:10DCF000789FF001799FF00D1124ED53F04FC49FF0
:10DD0000C001C59F900D1124AC0146595F4E53834D
:10DD10004283DC01A859BF4E15964D915C91169730
:10DD20005183408387599F4E95838483B187A08711
:10DD30006F5FD7CF81E08093F50BCF9108950F935C
:10DD40001F93CF93DF93FC01248135812115310589
:10DD500019F4FB01108211C0EA0121972C173D072D
:10DD600008F4E9018B01FC0160817181AE01C801F9
:10DD70000E9414C7C00FD11F1882DF91CF911F914D
:10DD80000F9108954115510521F06115710509F0B4
:10DD9000D6CF0895EF92FF920F931F93CF93DF9307
:10DDA0001F921F92CDB7DEB78C018CE789831A8250
:10DDB000F801E480F580FFEFEF1AFF0AB701C80110
:10DDC0000E943A46882381F0F801208131818481C4
:10DDD0009581BE016F5F7F4F820F931F0E940DC719
:10DDE000F801F582E48281E00F900F90DF91CF91EE
:10DDF0001F910F91FF90EF900895AF92BF92CF9235
:10DE0000DF92EF92FF920F931F93CF93DF9300D097
:10DE10001F92CDB7DEB78C0149835A836B837C8315
:10DE2000CE0101966C01580194E0A90EB11CE12CC1
:10DE3000F12CC8010E9494C2F60161916F0186170E
:10DE400031F0C8010E94A6C2FFEFEF1AFF0A0F5F70
:10DE50001F4F0A151B0569F781E0EF2809F480E0E0
:10DE60000F900F900F900F90DF91CF911F910F9116
:10DE7000FF90EF90DF90CF90BF90AF900895CF923A
:10DE8000DF92EF92FF920F931F93CF93DF93EC01FA
:10DE90000091B40FE0E0F0E020E030E0A90110E0F4
:10DEA000CE17DF071CF1309711F40D32E1F0DF01DE
:10DEB000AC54B04FFC9080ED8F0D8A30A8F4AAE0EE
:10DEC000B0E00E94D0C22F2DFF0C330B205331093C
:10DED0006901330FEE08FF089B01AC012C0D3D1DBD
:10DEE0004E1D5F1D01C011E03196DACFCA01B901A4
:10DEF000112339F090958095709561957F4F8F4FE4
:10DF00009F4FDF91CF911F910F91FF90EF90DF9086
:10DF1000CF9008958091FA0B811105C081E0909116
:10DF2000FC0B911101C080E0089560E089E30E943C
:10DF3000DA4A60E08AE30E94DA4A60E085E30E9400
:10DF4000DA4A60E085E00E94DA4A60E084E00E94FC
:10DF5000DA4A60E087E00E94DA4A59980895CF9340
:10DF6000C09111026C2F89E30E94DA4A81E0C82730
:10DF70006C2F8AE30E94DA4AC0931102CF91089570
:10DF8000CF93DF93C09110026C2F89E30E94DA4A8D
:10DF9000D1E0DC276D2F8AE30E94DA4A6C2F85E3FB
:10DFA0000E94DA4A6D2F85E00E94DA4A6D2F84E0E4
:10DFB0000E94DA4A6C2F87E00E94DA4ACC2311F0E3
:10DFC000599801C0599A9091100281E08927809355
:10DFD0001002DF91CF910895CF93DF938091AC131E
:10DFE00081110DC01092AB131092AA1381E090E042
:10DFF0009093A9138093A8138093AC1336C080919B
:10E00000AA139091AB13863191057CF18F3891055D
:10E0100034F48091A8139091A913019609C08D350D
:10E0200021E0920754F48091A8139091A9130296CD
:10E030009093A9138093A81318C0863222E0920708
:10E0400034F48091A8139091A9130496F1CF883EDF
:10E0500093403CF48091A8139091A9138A5B9F4F41
:10E06000E7CF1092A9131092A8138ADFC091AA13C8
:10E07000D091AB13C93E83E0D80754F01092AC1393
:10E0800054DF24E630E748EE53E060E070E007C07C
:10E090002CEE3FE6AE010D2E000C660B770B8DE6E5
:10E0A0009CE00E94543F9093A7138093A613809105
:10E0B000A8139091A9138C0F9D1F9093AB1380937D
:10E0C000AA13DF91CF910895CF93DF938091B0078A
:10E0D000882319F0DF91CF917FCFC091A613D09103
:10E0E000A713BE018DE69CE00E94ED3E882329F037
:10E0F000BE018DE69CE00E94053FDF91CF9115CFD8
:10E10000CF93C091A3136C2F70E088E00E94454B21
:10E1100089E18093A21390910F02992311F0CD5FB2
:10E1200001C0C350C093A3138091A313873970F02B
:10E13000992321F08FEF8093A31308C08D3D30F019
:10E1400086E98093A31388E78093A2138091A31399
:10E150008F3F19F410920F0205C08A3118F481E044
:10E1600080930F024091A21350E060E070E020E83D
:10E1700030E78DE69CE00E94543F909370148093AA
:10E180006F14CF910895CF92DF92EF92FF92CF93C9
:10E19000DF93EC019C01AFEFB0E00E9402C3CC24FE
:10E1A000CA9423E0D22EE12CF12CA70196010E9403
:10E1B000B4C2B90188E00E94454B9E01A4E6B0E0DC
:10E1C0000E9402C3A70196010E94B4C280917A13F3
:10E1D000821320937A13DF91CF91FF90EF90DF901D
:10E1E000CF900895CF93DF93C0916F14D0917014A6
:10E1F000BE018DE69CE00E94ED3E882329F0BE0121
:10E200008DE69CE00E94053F60E088E00E94DA4ACB
:10E2100080918F138823D1F080917114882319F095
:10E2200065E879E10DC080916E14882319F06CE6E1
:10E2300079E106C08091AD13811108C06DE579E1E7
:10E2400080918D1390918E130E94D3481092711477
:10E2500010926E14DF91CF91089561E088E00E94E2
:10E26000DA4A80918F13882361F0809171148111B3
:10E2700008C06FE479E180918D1390918E130C9416
:10E28000D348089580917114811110C0ABDF81E0F3
:10E290008093711480918F13882341F064EB79E1AE
:10E2A00080918D1390918E130E94D3488091A11379
:10E2B000882329F060E088E00E94DA4A01C0CDDFBF
:10E2C0009091A11381E089278093A113882329F0DD
:10E2D000409176135091771304C040917813509178
:10E2E000791360E070E022E431E78DE69CE00E9463
:10E2F000543F9093701480936F140895CF9380913E
:10E300009F1381110FC081E080939F1380918F1321
:10E31000882341F06DE179E180918D1390918E1306
:10E320000E94D348C0919E136C2F85E00E94DA4A68
:10E3300040917F1350E060E070E02EE731E78DE61A
:10E340009CE00E94543F90939D1380939C1381E026
:10E350006C2F682760939E13CF91089580910701D9
:10E3600080FF1BC080918F13882351F08BE39CE0CA
:10E370000E94E494811108C08091470C811104C06F
:10E380008BE39CE00C94D19464E978E180918D1347
:10E3900090918E130E94D348F3CF08958091070186
:10E3A00081FF1BC080918F13882351F08AE09CE08D
:10E3B0000E94E494811108C08091160C811104C060
:10E3C0008AE09CE00C94D19467E678E180918D130B
:10E3D00090918E130E94D348F3CF08958091070146
:10E3E00080FF17C080918F13882331F08BE39CE06E
:10E3F0000E94E494882321F08BE39CE00C94F89431
:10E400006EE778E180918D1390918E130E94D3482E
:10E41000F3CF08958091070181FF17C080918F137A
:10E42000882331F08AE09CE00E94E494882321F064
:10E430008AE09CE00C94F89461E578E180918D137A
:10E4400090918E130E94D348F3CF08956091A41346
:10E450007091A5138DE69CE00E94ED3E81112EC0C7
:10E4600060E089E30E94DA4A60E08AE30E94DA4AC7
:10E4700060E085E30E94DA4A60E085E00E94DA4AC3
:10E4800060E084E00E94DA4A60E087E00E94DA4AB5
:10E49000599880917C13882319F020EC3FE602C044
:10E4A0002FEA3FE642E350E060E070E08DE69CE05A
:10E4B0000E945C3F9093A5138093A413089560E09D
:10E4C0008AE30C94DA4A61E08AE30C94DA4A0F9307
:10E4D0001F93CF93DF938C01C1E0D0E00C171D0791
:10E4E0009CF0F1DF64E670E080E090E00E94504C28
:10E4F000E6DFC017D10734F46AE570E080E090E011
:10E500000E94504C2196EACFDF91CF911F910F913D
:10E51000089583E090E0DBCF82E090E0D8CF81E007
:10E5200090E0D5CF60E089E30C94DA4A61E089E3BA
:10E530000C94DA4A0F931F93CF93DF938C01C1E0C1
:10E54000D0E00C171D079CF0F1DF64E670E080E07E
:10E5500090E00E94504CE6DFC017D10734F46AE522
:10E5600070E080E090E00E94504C2196EACFDF916D
:10E57000CF911F910F91089583E090E0DBCF82E06F
:10E5800090E0D8CF81E090E0D5CF60917A1370E031
:10E5900088E00E94454B80918F13882341F06EE9FB
:10E5A00079E180918D1390918E130C94D348089546
:10E5B0001092A01380919D07811104C060E084E057
:10E5C0000E94DA4A80918F13882341F06CE379E14D
:10E5D00080918D1390918E130C94D348089581E00F
:10E5E0008093A01380919D07811106C060919713BD
:10E5F00070E084E00E94454B80918F13882341F0A6
:10E600006AE279E180918D1390918E130C94D34836
:10E610000895CF93DF93C091A413D091A513BE01A9
:10E620008DE69CE00E94ED3E882351F0BE018DE610
:10E630009CE00E94053F1092A5131092A41375DC74
:10E6400080917113882319F0DF91CF91C8CFDF91AA
:10E65000CF91089510929D078091A013811104C05D
:10E6600060E084E00C94DA4A6091971370E084E0F3
:10E670000C94454BCF93DF9360E085E00E94DA4A2B
:10E6800080919F1381110BC08091AA079091AB07D5
:10E69000DC01ED91FC9104ACF5ADE02D1995C09134
:10E6A0009C13D0919D13BE018DE69CE00E94ED3E2F
:10E6B000882329F0BE018DE69CE00E94053F8091F1
:10E6C0008F13882379F020919F1380918D1390915F
:10E6D0008E13222319F061E179E102C065E079E14E
:10E6E0000E94D34810929F13DF91CF91089561E06B
:10E6F00085E00E94DA4A8091AA079091AB07DC017D
:10E70000ED91FC9104ACF5ADE02D199580918F133E
:10E71000882341F06AEF78E180918D1390918E13F8
:10E720000C94D348089560E085E30E94DA4A809112
:10E73000AA079091AB07DC01ED91FC9100ACF1AD23
:10E74000E02D199580918F13882341F06EEE78E1CA
:10E7500080918D1390918E130C94D348089561E0AD
:10E7600085E30E94DA4A8091AA079091AB07DC0109
:10E77000ED91FC9100ACF1ADE02D199580918F13D6
:10E78000882341F063EE78E180918D1390918E1390
:10E790000C94D34808958F929F92AF92BF92CF92DC
:10E7A000DF92EF92FF9285E40E940C4CBC01990F1E
:10E7B000880B990B0E9471C120E030E040E85AE3D9
:10E7C0000E94D0C120E030E040EA50E40E94D0C175
:10E7D0006B017C0180910E02882351F0C092981346
:10E7E000D0929913E0929A13F0929B1310920E021A
:10E7F00026E636E646E65FE360919813709199133A
:10E8000080919A1390919B130E94D0C14B015C019F
:10E8100020ED3CEC4CEC5DE3C701B6010E94D0C199
:10E820009B01AC01C501B4010E9412C3609398130F
:10E830007093991380939A1390939B132DE33CE26A
:10E8400048E450E40E94D0C12AE939E949E95EE38D
:10E850000E9412C3FF90EF90DF90CF90BF90AF90D7
:10E860009F908F90089580910D02882351F093DF3F
:10E8700020E030E040E050E40E946BC187FF39C0E7
:10E88000089589DF20E030E04AE754E40E94D0C1D7
:10E890000E94E3C320916F13309170134091B00731
:10E8A0006217730710F4442351F1442309F445C05F
:10E8B00072DF20E030E04AE754E40E94D0C10E94B9
:10E8C000E3C320916F133091701362177307A8F19F
:10E8D0001092B00781E08093AF0780918F13882357
:10E8E00061F16BEA78E180918D1390918E130C9415
:10E8F000D34810920D0281E08093AF07089581E024
:10E900008093B0071092AF0780918F13882391F006
:10E910006AEC78E180918D1390918E130E94AF483C
:10E920000E944A9567EC78E180918D1390918E1347
:10E930000E94D3480E94725CC7CB0895CF93DF93A7
:10E940008091070180FD2AC0C0914607D0914707FA
:10E9500080914A07882371F08EE30E940C4C81302D
:10E9600092402CF010924707109246070AC081E0AF
:10E9700090E003C08EE30E940C4C90934707809375
:10E98000460780914607909147078C179D0719F419
:10E990001092480703C081E080934807DF91CF9130
:10E9A0000895CF93DF938091070181FD2AC0C09124
:10E9B0004007D091410780914407882371F08FE38D
:10E9C0000E940C4C813092402CF010924107109222
:10E9D00040070AC081E090E003C08FE30E940C4C26
:10E9E00090934107809340078091400790914107A1
:10E9F0008C179D0719F41092420703C081E08093A1
:10EA00004207DF91CF9108952F923F924F925F92EC
:10EA10006F927F928F929F92AF92BF92CF92DF922E
:10EA2000EF92FF920F931F93CF93DF9300D01F922B
:10EA3000CDB7DEB75C010E94725C41DD77DD80916D
:10EA40008D1390918E130E94B7470E943F5724E088
:10EA5000A216B10409F49CC00CF04FC0A3E0AA16A2
:10EA6000B10409F03CC18CE190E00E94E4C49C83B5
:10EA70008B8383E696E0AB81BC8111969C938E9349
:10EA80001396BC92AE92129781E09FEF15969C93DD
:10EA90008E9314978FEF90E017969C938E93169712
:10EAA00019961C921E92189758961C925897CD0151
:10EAB0000E940F4287E596E0EB81FC819183808381
:10EAC000E091450FF091460FD08C009128111091E4
:10EAD000291116950795E0902611F0902711F694CC
:10EAE000E79463EF7AE180918D1390918E130E94E9
:10EAF000D348812C9924939412C1B5E0AB16B1048C
:10EB000009F4A6C0E6E0AE16B10409F0E8C08CE155
:10EB100090E00E94E4C49C838B8383E696E0AB8103
:10EB2000BC8111969C938E931396BC92AE921297D1
:10EB300081E09FEF15969C938E9314978FEF90E052
:10EB400017969C938E93169719961C921E9218975F
:10EB500058961C925897CD010E940F4287E596E087
:10EB6000EB81FC8191838083E0919B07F0919C076E
:10EB7000D08C009167111091681116950795E0905F
:10EB80006511F0906611F694E79466E27BE1A0C00F
:10EB90008CE190E00E94E4C49C838B8383E696E042
:10EBA000AB81BC8111969C938E931396BC92AE92CE
:10EBB000129781E09FEF15969C938E9314978FEF99
:10EBC00090E017969C938E93169719961C921E921E
:10EBD000189758961C925897CD010E940F4287E5CE
:10EBE00096E0EB81FC819183808300913D1110912F
:10EBF0003E1116950795E0903B11F0903C11F6946C
:10EC0000E7948091C5128C50823040F4E091AC07BB
:10EC1000F091AD07D08C66E67BE15AC080910E136F
:10EC2000823009F07AC08091C3128C3009F075C02F
:10EC3000E0919B07F0919C07D08C66E47BE180918A
:10EC40008D1390918E130E94D3488824839466C0BC
:10EC50008CE190E00E94E4C49C838B8383E696E081
:10EC6000AB81BC8111969C938E931396BC92AE920D
:10EC7000129781E09FEF15969C938E9314978FEFD8
:10EC800090E017969C938E93169719961C921E925D
:10EC9000189758961C925897CD010E940F4287E50D
:10ECA00096E0EB81FC8191838083E091A807F0914D
:10ECB000A907D08C00915211109153111695079508
:10ECC000E0905011F0905111F694E79466E07BE1EA
:10ECD00080918D1390918E130E94D3481EC06AEDCF
:10ECE0007AE180918D1390918E130F900F900F9079
:10ECF0000F90DF91CF911F910F91FF90EF90DF90D8
:10ED0000CF90BF90AF909F908F907F906F905F90CB
:10ED10004F903F902F900C94D348812C912C0E94BF
:10ED20003F576DEC7AE180918D1390918E130E9484
:10ED3000D34861EC7AE180918D1390918E130E94FB
:10ED4000AF48B80180918D1390918E130E94BD6CD5
:10ED500065EB7AE180918D1390918E130E94AF48FC
:10ED6000B70180918D1390918E130E94BD6C69EA5A
:10ED70007AE180918D1390918E130E94AF488D2D72
:10ED80000E94155780918D1390918E130E94B74762
:10ED9000AB81BC81ED91FC9111970280F381E02D54
:10EDA000CD011995CA2C8A2D0E942C418D3D95408C
:10EDB000A8F464E378E08A2D0E942441EB81FC8171
:10EDC000F78AE68AB70182810E943C416CED75E0CA
:10EDD0008A2D0E942841DD20C1F01AC064E873E04A
:10EDE0008A2D0E942841AB81BC8157961C930E93BB
:10EDF0005697B80112968C910E943C416CED75E0DB
:10EE00008A2D0E942441DD2019F03324339401C05F
:10EE1000312C21E02983212C2A830E9411618091C9
:10EE2000D110882359F1AB81BC81ED91FC911197F0
:10EE30006091D6107091D7100190F081E02DCD0136
:10EE400019958C2D0E942C418D3DB5E09B075CF4FB
:10EE50008438E3E09E0784F08C018D3D954074F08A
:10EE60000CED15E00BC07C01853398403CF064E369
:10EE7000E62E68E0F62E02C004E813E02A81211194
:10EE80001FC08091C7108823C9F1E091CE10F09186
:10EE9000CF10858196814091CA105091CB109C0172
:10EEA00021533109421753074CF1C1968417950736
:10EEB0002CF10E94B3846415750586059705F0F062
:10EEC0008091C7108823C1F04091CA105091CB1097
:10EED000E091CE10F091CF10858196819C01285C45
:10EEE0003109421753072CF088539F4F8417950719
:10EEF0001CF481E0382605C021E02A83222009F491
:10EF00007CC0332009F445C0DD20F9F064E873E0EB
:10EF10008C2D0E942841992009F458C06091DF127D
:10EF20007091E01241E08C2D0E94E3400E94E9972D
:10EF3000AB81BC8112968C910E942C410817190755
:10EF4000ACF38C2D0E94B54041C064E378E08C2D79
:10EF50000E9424419920B1F06091DF127091E0127B
:10EF600040E08C2D0E94E3400E94E997AB81BC8178
:10EF700012968C910E942C418E159F05ACF38C2D1E
:10EF80000E94B540EB81FC81F78AE68AB701828155
:10EF900010C0DD20B1F064E378E08C2D0E942441A4
:10EFA000AB81BC815796FC92EE925697B7011296B0
:10EFB0008C910E943C416CED75E08C2D0E942841A3
:10EFC00012C064E873E08C2D0E942841EB81FC8123
:10EFD000178B068BB80182810E943C416CED75E075
:10EFE0008C2D0E9424410E94B3842B013C01F8EC3B
:10EFF0004F0E511C611C711C1A8229812223D1F1F0
:10F000008091BD108823A1F14091C0105091C11092
:10F01000E091C410F091C510858196819C01285C17
:10F020003109421753072CF088539F4F84179507D7
:10F03000FCF481E0D82680918D1390918E13DD2011
:10F0400039F06AE97AE10E94D34882E090E006C094
:10F0500068E87AE10E94D34881E090E038DA0E94C3
:10F06000B384AB81BC815896DC922224239403C0E4
:10F07000212C1EC0212C8091BD10882309F48AC246
:10F08000E091C410F091C510858196814091C01027
:10F090005091C1109C0121533109421753070CF4C0
:10F0A00079C2C19621E02983841795070CF472C2B6
:10F0B0000E9422440E94056C8DE69CE00E94643F01
:10F0C0008091FA0B882309F4A8CE8091FC0B882349
:10F0D00009F4A3CE0E94056C0E948A6F8823D1F3A5
:10F0E00084E0A816B104D9F134F4B3E0AB16B1044E
:10F0F00009F438C1C4C1E5E0AE16B10409F4CDC0CD
:10F10000F6E0AF16B10409F0BAC11093D312009320
:10F11000D212F092D512E092D412D092D612B80147
:10F120008CE291E00E94986BB7018EE291E00E9420
:10F13000986B6D2D80E391E00E94F26CB80186E03F
:10F140000E945A40B70186E00E943F40E0919B0731
:10F15000F0919C07D08E6CED75E086E091C0882020
:10F16000C1F01093D3120093D212F092D512E09214
:10F17000D412D092D612B8018CE291E00E94986B22
:10F18000B7018EE291E00E94986B6D2D80E391E0D3
:10F1900017C01093C7120093C612F092C912E092E2
:10F1A000C812D092CA12B80180E291E00E94986B16
:10F1B000B70182E291E00E94986B6D2D84E291E0AC
:10F1C0000E94F26CB80184E00E945A40B70184E0CA
:10F1D0000E943F40882049F0E0919B07F0919C07F6
:10F1E000D08E6CED75E084E04BC0E091AC07F091FF
:10F1F000AD07D08E8091C5128D3029F4E091AE1309
:10F20000F091AF13D08E6CED75E084E00E943C412C
:10F2100066E970E080E090E00E94504C8091C51259
:10F220008D3011F584E00E942C41A091AC07B09183
:10F23000AD078D3D95404CF0ED91FC9111970190FB
:10F24000F081E02D6FEF7FEF08C0ED91FC911197F9
:10F250000190F081E02D61E070E0CD011995809181
:10F26000AC079091AD076FC08091AC079091AD074E
:10F27000DC01ED91FC910480F581E02D1995FFC032
:10F280000E943C4166E970E080E090E00E94504CB2
:10F2900080919B0790919C07EBCF1093CE12009327
:10F2A000CD12F092D012E092CF12D092D112B801CA
:10F2B00087E291E00E94986BB70189E291E00E9499
:10F2C000986B6D2D8BE291E00E94F26CB80185E0A5
:10F2D0000E945A40B70185E00E943F40E091A80794
:10F2E000F091A907D08E6CED75E085E00E943C415D
:10F2F00066E970E080E090E00E94504C8091C4127A
:10F300008D3059F585E00E942C41A091A807B0915D
:10F31000A9078D3D95404CF0ED91FC91119701901E
:10F32000F081E02D6FEF7FEF08C0ED91FC91119718
:10F330000190F081E02D61E070E0CD0119958091A0
:10F34000A8079091A907DC01ED91FC910190F08153
:10F35000E02D60E070E0199592C08091A80790912F
:10F36000A90786CF1093E2120093E112F092E41203
:10F37000E092E312D092DB12B8018BE391E00E949D
:10F38000986BB7018DE391E00E94986B6D2D85E33A
:10F3900091E00E94F26CB80183E00E945A40B701EC
:10F3A00083E00E943F408091DB12E091450FF09195
:10F3B000460F808F8091DB120E94636B83E00E9476
:10F3C0002C412091DB12222369F1B9E0BC1538F001
:10F3D00020912811309129113695279502C02EEEE3
:10F3E00032E08217930709F44AC06091DF127091EE
:10F3F000E01241E083E00E94E3400E94E997EB8144
:10F40000FC8182810E942C4108171907B4F383E024
:10F410000E94B540AB81BC8157961C930E935697C2
:10F42000B80129C0A9E0AC1508F4B6C02091261196
:10F4300030912711369527958217930701F1609136
:10F44000DF127091E01240E083E00E94E3400E94EE
:10F45000E997EB81FC8182810E942C418E159F05EA
:10F46000B4F383E00E94B540AB81BC815796FC9217
:10F47000EE925697B70112968C910E943C41809172
:10F480008D1390918E130E94B7470E943F57B4E0AE
:10F49000AB16B10499F03CF4F3E0AF16B10449F5B2
:10F4A0006CE07AE120C025E0A216B104D1F086E03C
:10F4B000A816B104F1F46CE37AE115C08091C5128D
:10F4C0008C50823018F46EE67AE10DC080910E13F4
:10F4D000823079F48091C3128C3059F465E57AE179
:10F4E00002C063E27AE180918D1390918E130E94A5
:10F4F000D3480E943F5761E07AE180918D1390914B
:10F500008E130E94D34865EF79E180918D1390911D
:10F510008E130E94AF48B80180918D1390918E1385
:10F520000E94BD6C69EE79E180918D1390918E13EC
:10F530000E94AF48B70180918D1390918E130E9465
:10F54000BD6C6DED79E180918D1390918E130E94C9
:10F55000AF488D2D0E94155780918D1390918E1379
:10F560000E94B7470F900F900F900F90DF91CF91AF
:10F570001F910F91FF90EF90DF90CF90BF90AF90D1
:10F580009F908F907F906F905F904F903F902F90C3
:10F590000C94927219828CCD2AEC38E04DCFCF9327
:10F5A000DF93CDB7DEB728970FB6F894DEBF0FBE56
:10F5B000CDBF8091AD138823D9F11092AD1329D816
:10F5C00081E0809303028091AE07882389F16EEC7D
:10F5D00079E180918D1390918E130E94AF48E09154
:10F5E000F60BE4300CF0E0E080EF95E09A8389833D
:10F5F0008CEE95E09C838B8387EE95E09E838D83D4
:10F6000082EE95E098878F83EE0FFF0BEC0FFD1FC6
:10F610006181728180918D1390918E1328960FB61F
:10F62000F894DEBF0FBECDBFDF91CF910C94D348CD
:10F6300028960FB6F894DEBF0FBECDBFDF91CF91F5
:10F6400008958091B0139091B11391609093B1138C
:10F650008093B01308958091D113811112C082E874
:10F660009AEAA1E0BB27ABBFFC016791769182E0EB
:10F670000E94754081E08093DD131092E113109297
:10F68000DE13089581E08093B6136CED75E00C9461
:10F6900075406CED75E080E00C94754081E20E944D
:10F6A000B24A21E0892B09F420E0822F089580914D
:10F6B0003207882309F44BC08091E10B882309F4B9
:10F6C00046C081E08093DE0BE9DF882329F080913A
:10F6D00035078823D9F106C080913307811105C011
:10F6E000809132070E94306831C090913207963085
:10F6F00069F5823081F08330D1F0813039F5E091C5
:10F70000460BF091470B74978081918145E550E05D
:10F7100060E070E017C0E091460BF091470B7497E2
:10F72000808191814AE550E060E070E00BC0E0919B
:10F73000460BF091470B7497808191814FE550E023
:10F7400060E070E08A5B944F0E948D51E4C508959B
:10F750008091E413882339F08091E313882319F012
:10F7600081E08093DB0B80911D0790911E07DC01E7
:10F77000ED91FC91008CF18DE02D19958091D713BE
:10F7800081110E94BD868091D613882391F061E09B
:10F7900088E00E94DA4A4091D4135091D51360E07A
:10F7A00070E02FE234E880911B0790911C070E94C3
:10F7B000543F8091E413882321F08091E313811159
:10F7C00001C075DF8091E313882379F08091E41301
:10F7D000882359F08091DA13882339F0E091D81307
:10F7E000F091D91382810E94C3400C943D8780918F
:10F7F000E00B811158C052DF8823F1F081E0809343
:10F80000E00B80911D0790911E07DC01ED91FC91AA
:10F810000488F589E02D19953ED62FE632E848E9AF
:10F820005AE360E070E080911B0790911C070E94F2
:10F83000543F0E943D870AC08091E313882339F129
:10F840008091E413882319F00E94278730CF0E940B
:10F8500011878091DA13882339F0E091D813F09161
:10F86000D91382810E94C3404091D2135091D31387
:10F8700014161506BCF4052E000C660B770B28EA4F
:10F880003BE780911B0790911C070C94543F80919B
:10F89000DA13882339F0E091D813F091D9138281DB
:10F8A0000E94C34055CF08950F931F932091D11309
:10F8B000211135C042E85AEA61E077279C01220F06
:10F8C000331F820F931F092E000CAA0BBB0B02964D
:10F8D000A11DB11D840F951FA61FB71FABBFFC0153
:10F8E000879102E81AEA21E033274091E11393E07F
:10F8F000499FA0011124052E000C660B770B4E5F6B
:10F900005F4F6F4F7F4F040F151F261F371F2BBFF1
:10F91000F8010791801718F01F910F919CCE1F914D
:10F920000F910895833091F028F4813049F08230AE
:10F9300051F00895853081F060F0863081F00895AF
:10F9400089E090E00EC08AE090E00BC08BE090E090
:10F9500008C08CE090E005C08DE090E002C08EE031
:10F9600090E0A2CF8F929F92AF92BF92CF92DF9200
:10F97000EF92FF920F931F93CF93DF93EC01A62E8C
:10F980008091D11381116BC042E85AEA61E0772778
:10F990006E01CC0CDD1CCC0EDD1E0D2C000CEE0817
:10F9A000FF08D701C6010296A11DB11D480F591FBE
:10F9B0006A1F7B1F6BBFFA01879142E85AEA61E038
:10F9C0007727B090E11393E0B99E80011124012EB6
:10F9D000000C220B330B0E5F1F4F2F4F3F4F400F7A
:10F9E000511F621F731F6BBFFA014791481708F040
:10F9F00036C08090DF139090E0130091CA131091ED
:10FA0000CB13B401C8010E94ED3E882321F0B4015C
:10FA1000C8010E94053F82E89AEAA1E0BB278C0D4D
:10FA20009D1DAE1DBF1DABBFFC016791769182E0AD
:10FA30000E947540B092DE13C093E113AA2079F0C2
:10FA40001092DD132BE23BE742E350E060E070E010
:10FA5000C8010E94543F9093E0138093DF13DF911D
:10FA6000CF911F910F91FF90EF90DF90CF90BF90BB
:10FA7000AF909F908F900895CF92DF92EF92FF9278
:10FA80008091D113811134C08091D013882381F1EA
:10FA900061E08EE090E066DF6091CE137091CF134D
:10FAA000CB01A0E0B0E0C090CC13D090CD13E12CFE
:10FAB000F12CC816D906EA06FB0664F4BC01CD0198
:10FAC0006C197D098E099F090E944B47C60ED71EEF
:10FAD000E81EF91E2CE33DE7B701A6018091CA1389
:10FAE0009091CB130E94543F9093C9138093C813F5
:10FAF000FF90EF90DF90CF900895CF92DF92EF923A
:10FB0000FF928091D113811134C08091C713882353
:10FB100081F161E08DE090E025DF6091C513709187
:10FB2000C613CB01A0E0B0E0C090C313D090C413C3
:10FB3000E12CF12CC816D906EA06FB0664F4BC01D8
:10FB4000CD016C197D098E099F090E944B47C60E95
:10FB5000D71EE81EF91E2DE73DE7B701A6018091EB
:10FB6000CA139091CB130E94543F9093C213809379
:10FB7000C113FF90EF90DF90CF900895CF92DF9266
:10FB8000EF92FF928091D113811134C08091C01304
:10FB9000882381F161E08CE090E0E4DE6091BE13A7
:10FBA0007091BF13CB01A0E0B0E0C090BC13D09027
:10FBB000BD13E12CF12CC816D906EA06FB0664F445
:10FBC000BC01CD016C197D098E099F090E944B472C
:10FBD000C60ED71EE81EF91E2EEB3DE7B701A601A3
:10FBE0008091CA139091CB130E94543F9093BB1302
:10FBF0008093BA13FF90EF90DF90CF90089580919B
:10FC0000D11381112CC08091B913882341F08091C8
:10FC1000C013811104C081E08093C013AFDF8091D5
:10FC2000B813882361F08091D113811108C08091AD
:10FC3000C713811104C081E08093C7135EDF8091F8
:10FC4000B713882361F08091D113811108C080918E
:10FC5000D013811104C081E08093D0130DCF08959B
:10FC60001092B61322E43BE744EF51E060E070E00D
:10FC70008091CA139091CB130E94543F9093B51377
:10FC80008093B41308958091D11381110AC080919B
:10FC9000B613882331F060ED77E081E00E94754073
:10FCA000DFCF08950F931F93CF93DF93EC017093F1
:10FCB000CB136093CA134093D11381E090E00E946C
:10FCC000E4C48C010E940F421093DC130093DB13F9
:10FCD00091E09093B6139093DD131092B5131092A8
:10FCE000B4131092E0131092DF131092E1131092EC
:10FCF000DE131092B31324EF31E03093BD13209341
:10FD0000BC1328EB3BE03093BF132093BE1320E2DB
:10FD100033E03093C4132093C3132CEA3DE03093B7
:10FD2000C6132093C51328E037E03093CD132093FA
:10FD3000CC1324E931E13093CF132093CE131092EA
:10FD4000B9131092B8131092B7131092C0131092F7
:10FD5000C7131092D0131092B2131092BB131092CB
:10FD6000BA131092C2131092C1131092C9131092B9
:10FD7000C813988399839A83DF91CF911F910F9134
:10FD8000089508950895089508950895623039F00A
:10FD9000633041F0613041F44093B91308954093CA
:10FDA000B81308954093B7130895623069F0633033
:10FDB000A1F06130D1F45093BD134093BC13309344
:10FDC000BF132093BE1308955093C4134093C313DD
:10FDD0003093C6132093C51308955093CD134093C9
:10FDE000CC133093CF132093CE130895FC0185815B
:10FDF000089508950895089508952091D11321112B
:10FE000002C0FC01628308952091D113211102C028
:10FE1000FC01648308952091D113211102C0FC01DB
:10FE200063830895089508958091D113811101C0CD
:10FE300029CC0895089580E00895089508950895BF
:10FE40000895089508958091D113811103C08FE022
:10FE500090E02ACD08952091D113211107C0FC0113
:10FE60008481882319F082E090E01ECD08952091CE
:10FE7000D113211107C0FC018381882319F081E08F
:10FE800090E012CD08958091D113811103C08BE0D1
:10FE900090E00ACD08958091D113811104C060E0F3
:10FEA00080E190E05FCD08958091D113811104C06D
:10FEB00060E08FE090E056CD08958091D1138111DC
:10FEC00026C06330A1F028F4613049F0623059F067
:10FED00008956530A1F078F06630A9F0089560E0EB
:10FEE00089E090E013C060E08AE090E00FC060E03D
:10FEF0008BE090E00BC060E08CE090E007C060E039
:10FF00008DE090E003C060E08EE090E02BCD08959E
:10FF10008091D113811126C06330A1F028F46130A3
:10FF200049F0623059F008956530A1F078F06630FC
:10FF3000A9F0089561E089E090E013C061E08AE0F3
:10FF400090E00FC061E08BE090E00BC061E08CE0DE
:10FF500090E007C061E08DE090E003C061E08EE0DA
:10FF600090E000CD08952091D113211108C0FC012B
:10FF70008281882321F061E088E090E0F3CC08954D
:10FF80002091D113211108C0FC018481882321F024
:10FF900061E082E090E0E6CC08952091D113211138
:10FFA00008C0FC018381882321F061E081E090E0BA
:10FFB000D9CC08958091D113811104C061E086E00D
:10FFC00090E0D0CC08958091D113811104C060E0FD
:10FFD0008BE090E0C7CC08958091D113811104C0CB
:10FFE00061E087E090E0BECC08958091D11381114B
:10FFF00004C061E085E090E0B5CC08958091D11314
:020000021000EC
:10000000811104C061E08AE090E0ACCC0895CF9308
:10001000DF93FC0125812223A1F1EC018091D11312
:1000200081112EC06091BA137091BB138091CA13D5
:100030009091CB130E94053F1092C0138091D11371
:1000400081110CC06091C1137091C2138091CA13C9
:100050009091CB130E94053F1092C7138091D1134A
:1000600081110CC06091C8137091C9138091CA139B
:100070009091CB130E94053F1092D0131092B213AF
:100080001D82DF91CF910895CF93DF93FC012581ED
:1000900021111EC0EC018091D113811117C08091F4
:1000A000B213811113C02FEF3DE748EB5BE060E036
:1000B00070E08091CA139091CB130E94543F9093AB
:1000C000BB138093BA1381E08093B21381E08D83D8
:1000D000DF91CF910895862F9091D113911101C096
:1000E00021CC0895CF93C1E08091D113811102C03A
:1000F0008C2F18DCCF5FC730B9F7CF91089580916E
:10010000D113882329F06CED75E081E00C947540E3
:1001100084E090E0C9CB8091D113882329F068EE68
:1001200073E081E00C94754060E084E090E01ACCCC
:100130008091D11381111BC08091B6138823B9F02F
:1001400068EE73E081E00E9475401092B61322E4DD
:100150003BE748E95AE360E070E08091CA13909170
:10016000CB130E94543F9093B5138093B41308951A
:100170006CED75E080E00C94754024EF31E0DB011C
:100180000E94DEC42FEF30E040E050E00E94B4C295
:10019000CA01B90164527A4F8F4F9F4F80E00C948F
:1001A00075408091D113882331F060ED77E081E0D4
:1001B0000E94754055CD61E083E090E0D3CB209163
:1001C000D113211108C02091B313222321F00296EC
:1001D0005ADD1092B31308952091D113222389F090
:1001E0006FE676E080E00E94754029E43BE742E359
:1001F00050E060E070E08091CA139091CB130C94B2
:10020000543F2091B313211105C002963CDD81E0DB
:100210008093B313089580E00E949C4081E00E9487
:100220009C408091D113811103C082E00E949C40C8
:100230006CED75E080E00E9475406CED75E081E04A
:100240000E9475408091D11381110CC082E89AEA16
:10025000A1E0BB27ABBFFC016791769182E00E94D1
:100260007540F9C90895FC01848595859783868337
:1002700086859785918780878089918993878287F2
:10028000808D918D938B828B828D938D958B848BBA
:10029000848D958D978B868B0895FC01808991893B
:1002A00093878287828993899587848784899589B2
:1002B00097878687089526E00C944D4A8091120214
:1002C000882311F0599801C0599A9091120281E047
:1002D00089278093120208951092A5111092230786
:1002E00010921A07109224071092250710922607E1
:1002F0001092270781E08093DE0B40912E075091EA
:100300002F0760E070E02BE831E880911B079091A7
:100310001C070C94543F8091E10B882361F180917C
:10032000DF0A81111CC01092210B1092220B109237
:10033000230B1092240B1092250B1092260B109277
:10034000290B8091DC0B9091DD0BDC01ED91FC9190
:100350000190F081E02D19951092DE0B08952BE8A5
:1003600031E845E050E060E070E080911B0790913B
:100370001C070C94543F08956091EF137091F01393
:1003800080911B0790911C070E94ED3E882319F075
:1003900081E08093EE13089560E087E00E94DA4ADE
:1003A0001092DF0B089561E087E00E94DA4A81E055
:1003B0008093DF0B0895CF93DF938091FC1381111D
:1003C00010C084EF91E09093FB138093FA138BE2BB
:1003D00090E09093F9138093F81381E08093FC13DD
:1003E00020C08091F8139091F9138532910514F093
:1003F000049709C08331910514F0029704C082303C
:1004000091052CF001979093F9138093F813809144
:10041000F8139091F91397FF04C01092F9131092FA
:10042000F813C091F713CC2311F0B6DF01C0BBDF86
:1004300081E08C278093F713C091FA13D091FB13BE
:100440001C161D0654F01092FC13A6DF2BE432E8B4
:100450004AEF50E060E070E007C02BED31E8AE01FC
:100460000D2E000C660B770B80911B0790911C07DB
:100470000E94543F9093F6138093F5138091F813E4
:100480009091F913C81BD90BD093FB13C093FA13A7
:10049000DF91CF9108950F931F93CF93DF938091B6
:1004A000E00B882329F0DF91CF911F910F9183CF2B
:1004B0000091F5131091F613C0911B07D0911C0702
:1004C000B801CE010E94ED3E882321F0B801CE0193
:1004D0000E94053FDF91CF911F910F915DCFCF9289
:1004E000DF92EF92FF921092E00B20911F07309164
:1004F00020074091210750912207609124077091B5
:10050000250780912607909127070E9411C36B0150
:100510007C0120E030E0A9010E946BC187FD09C089
:10052000C0922407D0922507E0922607F092270771
:1005300008C01092240710922507109226071092E7
:100540002707FF90EF90DF90CF90A5CFEF92FF921B
:100550001F93CF93DF9300D0CDB7DEB784E68983B6
:100560008CE38A8388E28B831091F1131330E8F4D3
:10057000E12EF12C10FF02C00FDF01C014DFE1E01B
:10058000F0E0EC0FFD1FEE0DFF1D408150E060E03C
:1005900070E026EA32E880911B0790911C070E94C8
:1005A000543F1F5F1093F11303C0F6DE1092F11356
:1005B0000F900F900F90DF91CF911F91FF90EF90D0
:1005C00008958091DF0B882311F0E6DE01C0EBDE99
:1005D0009091DF0B81E089278093DF0B08950F93C3
:1005E0001F93CF93DF939091F4138091A5119111F4
:1005F0002AC0882309F44FC00091F2131091F3131D
:10060000C0911B07D0911C07B801CE010E94ED3E9E
:10061000882321F0B801CE010E94053FC4DE2FEEF1
:1006200032E842EC51E060E070E080911B0790916D
:100630001C070E945C3F9093F3138093F21381E0B8
:100640008093F41353C0882329F0DF91CF911F9139
:100650000F91B7CF8091DF0B8823B9F36091F2132C
:100660007091F31380911B0790911C070E94053F26
:100670002FEE32E844E150E060E070E080911B072B
:1006800090911C070E945C3F9093F3138093F213A8
:100690001092F4132BC0C0911302D0911402229730
:1006A000D0931402C09313021C161D0674F4BE01ED
:1006B000772787E00E94454BCC2321F081E080938F
:1006C000DF0B14C01092DF0B11C06091F213709118
:1006D000F31380911B0790911C070E94053F5CDE7D
:1006E0008FEF90E09093140280931302DF91CF91EB
:1006F0001F910F9108950F931F93CF93DF93009154
:10070000EA131091EB13C091EC13D091ED13C00FCD
:10071000D11FD093ED13C093EC13BE01772787E070
:100720000E94454BCC2321F081E08093DF0B02C077
:100730001092DF0B10161106ECF58091E8139091E2
:10074000E913C817D9070CF485C08091EE138823EC
:1007500071F01092E9131092E8138CEF9FEF9093D1
:10076000EB138093EA1381E08093E71373C068E78B
:1007700070E080E090E00E944B47DC01CB010A96DC
:10078000A11DB11D9093E9138093E81368E270E016
:1007900080E090E00E944B47DC01CB010A96A11D4E
:1007A000B11D66277727681B790B7093EB13609355
:1007B000EA1350C0012B09F44DC08091E8139091C9
:1007C000E9138C179D070CF445C08091E71388232B
:1007D00011F10091EF131091F013C0911B07D0910C
:1007E0001C07B801CE010E94ED3E882399F1B801A3
:1007F000CE010E94053FD0DD1092ED131092EC1354
:100800001092E7138091A511882321F1DF91CF91F8
:100810001F910F91E4CE69E670E080E090E00E94C5
:100820004B47DC01CB018A569F4FAF4FBF4F909390
:10083000E9138093E81368E270E080E090E00E94A2
:100840004B47DC01CB010A96A11DB11D9093EB1320
:100850008093EA13DF91CF911F910F91089560E08B
:1008600088E00C94DA4A61E089E20C94DA4A0F934A
:100870001F93CF93DF9360E08BE20E94DA4A0091EE
:10088000E5131091E613C0911B07D0911C07B80126
:10089000CE010E94ED3E882341F0B801CE01DF91E8
:1008A000CF911F910F910C94053FDF91CF911F9134
:1008B0000F91089580913707882361F08091E10BB3
:1008C000882341F081E08093DE0B809136070E94FF
:1008D000306821CD0895CF93DF93CDB7DEB765970C
:1008E0000FB6F894DEBF0FBECDBF81E08093E20B60
:1008F0008091E213882371F182E390E09A838983E7
:1009000088E290E09C838B838EE690E09E838D83CB
:1009100084EF91E098878F831D8A84E08F938DB751
:100920009EB745970FB6F8949EBF0FBE8DBFADB76B
:10093000BEB7119685E1FE01319601900D928A9520
:10094000E1F78CEE9AE00E9439930FB6F894DEBF7F
:100950000FBECDBF65960FB6F894DEBF0FBECDBFFC
:10096000DF91CF9108952FB7F8946091FE137091A5
:10097000FF1380910014909101142FBF08951F92CE
:100980000F920FB60F9211242F933F938F939F9343
:10099000AF93BF938091FE139091FF13A091001429
:1009A000B09101143091FD1323E0230F2D3720F473
:1009B0000196A11DB11D05C026E8230F0296A11DB9
:1009C000B11D2093FD138093FE139093FF13A0930A
:1009D0000014B09301148091050F9091060FA0911F
:1009E000070FB091080F0196A11DB11D8093050F4F
:1009F0009093060FA093070FB093080FBF91AF918C
:100A00009F918F913F912F910F900FBE0F901F904C
:100A100018950F931F93CF93DF930091F5131091C7
:100A2000F613C0911B07D0911C07B801CE010E949C
:100A3000ED3E8823A1F0B801CE010E94053F2CEBCA
:100A400031E848EB5BE060E070E080911B0790913B
:100A50001C070E94543F9093F6138093F513609106
:100A6000EF137091F01380911B0790911C070E9467
:100A7000ED3E81114BC01092EE138FEF90E09093FA
:100A8000ED138093EC138FDC68E770E080E090E07A
:100A90000E944B47DC01CB010A96A11DB11D90932A
:100AA000E9138093E81368E270E080E090E00E9430
:100AB0004B47DC01CB010A96A11DB11D66277727A4
:100AC000681B790B7093EB136093EA132BE733E801
:100AD00044E150E060E070E080911B0790911C07BA
:100AE0000E945C3F9093F0138093EF132CEB31E85E
:100AF00048EB5BE060E070E080911B0790911C0781
:100B00000E94543F9093F6138093F513DF91CF9199
:100B10001F910F9108958F929F92AF92BF92CF92A3
:100B2000EF92FF920F931F93CF93DF93209139079A
:100B3000223008F078C07B018C01809024079090CF
:100B40002507A0902607B090270720E030E0A901F4
:100B5000C501B4010E946BC1181654F520E030E0C5
:100B6000A901C501B4010E940FC4181654F420E075
:100B700030E048E452E4C501B4010E946BC118168C
:100B8000D4F420E030E048E452E4C501B4010E940E
:100B90000FC418169CF420E030E048EC52E4C50184
:100BA000B4010E946BC187FF09C0CBE4D0E008C04C
:100BB000C0E0D0E005C0C2E3D0E002C0C4E6D0E0AF
:100BC0008FEF8C0D823068F4209739F06C2FC801BC
:100BD0000E94CE4D6C2FC7010CC0C8015EDBC7015F
:100BE00016C08DEF8C0D8330F0F4209779F06C2FC8
:100BF000C801DF91CF911F910F91FF90EF90CF909F
:100C0000BF90AF909F908F900C94CE4DC801DF9114
:100C1000CF911F910F91FF90EF90CF90BF90AF9029
:100C20009F908F903ACBDF91CF911F910F91FF90C2
:100C3000EF90CF90BF90AF909F908F9008958F923C
:100C40009F92AF92BF92CF92DF92EF92FF92C090AD
:100C50002407D0902507E0902607F090270720E092
:100C600030E0A901C701B6010E940FC420E030E0C6
:100C700040E05FE387FD0BC0C701B6010E9412C3CD
:100C80004B015C010E94DEC397FD27C010C0C70165
:100C9000B6010E9411C30E94DEC397FD1EC06536D7
:100CA000710581059105DCF424E6822F14C0C5018D
:100CB000B4010E94DEC365367105810591057CF49F
:100CC00020E030E040E05FE3C701B6010E9412C3BC
:100CD0000E94DEC384E6861B03C084E601C080E078
:100CE000FF90EF90DF90CF90BF90AF909F908F904C
:100CF00008950F931F93CF93DF93009114071091E2
:100D00001507C0911B07D0911C07B801CE010E94A6
:100D1000ED3E882321F0B801CE010E94053F80916D
:100D2000E00B882339F01092E00BDF91CF911F91F7
:100D30000F91B1CBDF91CF911F910F910895EC9856
:100D40001092E10B68EC70E082E00C946567809192
:100D50003207811105C080913607811101C0EFCFA4
:100D60008091DC0B9091DD0B0E94799581E080935E
:100D7000E10B64E670E00C94656760E089E20E9434
:100D8000DA4A23E334E842E350E060E070E0809127
:100D90001B0790911C070C94543F1F920F920FB6A3
:100DA0000F9211240BB60F922F933F934F935F93A3
:100DB0006F937F938F939F93AF93BF93EF93FF9323
:100DC0008091E4138823B1F0489918C0E89827E38C
:100DD00034E84CE251E060E070E080911B079091B4
:100DE0001C070E94543F8091E313882339F00E942E
:100DF000A87B04C0489B02C0E89839DDFF91EF91C1
:100E0000BF91AF919F918F917F916F915F914F9122
:100E10003F912F910F900BBE0F900FBE0F901F9020
:100E2000189561E08BE20E94DA4AE89A27E334E8F9
:100E300048E853E160E070E080911B0790911C0747
:100E40000E94543F9093E6138093E513089561E068
:100E50008BE20E94DA4AE89A27E334E848E853E153
:100E600060E070E080911B0790911C070E94543F46
:100E70009093E6138093E51308951092E20B40914E
:100E80002C0750912D0760E070E02BE634E880914C
:100E90001B0790911C070C94543F8091B0139091C4
:100EA000B11380689093B1138093B013089580912B
:100EB000B0139091B11380619093B1138093B013EC
:100EC0000895FC018281882371F08381882359F081
:100ED00013828091B0139091B11324E082279093F4
:100EE000B1138093B0130895FC018281882371F0BF
:100EF000838181110BC081E083838091B013909135
:100F0000B11384609093B1138093B0130895FC01E2
:100F10008481882371F08581882359F0158280911E
:100F2000B0139091B11328E082279093B11380936E
:100F3000B0130895FC018481882371F085818111AB
:100F40000BC081E085838091B0139091B1138860CC
:100F50009093B1138093B01308958091B013909142
:100F6000B11320E282279093B1138093B0130895B8
:100F70008091B0139091B11380629093B1138093DC
:100F8000B0130895DC01ED91FC910680F781E02D0E
:100F900060E070E0199477FF03C071956195710965
:100FA0006F3F710519F014F06FEF70E08091B0138E
:100FB0009091B1138C7B91709093B1138093B01387
:100FC0008091B0139091B1136F30710514F4806467
:100FD0001FC06733710514F481641AC06F35710541
:100FE0001CF48164906114C0673871051CF481643D
:100FF00090630EC06F3A71051CF48164906408C060
:10100000673D71051CF48164906502C0816490663F
:101010009093B1138093B013089580E094E090937F
:10102000B1138093B01308958091B0139091B113D0
:1010300092609093B1138093B0130895089508952A
:1010400008950895089508950895089508950895B8
:1010500080E00895089508950895089508950895E5
:101060000895089508950895089508950895089598
:1010700008950895089508950895089580E00895C5
:10108000089508950895FC0164830895FC01628326
:101090000895FC011382148215821682178210862D
:1010A00011860895089508950895FC018381089597
:1010B000FC0165830895FC0164830895FC01608749
:1010C0000895FC0166830895FC0112821382148244
:1010D000158261E086E10E94094B61E086E10E9491
:1010E000DA4AE2E7F0E08081816080831092B113F8
:1010F0001092B01308951F920F920FB60F92112401
:101100000BB60F920F931F932F933F934F935F93C1
:101110006F937F938F939F93AF93BF93EF93FF93BF
:1011200080910A148F5F80930A1490910914891793
:1011300008F42EC110920A148091081490E08730B0
:10114000910508F025C1FC018827E155FE4F8F4F1E
:101150000C94D0C460E086E10E94DA4A80E4809377
:10116000091481E048C061E086E10E94DA4A88E023
:101170008093091436C060E086E10E94DA4A8091CB
:1011800006149091071497FF05C088E18093091415
:1011900084E031C088E08093091483E02CC061E0D2
:1011A00086E10E94DA4A88E180930914809105144F
:1011B0008F5F80930514803150F01092051485E004
:1011C0001AC061E086E10E94DA4A88E0EDCF8091A2
:1011D000061490910714880F991F90930714809319
:1011E000061482E008C060E086E10E94DA4A88E0E6
:1011F0008093091486E080930814CAC061E086E1F8
:101200000E94DA4A80EC809309148091B013909187
:10121000B11390930714809306148091B0139091AA
:10122000B11391FF1CC080910414882369F0809150
:10123000B0139091B11322E092279093B113809351
:10124000B013109204140BC081E0809304148093B7
:1012500003148093021486E69BE00E9458678091F5
:1012600002148823C9F0809103148823A9F07BDB42
:101270000091660B1091670B2091680B3091690B00
:10128000DC01CB01801B910BA20BB30B8D3690427E
:10129000A105B10508F070C08091B0139091B11311
:1012A00092FF12C080910414882339F01092B11378
:1012B0001092B0131092041407C081E080930414BC
:1012C00010920314109202148091B0139091B113F4
:1012D00084FF14C080910414882369F08091B013B6
:1012E0009091B11320E182279093B1138093B013B2
:1012F0001092041403C081E0809304148091B01311
:101300009091B11387FF13C080910414882361F07A
:101310008091B0139091B11380589093B113809342
:10132000B0131092041403C081E0809304148091E0
:10133000B0139091B11390FF14C0809104148823CE
:1013400069F08091B0139091B11321E092279093AE
:10135000B1138093B0131092041403C081E0809302
:1013600004148091B0139091B1139093071480935B
:101370000614109208140CC0109202148091B0133D
:101380009091B11380649093B1138093B01384CF84
:10139000FF91EF91BF91AF919F918F917F916F914D
:1013A0005F914F913F912F911F910F910F900BBE25
:1013B0000F900FBE0F901F901895FF920F931F93E1
:1013C000CF93DF938C01C62FF42ED22F6AED70E0FD
:1013D000DC011A968D919C911B9755D5F801828559
:1013E0009385DC01ED91FC910190F081E02D6C2F53
:1013F0001995F80182859385DC01ED91FC910190AE
:10140000F081E02D6F2D1995F80182859385DC011F
:10141000ED91FC910190F081E02D6D2F1995EC2F4D
:10142000F0E0BF0166527F4F6F0D711D6D0F711D92
:101430006F777727F80182859385DF91CF911F9190
:101440000F91FF9020C520E040E0B7CF65E4FBCFCF
:1014500068E4F9CFCF93DF93FC012381222321F0AD
:10146000EC0161E4F0DF1B82DF91CF910895CF930F
:10147000DF93FC012381211105C0EC0160E4E3DF6F
:1014800081E08B83DF91CF91089563E5DCCFFC0190
:101490002581222311F060E5D6CF0895FC01248137
:1014A000222311F06CE3CFCF0895FC012085222385
:1014B00031F02185222319F011866BE3C4CF089502
:1014C000FC012085222339F02185211104C021E06F
:1014D00021876AE3B8CF0895FC012681222331F0E9
:1014E0002781222319F0178269E3ADCF0895FC010B
:1014F0002681222339F02781211104C021E027838E
:1015000068E3A1CF089567E39ECF6AE49CCF69E4C6
:101510009ACF66E398CF65E396CF6EE494CF64E309
:1015200092CF63E390CF242F462F6CE446CF462F13
:1015300020E067E442CF462F20E066E43ECF262F2E
:1015400064E43BCFCF92DF92FF920F931F93CF9330
:10155000DF938C01F62E443F81E0580738F041318B
:1015600087E2580728F040E157E202C044EF51E01B
:10157000243F81E0380738F0E9012131374228F073
:10158000C0E1D7E202C0C4EFD1E0CA01845F91405C
:1015900022E3C22ED12CB6010E94A9C4462F2F2DC2
:1015A00062E4C8010ADFCE01845F9140B6010E9467
:1015B000A9C4462F2F2D63E4C801DF91CF911F915D
:1015C0000F91FF90DF90CF90F8CE242F462F62E549
:1015D000F4CE242F462F61E5F0CE262F40E06FE3B6
:1015E000ECCE262F40E06EE3E8CE262F40E06DE300
:1015F000E4CE462F20E06FE4E0CE08950895FC018C
:10160000828193818830910529F410922B011092E8
:101610002A010895099721F41092290110922801B6
:101620000895FC01178A168A6CED75E082810C948E
:101630003C41CF93DF93EC011F8A1E8A8A810E946E
:10164000B5408B8D882331F08A810E942C419A8F7E
:10165000898F1B8EDF91CF910895DF92EF92FF92D9
:101660000F931F93CF93DF93EC018A81893010F49D
:101670000E949C40DD8C6B8D7C8D098D1A8DEA80DB
:10168000FB8089E08E1508F466C00F30110538F034
:1016900001369DE6190728F000E61DE602C00FE0BE
:1016A00010E06F30710538F061368DE6780728F06C
:1016B00060E67DE602C06FE070E080E090E00E94AE
:1016C0006FC120E030E04AE754E40E9476C320E096
:1016D00030E04CE852E40E94D0C19B01AC0160E0D4
:1016E00070E08AEF94E40E9476C30E94DEC3FF2478
:1016F00025E12E9DF0012F9DF00D1124EC51FF4EA0
:10170000DD2071F023813481AB0177FF04C04427D1
:101710005527461B570B88279927841B950B0AC012
:1017200025813681AB0177FF04C044275527461B2E
:10173000570BCA014FB7F89455E15E9DF0015F9DCC
:10174000F00D1124EC51FF4E108B0787328B218B4B
:10175000948B838B4FBF9D8D6B8D7C8D8A8199235C
:10176000F9F08A3058F495E1899FF0011124EC5189
:10177000FF4E058116811695079502C00EEE12E008
:1017800041E00E94E34061E070E080E090E00E9470
:10179000504C8A810E942C4108171907A0F31EC0E3
:1017A0008A3058F495E1899FF0011124EC51FF4EE5
:1017B000038114811695079502C00AEC18E040E0F9
:1017C0000E94E34061E070E080E090E00E94504CB5
:1017D0008A810E942C4180179107A0F38A810E9480
:1017E000B540B8018A81DF91CF911F910F91FF9091
:1017F000EF90DF900C943C41CF93DF93EC018A8112
:10180000893010F40E949C4048EE53E05B874A8781
:1018100020ED37E03D872C878CED95E09F878E8704
:10182000598B488B3B8B2A8B9D8B8C8BDF91CF9177
:101830000895CF93DF93EC017F8B6E8B888599851C
:101840006817790769F48A810E94B5408B8D8823D7
:1018500029F18A810E942C419A8F898F1B8E1EC08C
:10186000CE010E945F4EEA81EA30B0F49C01C3973A
:1018700014F022E330E02E3C8FEF380714F42EEC06
:101880003FEF8FB7F89495E1E99FF0011124EC51F7
:10189000FF4E318720878FBF81E08B8FDF91CF9103
:1018A00008950F931F93CF93DF938C01FC01778BE7
:1018B000668B0E945F4EEC01F80182819381883033
:1018C0009105D1F4D7FF06C060E08AE00E94DA4AB1
:1018D00061E005C061E08AE00E94DA4A60E086E0EB
:1018E0000E94DA4AD7FF03C0D195C195D109D093A0
:1018F0002B01C0932A011BC00997C9F4D7FF06C06A
:1019000060E08DE00E94DA4A61E005C061E08DE0B0
:101910000E94DA4A60E08BE00E94DA4AD7FF03C0F7
:10192000D195C195D109D0932901C0932801DF91A8
:10193000CF911F910F910895CF93DF93EC018A818E
:10194000893010F40E949C402EEC3FEF3B872A87A1
:1019500082E390E09D878C871F861E86398B288BBB
:101960009B8B8A8B1D8A1C8A6EEE72E08A810E9494
:1019700028416AEC78E08A810E9424418CED95E050
:101980009A8F898F1B8EDF91CF910895CF93DF932C
:10199000EC0121E03FEF3B872A878FEF90E09D87A6
:1019A0008C871F861E86398B288B9B8B8A8B1D8A82
:1019B0001C8A61E08AE00E94094B61E086E00E9497
:1019C000094B61E08DE20E94094B61E08DE00E94CD
:1019D000094B61E08BE00E94094B61E08EE20E94BE
:1019E000094B8A819B818830910529F410922B0143
:1019F00010922A0106C0099721F410922901109231
:101A00002801DF91CF9108950F931F93CF93DF9318
:101A1000EC010E94B3840C8D1D8D2E8D3F8DDC0159
:101A2000CB01801B910BA20BB30B853F9140A1050D
:101A3000B10548F06E897F89CE01DF91CF911F916A
:101A40000F910C94D84EDF91CF911F910F91089573
:101A50000F931F93CF93DF938C01FC01178A168A93
:101A6000EC01699640E068E0CE010E946D9E4FE770
:101A700066E0CE010E946D9E40E06CE0CE010E94C7
:101A80006D9E4FE767E0CE010E946D9E0E94B38479
:101A9000F801648F758F868F978FDF91CF911F919B
:101AA0000F9108956F927F928F929F92AF92BF9203
:101AB000CF92DF92EF92FF920F931F93CF93DF931A
:101AC0008091AA149091AB14DC01ED91FC910084FB
:101AD000F185E02D1995B12C181619060CF0D1C01E
:101AE000AA24A3948091AA149091AB14DC01ED91E7
:101AF000FC910084F185E02D1995892B09F4C1C072
:101B0000C0916D1481E08C0F80936D148091AA14A4
:101B10009091AB14DC01ED91FC910284F385E02DF2
:101B20001995EC2FF0E0E35DFB4E80838A30D1F60F
:101B3000E0906D14F12C1092BA0E1092B90E109222
:101B4000B50E1092B60E1092B70E1092B80E1092FB
:101B5000B40E1092B30E1092B20E8DE2C82E84E134
:101B6000D82E00E010E0D0E0C0E00E151F050CF00C
:101B70006CC0F60191916F019D3009F463C09C37F0
:101B800089F19A3009F052C0D33009F059C0CC2302
:101B900009F456C06C2E712CC30101970E943F6F4F
:101BA0007093BA0E6093B90E0E94B3846093AD1423
:101BB0007093AE148093AF149093B01480910B1473
:101BC000882309F45BC08090B90E9090BA0EB801DA
:101BD000661977098DE294E10E94B09F88169906F4
:101BE00079F54CC08C2F90E0FC01EC54F04F108242
:101BF000D13099F068F0D230B1F40E943F6F609319
:101C0000B50E7093B60E8093B70E9093B80E0BC0BE
